:020000040800F2
:1000000000000120453E0408913E0408C5C90108CE
:10001000913E0408913E0408913E0408000000004F
:10002000000000000000000000000000913E0408F5
:10003000913E040800000000913E04089DFE010866
:10004000913E0408913E0408913E0408913E040844
:10005000913E0408913E0408B9030208E504020831
:10006000A90402086D040208310402080D220108E7
:10007000FD210108ED210108DD210108CD21010844
:10008000B9210108A5210108913E0408913E040808
:10009000913E0408913E0408913E0408F5030208CD
:1000A000913E0408913E0408913E0408913E0408E4
:1000B000D5110108C5110108913E04084D2201081F
:1000C000592201083522010841220108913E040805
:1000D000913E0408A1070108913E04089507010814
:1000E0007F030208913E0408913E0408913E0408F3
:1000F000C1110108913E0408B111010891210108C4
:10010000913E0408913E0408913E0408913E040883
:10011000913E0408913E0408913E0408EDF0020867
:100120007D210108692101085521010841210108AB
:100130002D210108913E0408913E0408913E0408D7
:10014000913E0408913E0408913E0408D15F0308E3
:100150001921010805210108F1200108890701087A
:100160001D22010829220108913E0408913E04083D
:10017000913E0408913E0408913E040800000000EE
:10018000913E0408913E0408913E0408913E040803
:10019000913E0408913E0408913E0408913E0408F3
:1001A0000000000000000000913E0408913E040899
:1001B000913E0408913E0408913E0408913E0408D3
:0801C000913E0408913E040881
:1001C80002020300941E0120901E0120000000007E
:1001D80000000000270004007C2201207C2301206D
:1001E800000000003C0600081600080080230120DB
:1001F8008823012000000000400600081500700058
:10020800AC260120FC2B01200000000000000000AB
:1002180003000100A82601206C2C0120000000002A
:10022800000000002A006000B8250120702C012081
:10023800000000000D15020829005000943001202C
:100248009C3401200000000000000000140002009F
:1002580090300120EC34012000000000480600081E
:1002680013000400E4360120F036012000000000ED
:100278004C06000810000300E0360120F436012087
:10028800000000005006000828000C00D4360120A9
:10029800F836012000000000540600082300100072
:1002A800C43601200437012000000000D9480208A4
:1002B80019000500BC360120143701200000000099
:1002C80060060008F8110100B83601201C3701202B
:1002D800000000006606000800010400B436012092
:1002E8002037012000000000680600082F001100D8
:1002F800A036012024370120000000006C06000809
:100308000B201000843A0120BC3A012000000000B4
:100318007E0600081F000E00F8370120CC3A0120A5
:10032800000000008E060008050201004C3801207C
:10033800DC3A0120000000009C0600081E000400B2
:10034800183C01204C3F0120000000009E060008D8
:1003580022000C009C3B0120503F012000000000BF
:10036800A206000826000E006C3F01205C3F012019
:1003780000000000C5C5020804008000746F012059
:10038800747101200000000000000000F901040061
:1003980000520120F47101200000000075F50108E9
:1003A8000301060048720120847201200000000049
:1003B800AE0600080312330003740120D073012035
:1003C80000000000B406000825005A001C73012034
:1003D800767301200000000000000000F6110C00F8
:1003E800107301200473012000000000E8060008D3
:1003F800012008000C75012058750120000000003C
:10040800F40600081A000800F47401206075012041
:1004180000000000FC06000801010400B875012076
:10042800EC870120000000000000000008020C001A
:100438008A870120F08701200000000085F5010867
:100448000602100096870120FC87012000000000AA
:1004580059F8010807020200D48701200C880120FE
:100468000000000004070008FF010100E8870120E0
:1004780010880120000000000607000802000C0098
:10048800A887012014880120000000000000000057
:10049800F701060084870120208801200000000061
:1004A8000807000809020100D48801202C890120CE
:1004B800000000000E07000812100B0054880120ED
:1004C8003089012000000000100700080C002400FB
:1004D800648801203C890120000000004D9F03082A
:1004E8000002050034880120608901200000000016
:1004F800000000000A020A008C9701209C97012046
:10050800000000001C07000818102C000CAB01208C
:1005180054AB01200000000099F00308FD012400FD
:10052800E8AA012080AB01200000000001F50108C5
:10053800FB010100B4AA0120A4AB012000000000C7
:1005480001B90108FC01090080A90120A8AB01201C
:1005580000000000CDB801080A10120054A90120BB
:10056800B4AB0120000000002607000806001600B2
:1005780038990120C8AB01200000000039010308A8
:1005880034001000A8970120E0AB01200000000013
:10059800411402080D003400DCB0012010B1012024
:1005A80000000000516E0308FA01020070AD01203E
:1005B80044B101200000000025B90108FE0108002F
:1005C8004CAC012048B101200000000009B9010825
:1005D8002C0010004CB401203CB4012000000000A5
:1005E800FDED03082B00240080B401205CB4012039
:1005F80000000000CDED03080500060068B60120E4
:10060800A4B6012000000000380700080E20EA0008
:100618004CB50120ACB601200000000035150208D9
:100628000201030039B5012098B70120000000003D
:04063800E91E0308AC
:10063C0020030000C4090000190128280300000051
:10064C00080000000001050000000001000000008F
:10065C0000000000000028010000040090010000D0
:10066C00000000000000000000000000000000007E
:10067C0000002B21231E64010200000001000A016E
:10068C00290000000000000001000000000500002F
:10069C00000000000100C800141E010064002C01C1
:1006AC002800040101000000000000000000000010
:1006BC00000000000000000000000000000000002E
:1006CC00000000000000000000000000000000001E
:1006DC00000000000000000000000100000000000D
:1006EC000000000000000000E8036400040A0001A0
:1006FC007E05EA05B4053200013C00004A01000009
:10070C000000390000000001004659463700000087
:10071C0000004A01B400D601000000300100005A6C
:10072C000000000090012C01C800640020000200B1
:02073C000100BA
:10073E000101000078A00408E4BF040800000000D6
:10074E000000000088A0040890A00408000000002B
:10075E000120000094A004089CA0040800000000E2
:10076E0001400000A0A00408D8B204080000000058
:10077E0001200000ACA00408B8A00408000000008E
:10078E0004000000BCA00408C8A00408000000007B
:10079E0004000000CCA00408BCCD0408000000003A
:1007AE0001000000020100000000803F0000803FB9
:1007BE00FF000000FFFFFFFF7D4E0208000000005B
:1007CE000000000000010101010000003030303057
:1007DE002D30312D30315430303A30303A30300007
:1007EE00010100000000803FE8BF04080000000087
:1007FE0000000000F91E0308A0860100040000009E
:10080E0000000000000000000000000000000000DA
:10081E000000000000000000000000009CBA040868
:10082E00D0B8040800000000D16B01087D00000064
:10083E0006000000000000000000000000000000A4
:10084E00000000000000000000000000000000009A
:10085E00F0BF04080000000000000000E51C0408C2
:10086E00E80300000300000000000000000000008C
:10087E00000000000000000000000000000000006A
:10088E0000000000F8BF0408000000000000000097
:10089E0051020308102700000300000000000000B2
:1008AE00000000000000000000000000000000003A
:1008BE00000000000000000044D104080000000009
:1008CE0085EC0308A1D10108204E000005000000B0
:1008DE00000000000000000000000000000000000A
:1008EE000000000000000000000000006CC60408BC
:1008FE0000000000000000007D1704081027000013
:10090E0001000000000000000000000000000000D8
:10091E0000000000000000000000000000000000C9
:10092E0004C00408000000000000000099B801088F
:10093E00E8030000050000000000000000000000B9
:10094E000000000000000000000000000000000099
:10095E000000000010C004080000000000000000AD
:10096E001D210308204E00000300000000000000BF
:10097E000000000000000000000000000000000069
:10098E00000000000000000020C00408000000006D
:10099E0000000000291F0308204E00000300000085
:1009AE000000000000000000000000000000000039
:1009BE0000000000000000000000000030C004082D
:1009CE00000000000000000005150408400D0300A3
:1009DE000300000000000000000000000000000006
:1009EE0000000000000000000000000000000000F9
:1009FE0040C004080000000000000000D17F030882
:100A0E0010270000010000000000000000000000A0
:100A1E0000000000000000000000000000000000C8
:100A2E0000000000ECB80408000000000000000008
:100A3E00F1D502081027000003000000000000009E
:100A4E000000000000000000000000000000000098
:100A5E00000000000000000048C004080000000074
:100A6E000000000041540308A086010001000000B0
:100A7E000000000000000000000000000000000068
:100A8E0000000000000000000000000054C0040838
:100A9E000000000000000000B1250108A00F0000BA
:100AAE000100000000000000000000000000000037
:100ABE000000000000000000000000000000000028
:100ACE0060C0040800000000000000008DB00208A5
:100ADE0010270000010000000000000000000000D0
:100AEE0000000000000000000000000000000000F8
:100AFE0000000000C4B80408000000000000000060
:100B0E0021E003081A41000001000000000000006F
:100B1E0000000000000000000000000000000000C7
:100B2E0000000000000000006CC00408000000007F
:100B3E00000000002D6E0308400D030000000000B1
:100B4E000000000000000000000000000000000097
:100B5E0000000000000000000000000074C0040847
:100B6E000000000000000000E96D0308400D0300C6
:100B7E000000000000000000000000000000000067
:100B8E000000000000000000000000000000000057
:100B9E007CC00408000000000000000025230308AC
:100BAE00A08601000300000000000000000000000D
:100BBE000000000000000000000000000000000027
:100BCE000000000000C201000000080000FFFF004E
:100BDE0000000000AA5505010000AA5507010000FB
:100BEE00AA5503009FAA550B010000AA5509020041
:100BFE000000000001000000C01200000000803F55
:100C0E0074970408050804000000000024A00408DE
:100C1E00C09F04086097040800000000A097040815
:100C2E0005080A000000000024A00408C09F040864
:100C3E00809A0408000000000A060002000000402E
:100C4E000100000009074300020104C0320904003C
:100C5E00000102020100052400100105240100011B
:100C6E00042402020524060001070582030800FF82
:100C7E0009040100020A00000007050102400000FD
:100C8E00070581024000000009024300020100C076
:100C9E0032090400000102020100052400100105C2
:100CAE002401000104240202052406000107058226
:100CBE000308001009040100020A000000070501E4
:100CCE000200020007058102000200000902430033
:100CDE00020100C0320904000001020201000524D5
:100CEE00001001052401000104240202052406005F
:100CFE00010705820308001009040100020A000022
:100D0E0000070501024000000705810240000000B7
:100D1E001A030000000000000000000000000000A8
:100D2E0000000000000000000000000004030904A1
:100D3E00120100020200004083044057000201022B
:100D4E0003010000655F0308595F0308995F0308FC
:100D5E00AD5F0308115F0308855F0308715F030829
:100D6E000139030841380308BD460308000000009E
:100D7E0091350308ED350308B9350308000000006E
:100D8E0000000000000000007935030885350308D7
:100D9E006D35030861350308DDE1020855E00208F0
:100DAE0009E00208F9DF020800E6DF0C010000008E
:100DBE00006002401060024000000000000B0000C6
:100DCE000000200000000000000000000060024053
:100DDE002860024000000000060C00000000200009
:100DEE000000000000000000006002404060024071
:100DFE0000000000100D00000000200000000000A8
:100E0E000000000000600240586002400000000038
:100E1E00160E000000002000000000000000000080
:100E2E00006002407060024000000000200F0000D1
:100E3E0000002000000000000000000000600240E2
:100E4E008860024000000000261000000000200014
:100E5E00000000000000000000600240A0600240A0
:100E6E000000000030110000000020000000000013
:100E7E000000000000600240B86002400000000068
:100E8E00362F0000000020000000000000000000CF
:100E9E0000640240106402400000000000380000B0
:100EAE00000040000000000000000000006402404E
:100EBE0028640240000000000639000000004000D7
:100ECE000000000000000000006402404064024088
:100EDE0000000000103A000000004000000000007A
:100EEE000000000000640240586402400000000050
:100EFE00163B000000004000000000000000000053
:100F0E00006402407064024000000000203C0000BB
:100F1E0000004000000000000000000000640240DD
:100F2E0088640240000000002644000000004000DB
:100F3E00000000000000000000640240A0640240B7
:100F4E0000000000304500000000400000000000DE
:100F5E000000000000640240B8640240000000007F
:100F6E0036460000000040000000000000000000B7
:100F7E000000000100000000000000000000000062
:100F8E006CD504080E0000000000000000000000F8
:100F9E0000000000BC150120FFFFFFFFFA0000005B
:100FAE00010000000100000004D004080000000051
:100FBE00000000000000000000000000F9CF04084F
:100FCE0004000000192804080000000000000000C2
:100FDE000CD004080100000000000000000000001A
:100FEE0000000000000000000D00000000000000E6
:100FFE0000000000000000005E7001200100C40926
:10100E00000000005C7001200100C4090000000017
:10101E005A7001200100C409000000005870012020
:10102E000100C40900000000547001200100C40931
:10103E0000000000567001200100C40900000000ED
:10104E00527001200100C409000000005070012000
:10105E000100C4090000000030D004080E0000009A
:10106E0000000000000000000000000078080120D1
:10107E00447201209CFF2C01000000007616012016
:10108E000A000000809A040824B50120E0150C1710
:10109E00000000007516012008000000C09F040823
:1010AE00741601200500000024A0040826B50120B6
:1010BE0002000000989A04086EB601200100FF7F1E
:1010CE000100000066B6012002000000A49A040888
:1010DE0040B5012003000000B49A04083FB501207A
:1010EE0003000000B49A04083EB601200000F4018B
:1010FE00010000003CB601200000F40101000000D8
:10110E003AB601200000F4010100000038B60120BB
:10111E000000F4010100000036B6012000FF0100BE
:10112E0052B60120E803D0070A00000050B6012095
:10113E00006401000A00000051B6012000640100A5
:10114E000A0000004AB60120006401000A000000F7
:10115E004FB60120006401000A0000004EB60120C7
:10116E00006401000A0000004DB601200064010079
:10117E000A00000049B6012000FF01000A0000002D
:10118E0048B6012000FF01000A00000048B501200A
:10119E000000F4010100000046B501200000F4013A
:1011AE000100000044B501200000F4010100000020
:1011BE0042B501200000F4010100000045B60120F7
:1011CE0000C8010044B6012000C8010043B601204A
:1011DE0000C8010042B60120006401000A000000B0
:1011EE0041B6012000FF01000A0000005DB601209B
:1011FE0000C801005CB6012000C801005BB60120EA
:10120E0000C801005AB6012000C8010059B60120DD
:10121E0000C8010058B6012000C8010057B60120D1
:10122E0000C8010056B6012000C8010055B60120C5
:10123E0000C8010038D004080000000000000000C3
:10124E00000000000000000048D004080900000063
:10125E00000000001C0901200400000050D004080A
:10126E000900000000000000100901200400000029
:10127E0014D4040809000000000000000409012035
:10128E000400000064CF0408090000000000000004
:10129E00F80801200400000058D0040809000000DE
:1012AE0000000000EC0801200400000060D00408DB
:1012BE000900000000000000E0080120040000000A
:1012CE0068D004080900000000000000D4080120C6
:1012DE000400000070D004080900000000000000A7
:1012EE00C8080120040000000CD004080100000012
:1012FE0000000000000000000000000000000000E0
:10130E000D000000000000000000000000000000C2
:10131E0054D104080000000000000000000000008E
:10132E0000000000E4BF0408000000000000000000
:10133E00641801200400000060CF04080C000000B7
:10134E00612804087C09012000000000ACD80408C4
:10135E000C000000ED2304087009012000000000BD
:10136E0060D104080C000000B923040864090120B0
:10137E000000000068D10408080000000000000012
:10138E00580901200400000070D104080C00000070
:10139E00A52304084C0901200000000078D10408A0
:1013AE0009000000000000004009012004000000B8
:1013BE0080D1040803000000F1DE03082809012093
:1013CE00000000000CD00408010000000000000026
:1013DE000000000000000000000000000D000000F2
:1013EE0000000000000000000000000084D104088E
:1013FE0000000000000000000000000000000000DF
:10140E0094D104080C000000000000009409012093
:10141E00000000009CD104080A000000000000003B
:10142E007FB6012000000000A8D104080A000000C9
:10143E000000000087B6012000000000B0D10408B3
:10144E000A000000000000008FB60120000000001E
:10145E00B8D104080800000000000000880901202F
:10146E0000000000C0D1040804000000F92C04089C
:10147E0000000000000000000CD004080100000075
:10148E00000000000000000000000000000000004E
:10149E000D00000000000000000000000000000031
:1014AE00CCD1040800000000000000000000000085
:1014BE0000000000E0D104080C0000000000000055
:1014CE00AC09012000000000F0D104080400000067
:1014DE00C52A04080000000000000000F8D104082E
:1014EE000C00000000000000A00901200000000018
:1014FE000CD2040804000000A52A04080000000015
:10150E00000000000CD004080100000000000000E4
:10151E000000000000000000000000000D000000B0
:10152E0000000000000000000000000014D20408BB
:10153E00000000000000000000000000000000009D
:10154E0028D204080700000000000000E80901206E
:10155E000000000034D20408080000000000000063
:10156E00DC0901200000000040D204080800000041
:10157E0000000000D0090120000000004CD2040839
:10158E000800000000000000C40901200000000057
:10159E0058D204080800000000000000B80901201D
:1015AE00000000000CD00408010000000000000044
:1015BE000000000000000000000000000D00000010
:1015CE0000000000000000000000000064D20408CB
:1015DE0000000000000000005F1801200000000065
:1015EE0070D204080B00000000000000500A012019
:1015FE000000000078D204080B000000000000007C
:10160E00440A01200000000084D204080B000000F0
:10161E0000000000380A01200000000090D20408EB
:10162E000B000000000000002C0A0120000000004A
:10163E009CD204080B00000000000000200A0120CC
:10164E0000000000A8D204080B00000000000000FB
:10165E00140A012000000000B0D204080B000000A4
:10166E0000000000080A012000000000BCD204089F
:10167E000B00000000000000FC090120000000002B
:10168E00C8D204080800000000000000F009012084
:10169E00000000000CD00408010000000000000053
:1016AE000000000000000000000000000D0000001F
:1016BE00000000000000000000000000D4D204086A
:1016CE00000000000000000000000000000000000C
:1016DE00E8D204080800000000000000800A012083
:1016EE0000000000F4D20408080000000000000012
:1016FE00740A01200000000000D304080800000056
:10170E0000000000680A0120000000000CD304084D
:10171E0008000000000000005C0A0120000000002C
:10172E000CD00408010000000000000000000000C2
:10173E0000000000000000000D000000000000008E
:10174E00000000000000000014D304080000000098
:10175E00000000005C1801200000000024D30408E3
:10176E000B00000000000000B00A01200000000085
:10177E0030D304080B00000000000000A40A012072
:10178E00000000003CD30408070000000000000029
:10179E009C0A01200000000048D304080700000046
:1017AE0000000000940A01200000000054D3040839
:1017BE0007000000000000008C0A0120000000005D
:1017CE000CD0040801000000000000000000000022
:1017DE0000000000000000000D00000000000000EE
:1017EE00000000000000000060D3040800000000AC
:1017FE00000000005C180120000000006CD30408FB
:10180E000700000000000000FC0A0120000000009C
:10181E0074D304080700000000000000F40A012041
:10182E00000000007CD30408070000000000000048
:10183E00EC0A01200000000084D304080700000019
:10184E0000000000E40A0120000000008CD3040810
:10185E000700000000000000DC0A0120000000006C
:10186E0094D304080700000000000000D40A0120F1
:10187E00000000009CD304080700000000000000D8
:10188E00CC0A012000000000A4D3040807000000C9
:10189E0000000000C40A012000000000ACD30408C0
:1018AE000700000000000000BC0A0120000000003C
:1018BE000CD0040801000000000000000000000031
:1018CE0000000000000000000D00000000000000FD
:1018DE000000000000000000B4D304080E00000059
:1018EE00000000007925040800000000040B012010
:1018FE003EB5012017000000C49A04083DB5012032
:10190E000A3201003CB5012001FA010038B5012070
:10191E0000C8010036B50120E803D0070100000021
:10192E004655525946370000BCD304080E0000003D
:10193E00052304080000000000000000E00B012059
:10194E00C4D304080E000000D92C0408B1270408E3
:10195E00AD270408BC0C0120CCD304080E000000F7
:10196E008F2504080000000000000000700D01200B
:10197E00D4D304080E0000001D260408ED2504082B
:10198E0000000000FC0D0120DCD304080E00000056
:10199E0099260408E1260408000000009C0E012090
:1019AE0046B6012001030100E8D304080E00000032
:1019BE00C12504089D250408000000008C0F01209D
:1019CE00F0D304080E0000004D260408E52A040892
:1019DE000000000018100120FCD304080E000000C7
:1019EE0011270408312B040800000000B810012054
:1019FE0040B601200103010004D4040800000000D9
:101A0E0000000000000000000000000010D40408D8
:101A1E000800000000000000E4110120000000009A
:101A2E0018D404080700000000000000DC1101209B
:101A3E000000000028D40408070000000000000089
:101A4E00D41101200000000034D404080700000067
:101A5E0000000000CC1101200000000040D404085A
:101A6E000C00000000000000C0110120000000006A
:101A7E004CD4040803000000F1DE0308A811012075
:101A8E00000000000CD0040801000000000000005F
:101A9E000000000000000000000000000D0000002B
:101AAE0000000000000000000000000054D40408F4
:101ABE000000000000000000000000000000000018
:101ACE0064D404080A00000000000000D8A0040836
:101ADE00000000006CD404080A00000000000000A2
:101AEE0058A004080000000074D404080A00000086
:101AFE00000000005EB60120000000007CD4040847
:101B0E000A00000000000000F0110120000000009B
:101B1E000CD00408010000000000000000000000CE
:101B2E0000000000000000000D000000000000009A
:101B3E00000000000000000084D404080000000033
:101B4E0000000000000000000000000098D404080F
:101B5E0003000000F1DE0308101201200000000057
:101B6E00A4D4040803000000F1DE03087816012057
:101B7E0000000000ACD4040803000000F1DE0308EE
:101B8E00F8110120000000000CD004080100000034
:101B9E000000000000000000000000000000000037
:101BAE000D0000000000000000000000000000001A
:101BBE00B4D4040800000000000000000000000083
:101BCE0000000000C0D40408070000007D2B0408AC
:101BDE00C0120120000000009CBA0408030000009F
:101BEE00F1DE0308A812012000000000CCD4040886
:101BFE0003000000F1DE0308901201200000000037
:101C0E00D4D4040803000000F1DE0308781201208A
:101C1E0000000000DCD4040807000000612B04085B
:101C2E007012012000000000C8D804080300000054
:101C3E00F1DE03085812012000000000E8D4040869
:101C4E0003000000F1DE0308401201200000000036
:101C5E00F4D4040803000000F1DE0308281201206A
:101C6E00000000000CD0040801000000000000007D
:101C7E000000000000000000000000000D00000049
:101C8E0000000000000000000000000000D5040865
:101C9E000E0000004125040809250408000000007C
:101CAE00C812012008D504080E0000008127040880
:101CBE0000000000000000007C13012014D5040871
:101CCE000E000000000000000000000000000000F8
:101CDE000814012024D504080E000000592704081A
:101CEE00992B040800000000801401202CD5040854
:101CFE0000000000000000000000000000000000D6
:101D0E0068CF040803000000F1DE0308A4150120CB
:101D1E000000000018D5040803000000F1DE0308DF
:101D2E008C1501200000000038D5040803000000C7
:101D3E00F1DE0308741501200000000044D50408EC
:101D4E0003000000F1DE03085C1501200000000016
:101D5E004CD5040802000000FDDD03080000000061
:101D6E000000000054D5040802000000FDDD030849
:101D7E00010000000000000060D504080200000011
:101D8E00FDDD03080200000000000000000000005E
:101D9E000D00000000000000000000000000000028
:101DAE0001010000010101004CD904080E000000E1
:101DBE00412404080000000000000000F817012074
:101DCE0020D9040800000000000000000000000000
:101DDE0000000000E4BF0408000000000000000046
:101DEE008418012004000000ACD804080C00000088
:101DFE00FD290408981C01200000000060D1040891
:101E0E000C000000CD2904088C1C012000000000ED
:101E1E0068D104080800000000000000801C0120AA
:101E2E000400000070D104080C000000E52804082E
:101E3E00741C01200000000080D104080300000083
:101E4E00F1DE03085C1C01200000000030D90408FC
:101E5E0003000000F1DE0308441C01200000000016
:101E6E000CD004080100000000000000000000007B
:101E7E0000000000000000000D0000000000000047
:101E8E00000000000000000020D90408000000003F
:101E9E00000000000000000000000000E4BF040885
:101EAE000000000000000000841801200400000063
:101EBE0058D8040803000000892804082C1C0120AF
:101ECE000800000070D104080C000000E52804088A
:101EDE00741C01200000000080D1040803000000E3
:101EEE00F1DE03085C1C01200000000030D904085C
:101EFE0003000000F1DE0308441C01200000000076
:101F0E000CD00408010000000000000000000000DA
:101F1E0000000000000000000D00000000000000A6
:101F2E00000000000000000038D904080000000086
:101F3E00000000000000000000000000E4BF0408E4
:101F4E0000000000000000008418012004000000C2
:101F5E0060D8040803000000F1DE0308A41C012071
:101F6E00000000000CD0040801000000000000007A
:101F7E000000000000000000000000000D00000046
:101F8E000000000000000000000000002070002093
:101F9E00702D72002D202D2D202D2D2D2D202D2D2F
:101FAE002D2D0000000000000000000000000000C9
:101FBE00000000002D202D2D202D2D2D2D202D2D1E
:101FCE002D000000000000000000000000000000D6
:101FDE000000000032B5012088130C17010000002C
:101FEE0034B5012088130C1700000000B0D7040888
:101FFE0000000000000000000000000000000000D3
:10200E00C0D704080800000000000000B01801202E
:10201E0004000000CCD704080800000000000000F7
:10202E00A41801200000000080D104080400000064
:10203E00C928040800000000000000000CD00408AD
:10204E000100000000000000000000000000000081
:10205E00000000000D000000000000000000000065
:10206E000000000030B5012088130C17010000009D
:10207E002EB5012088130C170000000008D80408A4
:10208E000E0000009924040800000000000000006B
:10209E00BC1801207EB6012001000000E49F040858
:1020AE002DB5012001000000F09F04087A72012076
:1020BE0002000000F89F04083A70012000000000A2
:1020CE000000000038700120000000000000000039
:1020DE003670012000000000000000003470012066
:1020EE00000000000000000032700120000000001F
:1020FE000000000030700120000000000000000011
:10210E00C804012000000000000000002CB50120D2
:10211E000200000004A0040810D80408000000000B
:10212E00000000000000000000000000C0D70408FE
:10213E00080000000000000040190120040000000B
:10214E00CCD704080800000000000000341901205C
:10215E000000000080D10408040000007924040867
:10216E0000000000000000000CD004080100000078
:10217E000000000000000000000000000000000051
:10218E000D00000000000000000000000000000034
:10219E0020D804080000000000000000000000002D
:1021AE000000000030D804080C0000006D2904085F
:1021BE007C190120040000003CD804080C0000002B
:1021CE00BD240408701901200400000048D804083A
:1021DE000C0000002D2904086419012000000000E5
:1021EE0054D8040803000000A92804084C19012043
:1021FE000800000060D8040803000000F1DE0308A8
:10220E00A41C0120000000000CD0040801000000F6
:10221E0000000000000000000000000000000000B0
:10222E000D00000000000000000000000000000093
:10223E0004D00408000000000000000000000000B0
:10224E000000000068D80408040000002D2A0408CD
:10225E0000000000000000000CD004080100000087
:10226E000000000000000000000000000000000060
:10227E000D00000000000000000000000000000043
:10228E00B4D80408000000000000000000000000A8
:10229E000000000054C704080C00000000000000FD
:1022AE00DC19012004000000C4D804080800000056
:1022BE0000000000D019012004000000D0D804084E
:1022CE000800000000000000C419012004000000F6
:1022DE00D8D804080800000000000000B81901203A
:1022EE0004000000E0D80408080000000000000010
:1022FE00AC19012004000000E8D804080800000012
:10230E0000000000A019012004000000F0D804080D
:10231E0008000000000000009419012004000000D5
:10232E00F8D80408080000000000000088190120F9
:10233E00040000000CD004080100000000000000A2
:10234E000000000000000000000000000D00000072
:10235E0000000000000000000000000000D904088A
:10236E000E00000089240408000000000000000098
:10237E00E819012008D904080E0000000000000032
:10238E000000000000000000601A012010D90408AF
:10239E000E00000000000000000000000000000021
:1023AE00001B01207DB601200400000010A00408CF
:1023BE0028B50120E0150C17000000002BB50120F8
:1023CE0008000000C09F04082AB501200500000087
:1023DE0024A0040818D904080E0000000000000014
:1023EE000000000000000000501B01204300000010
:1023FE0000000000000000000000000000000000CF
:10240E00000000000000000000000000430000007B
:10241E0000000000000000000000000000000000AE
:10242E00000000000000000000000000430000005B
:10243E00000000000000000000000000000000008E
:10244E00000000000000000000000000430000003B
:10245E00000000000000000000000000000000006E
:10246E00000000000000000000000000430000001B
:10247E00000000000000000000000000000000004E
:10248E0000000000000000000000000043000000FB
:10249E00000000000000000000000000000000002E
:1024AE0000000000000000000000000043000000DB
:1024BE00000000000000000000000000000000000E
:1024CE00000000000000000000000000ED470408BE
:1024DE00454604080000000068D90408F4CF04083B
:1024EE0070BE040870BE040870BE040870BE0408F6
:1024FE0070BE040870BE040870BE040870BE0408E6
:10250E0070BE0408FFFFFFFFFFFFFFFFFFFFFFFF8F
:10251E00FFFF000001004153434949000000000045
:10252E00000000000000000000000000000000009D
:10253E000000000000004153434949000000000024
:10254E00000000000000000000000000000000007D
:10255E0000000000000000002C1E01200000000002
:10256E00000000000000000000000000000000005D
:10257E00000000000000000000000000000000004D
:10258E00000000000000000000000000000000003D
:10259E00000000000000000000000000000000002D
:1025AE00000000000000000000000000000000001D
:1025BE00000000000000000000000000010000000C
:020000040801F1
:10000000012250F8043CA0F1100180F849200BB106
:1000100008461847704700BF4FF4006303837047DA
:10002000D0F8F020034630B46AB1C168D0F8082196
:100030004469881A013A205C08BF0A46C0B2C3F876
:10004000082130BC7047006A5D69411CDC68285C8F
:10005000A14228BF1146C0B2196230BC704700BF30
:10006000D0F8F43013B190F888017047836A406A81
:10007000181AB0FA80F04009704700BF416A836ADD
:1000800099420ED3CB1AD0F8F410026981B1D0F89E
:100090007411501E0A685268134483420BD2C01A6E
:1000A000704702691144CB1AD0F8F4100029EED140
:1000B000501EC01A70470020704700BFD0F8F030C3
:1000C0006BB1D0F87831D0F808211B685B68934297
:1000D00001D3981A7047C068801A18447047C269E3
:1000E000036A9A4203D2C0681044C01A7047D01AFB
:1000F000704700BFBFF34F8F0549064BCA6802F433
:10010000E0621343CB60BFF34F8F00BFFDE700BF3A
:1001100000ED00E00400FA05704700BF70B582B042
:100120000446856A06236A463B210830A847A8B1E1
:100130009DF8003001209DF801109DF8026041EA11
:1001400003219DF803209DF804509DF8053042EAF4
:100150000622618343EA0523A283E38302B070BDD4
:10016000F8B590F87D3190F87E21134303F0210318
:10017000212B0FD0436A846AA3420CD80269002362
:10018000121B92B290F87D1100258362202980F81D
:10019000885103D0F8BD1A1B92B2F3E78369E3429A
:1001A00003EB0401F6D0B2FA82F46409002CF1D119
:1001B00090F87C31012BEDD005460127A0F866218F
:1001C0001346A0F864214FF0210ED0F87461C0F8F6
:1001D0006011C0F88041304685F87C710C4A0D4FA3
:1001E00085F87DE1F76332640B4FD5F8142134654F
:1001F0002832F76418F01CFDD5F8143140221A6239
:1002000085F87C419A6842F080029A60C2E700BF9C
:100210009D810208D981020835810208426A10B422
:100220008469A154426A04690132D0F8F410A242F0
:1002300028BF0022426241B10B68DB0702D55DF89E
:10024000044B70475DF8044B8AE7D0F814215DF841
:10025000044B136843F0800313607047406990308B
:1002600018F04EBAF8B544695C4D6601321B05EBD7
:10027000C2077B8903EB42031E3355F8230018F0B5
:100280003FFA7B68DA79587953070BD40C2800F2CF
:100290009580DFE800F03E939393479393935093B8
:1002A000939313000C2800F28E80DFE800F07E8C20
:1002B0008C8C758C8C8C6C8C8C8C4D00331B05EB72
:1002C000C3039B6DDA6822F48052DA6001211A6A56
:1002D000434F8140BB4222EA01021A621A6A1A6243
:1002E00076D0404A934273D0196A41F211121142FA
:1002F00008D1196A40F24442114203D11A6822F02F
:1003000001021A60341B012305EBC40585F8953002
:10031000F8BD331B05EBC3039B6DDA6822F4007252
:10032000DA60D3E7331B05EBC3039B6DDA6822F475
:100330008062DA60CAE7331B05EBC3039B6DDA68A2
:1003400022F40062DA60C1E7331B05EBC3039B6D47
:10035000DA6822F48052DA6004211A6A41F2111735
:10036000814022EA01021A621A6A1A621A6A3A4241
:10037000BAD1196A40F244421142B5D15A6C22F402
:1003800000425A64B0E7331B05EBC3039B6DDA6888
:1003900022F40062DA60DFE7331B05EBC3039B6DD9
:1003A000DA6822F48062DA60D6E7331B05EBC30318
:1003B0009B6DDA6822F40072DA60CDE7331B05EB3F
:1003C000C3039B6D82E7331B05EBC3039B6DC3E740
:1003D000196A41F21112114286D1CAE760990120CF
:1003E0000000014000040140F8B5D0F81431044683
:1003F000DA69910614D5586AE36AC0B2002B00F09E
:10040000A1809847D4F814311A6822F480721A60D7
:100410009A6822F001029A609A6942F008029A6191
:10042000DA69D20701D501221A62DA69970701D584
:1004300002221A62DA69560701D504221A62DA69C1
:10044000150701D508221A62D4F8F420002A00F01A
:100450008580D969490600D4F8BDD96904F58A7048
:100460001E680F079D6818D18F0602D5B50600F1EA
:10047000F0800F0602D5350600F1CD80480602D582
:10048000710600F1A780002AE6D0626AA36A9A4248
:100490007DD1012384F88831F8BD15F001057AD1AA
:1004A00016F4907FE5D011F0010700F0D08016F42B
:1004B000807774D13D4605EA91073FB104271F625A
:1004C000D4F8807147F00207C4F880710F070AD58D
:1004D000B70640F18E8008251D62D4F8805145F0A2
:1004E0000805C4F88051D4F88051002DCBD08F0678
:1004F00005D5B50603D517F08FFFD4F81431D4F81D
:10050000802111076ED51A68202122F490721A609A
:100510009A6822F001029A6084F87E119A68520665
:100520000DD59A68D4F8781122F040029A6031B162
:10053000564B08460B6518F0B7F900285DD1D4F882
:10054000F420A0E7E3696269D054E369E16801330C
:10055000B3FBF1F201FB1233E36153E7D9690806FB
:100560007FF577AF94F87D1121293FF472AFA16A2E
:10057000606A814248D0A069405C0131C0B2986293
:100580002569B1FBF5F005FB1011A16261E720467A
:10059000BDE8F840E4E5CF0709D5F70507D5012701
:1005A0001F62D4F8807147F00107C4F88071EDB282
:1005B00015EA51073FF47FAF4FF0020E3D46C1F3FD
:1005C0008007C3F820E0D4F880E14EF0040EC4F8B0
:1005D00080E172E71968202021F04001196084F859
:1005E0007D0150E79A6812F040028CD1C4F8802156
:1005F000A5E7002D3FF477AF6DE7D4F87801036DE0
:100600009847D4F8F4203EE7A4F86621196821F051
:10061000800119601DE794F87D1121297FF433AF23
:10062000B4F8661189B2C9B1D4F81C11B1F5805F74
:100630001DD0D4F86011481CC4F860010978996293
:10064000B4F86631013B9BB2A4F866311BE73D4626
:100650003CE717F0E1FED4F8F42014E7196821F024
:1006600080011960196841F0400119600BE7D4F866
:1006700024110029DDD1D4F8601131F8020BC0F348
:1006800008009862C4F86011DAE700BF258102080B
:100690002DE9F0470569C3681D4028D00F4606467E
:1006A0004FF000484FF00009B5FA85F328FA03F23D
:1006B0001B3BD24332611540042B16D8DFE803F010
:1006C0003129211903007B6A002B32D003F1FF3A54
:1006D000C7F824901FFA8AFA3C6A34B1236820468E
:1006E000514698476468002CF8D1002DDCD1BDE854
:1006F000F0873868716B036889B29847002DD3D1B1
:10070000F5E77868B16B036889B29847002DCBD1C3
:10071000EDE7B868F16B036889B29847002DC3D143
:10072000E5E7F868316C036889B29847002DBBD1C2
:10073000DDE7F36A1FFA83FACEE700BF00B583B0A6
:10074000002002AB03F8012D0A46682127F02CFF98
:1007500003B05DF804FB00BF0846194628F04AB90B
:10076000074A084B10781B78834205D9C3F18003F0
:100770001844C0F17F007047C01AC0F17F00704775
:1007800084B2012000B20120014B58692CE600BF61
:1007900064870120014B986826E600BF648701202A
:1007A000014B186820E600BF64870120F8B510F5FA
:1007B0008A75044614D0D0F814212421002380F82F
:1007C0007D11116821F00101116013605360936085
:1007D000C0F8803180F87C3180F87D3180F87E313E
:1007E000A279A36812F00401C4F8183100F0F8806F
:1007F0004FF48053C4F81C3112F0020300F0298139
:100800004FF400534FF48061C4F820316379002025
:10081000C4F8241113F00101C4F82C01C4F8340108
:10082000C4F8280102D00420C4F8280113F00206FD
:1008300005D0D4F8280140F00800C4F82801D007FA
:100840000DD549B1D4F838014FF4803740F002009B
:10085000C4F84071C4F83801002E40F0E880120757
:100860002AD5002D58D094F87D3103F0FF02002BDB
:1008700000F0E880D4F814212423284684F87D3140
:10088000136823F00103136018F000FC012840D026
:10089000D4F83831002B40F0D880D4F814312846F1
:1008A0005A6822F490425A609A6822F022029A60B2
:1008B0009A6842F0080225E075B394F87D3103F0A0
:1008C000FF020BB984F87C21D4F814212423284694
:1008D00084F87D31136823F00103136018F0D6FB10
:1008E000012816D0D4F8383113B1284623F060FF20
:1008F000D4F8143128465A6822F490425A609A6813
:1009000022F02A029A601A6842F001021A6023F06B
:1009100019FF637903F0010100292ED0D4F8F020EB
:10092000002A75D00023D4F8F8004FF4806E4FF4FD
:10093000803104F130074FF48076A363E36363648E
:10094000A3646365A3652366E36522636063384639
:10095000C4F840E02165E66418F0AEF9384618F0B6
:10096000E9F994F87E31C4F87871202BA5667AD025
:10097000226B63795268C4F808219B072FD5D4F8FD
:10098000F420002A3DD0002340204FF48031C4F8E9
:10099000902004F19006D4F8FC204FF48067C4F84E
:1009A0009800C4F894203046C4F89C30C4F8A430B1
:1009B000C4F8A830C4F8AC30C4F8B430C4F8B830C7
:1009C000C4F8C030C4F8BC30C4F8A070C4F8B0108B
:1009D00018F072F9304618F0ADF950B1FEE7F8BDE5
:1009E00012F00203C4F81C1138D1C4F820311946A2
:1009F0000CE7D4F89030C4F87461C4F8C85058605B
:100A0000F8BDD4F88421136843F080031360F8BD67
:100A1000D4F88421116841F480711160916841F02B
:100A200001019160116841F020011160A5E7D4F83F
:100A300038014FF4003640F00100C4F83C61C4F8BE
:100A400038010CE784F87C2114E7284623F0B0FE37
:100A500023E7C4F820314FF48061D7E64FF4005308
:100A6000C4F82031D2E6E368626999B2002A3FF403
:100A70007FAFB1FA81F67609002E7FF479AF94F852
:100A80007C0101283FF474AF0B46A4F86C11384682
:100A90001449154F4FF0010C4FF0220E2167E76605
:100AA000D4F81411114FC4F880612431C4F86821BE
:100AB000C4F8806084F87CC184F87EE1E76718F0B0
:100AC000B7F8D4F8143184F87C611A6842F4807263
:100AD0001A609A6842F001029A609A6842F04002F5
:100AE0009A6045E7A1810208A581020835810208C4
:100AF00041715BE6816059E6B0B5C14BBEB0C149FA
:100B00001A6C00AFC04842F08052C04C1A641A6C94
:100B100002F08052C7F8F020D7F8F0201A6B42F4A8
:100B200080221A631A6B02F48022C7F8EC20D7F8EF
:100B3000EC200A6842F480720A600268A24200F067
:100B40009382B34C4FF6FF05B24AE168B2482940A0
:100B50000A43E2605A6F02601A6B42F480221A6301
:100B60001A6B02F48022C7F8F420D7F8F4201A6B2D
:100B700042F480121A631A6B02F48012C7F8E8205C
:100B8000D7F8E8201A6B42F480021A631A6B02F459
:100B90008002C7F8E420D7F8E4201A6B42F0005234
:100BA0001A631A6B02F00052C7F8E020D7F8E02071
:100BB0001A6B42F080421A631A6B02F08042C7F847
:100BC000DC20D7F8DC201A6B42F001021A631A6BA2
:100BD00002F00102C7F8D820D7F8D8201A6B42F0EB
:100BE00002021A631A6B02F00202C7F8D420D7F887
:100BF000D4201A6B42F004021A631A6B02F004024A
:100C0000C7F8D020D7F8D0201A6B42F008021A6338
:100C10001A6B02F00802C7F8CC20D7F8CC201A6B68
:100C200042F010021A631A6B02F01002C7F8C820D3
:100C3000D7F8C8201A6B42F020021A631A6B02F030
:100C40002002C7F8C420D7F8C4201A6B42F0400233
:100C50001A631A6B02F04002C7F8C020D7F8C02010
:100C60001A6B42F080021A631A6B02F08002C7F816
:100C7000BC20D7F8BC201A6B42F480721A631A6B3E
:100C800002F48072C7F8B820D7F8B8201A6B42F483
:100C900000021A631A6B02F40002C7F8B420D7F8F6
:100CA000B4201A6B42F400721A631A6B02F40072D9
:100CB000C7F8B020D7F8B0201A6B42F480621A63EC
:100CC0001A6B02F48062C7F8AC20D7F8AC201A6C1B
:100CD00042F001021A641A6C02F00102C7F8A8205F
:100CE000D7F8A8201A6C42F002021A641A6C02F0BB
:100CF0000202C7F8A420D7F8A4201A6C42F004021C
:100D00001A641A6C02F00402C7F8A020D7F8A020D9
:100D10001A6C42F008021A641A6C02F00802C7F852
:100D20009C20D7F89C201A6C42F010021A641A6CAE
:100D300002F01002C7F89820D7F898201A6C42F0F9
:100D400020021A641A6C02F02002C7F89420D7F827
:100D500094201A6C42F040021A641A6C02F04002AD
:100D6000C7F89020D7F890201A6C42F080021A64DD
:100D70001A6C02F08002C7F88C20D7F88C201A6C0D
:100D800042F480721A641A6C02F48072C7F88820E8
:100D9000D7F888201A6C42F400721A641A6C02F4B4
:100DA0000072C7F88420D7F884201A6C42F480427D
:100DB0001A641A6C02F48042C7F88020D7F88020A9
:100DC0001A6C42F400421A641A6C02F40042FA6788
:100DD000FA6F1A6C42F400321A641A6C02F4003290
:100DE000BA67BA6F1A6C42F480221A641A6C02F461
:100DF00080227A677A6F1A6C42F400220EE000BFFC
:100E0000003802400070004004400240EFBEADDEFA
:100E100000ED00E00005FA05FC5101201A641A6C8F
:100E200002F400223A673A6F1A6C42F480121A6494
:100E30001A6C02F48012FA66FA6E1A6C42F400120E
:100E40001A641A6C02F40012BA66BA6E1A6C42F492
:100E500080021A641A6C02F480027A667A6E1A6C46
:100E600042F400021A641A6C02F400023A663A6E06
:100E70001A6C42F000721A641A6C02F00072FA6581
:100E8000FA6D1A6C42F000521A641A6C02F00052A9
:100E9000BA65BA6D1A6C42F080421A641A6C02F09C
:100EA00080427A657A6D1A6C42F000421A641A6CBC
:100EB00002F000423A653A6D1A6C42F080721A6490
:100EC0001A6C02F08072FA64FA6C1A6C42F080625A
:100ED0001A641A6C02F08062BA64BA6C1A6C42F03E
:100EE00000621A641A6C02F000627A647A6C5A6CBE
:100EF00042F001025A645A6C02F001023A643A6C00
:100F00005A6C42F002025A645A6C02F00202FA630E
:100F1000FA6B5A6C42F010025A645A6C02F01002DA
:100F2000BA63BA6B5A6C42F020025A645A6C02F0EF
:100F300020027A637A6B5A6C42F480725A645A6C5B
:100F400002F480723A633A6B5A6C42F400725A644B
:100F50005A6C02F40072FA62FA6A5A6C42F48062C5
:100F60005A645A6C02F48062BA62BA6A5A6C42F4E9
:100F700000625A645A6C02F400627A627A6A5A6CAD
:100F800042F480525A645A6C02F480523A623A6ACD
:100F90005A6C42F400525A645A6C02F40052FA61DC
:100FA000FA695A6C42F480325A645A6C02F4803204
:100FB000BA61BA695A6C42F400325A645A6C02F44B
:100FC00000327A617A695A6C42F480225A645A6C0F
:100FD00002F480223A613A695A6C42F480125A64EF
:100FE0005A6C02F48012FA60FA685A6C42F4800279
:100FF0005A645A6C02F48002BA60BA685A6C42F4BD
:1010000000025A645A6C02F400027A607A685A6CE0
:1010100042F400125A645B6C03F400133B603B68BB
:1010200017F0F8FF1D4B02461D491B681D48A1FB28
:1010300003131D49A0FB02029B09920C013B0A60AD
:10104000B3F1807F08D2194AF025002007215360B0
:1010500084F8235090601160144AF837136843F005
:1010600004031360BD46B0BD114A01F5484102605A
:101070005A6C104842F480425A645B6C03F480431B
:10108000C7F8F430D7F8F4300A6803680A6083F3CD
:101090000888094B1B689847FEE700BF78060120C7
:1010A000D34D621083DE1B431094012010E000E05A
:1010B000EDFEFECA0000F01F0400F01F08B5054B4E
:1010C0001B6803B19847044B044A1A6072B6FFF7D5
:1010D00011F800BFF030012004400240EFBEADDE49
:1010E00008B5034B1B6803B1984772B6FFF702F8C7
:1010F000F030012030B439240C4D0022A0422B46A0
:1011000006D001321833052A0CD01C79A042F8D140
:101110009C79214201D10029F3D102EB420205EB77
:10112000C20000E0002030BC704700BF4C990408AA
:1011300030B5A02285B000211A4835F0DDFC1A4AEE
:1011400001231A4C116C04F1780519431164116CD8
:10115000194001910199116C41F002011164116C67
:1011600001F0020102910299516C41F002015164B7
:10117000526C02F002020392039A2BB91834AC426B
:101180000DD0A379002BF9D0207918340EF0C1FFCF
:1011900014F8102C02210FF085F8AC42F1D105B003
:1011A00030BD00BFCC960120003802404C990408A5
:1011B00001490248FFF76CBA1C9701200004014066
:1011C000FFF7F6BF01490248FFF762BAF496012023
:1011D0000004004002494FF08040FFF759BA00BFB9
:1011E000CC96012003680D4A9B0A934213D04032EB
:1011F00093420ED0B3F5801F00D070470021427992
:10120000022389010648DA4041589340DB430B61D1
:1012100070470221F3E70121F1E700BF0100100050
:101220005CAC01200368154A9B0A934223D04032EC
:10123000934211D0B3F5801F00D07047002371B9DD
:101240009B01417902220E48D140C0588A40C368B0
:1012500023EA0203C360704702230029F0D0022270
:101260009B0141790648D140C05802FA01F3C26897
:101270001343C36070470123E1E700BF0100100082
:101280005CAC012003682DE9F0439B0A464CA34265
:101290007ED04034A34258D0B3F5801F01D0BDE8C2
:1012A000F08300244079414F8608002953D04FEA4B
:1012B000841E02254FEA840C57F80E8005FA06F0CA
:1012C0000CEB040ED8F80C9006EB4E05DFF8E0E0CE
:1012D00040EA09002E1D4EF825104EF82620C8F8C9
:1012E0000C00314A934257D04032934252D0B3F56A
:1012F000801FD4D100260CEB0403DB0003F1200097
:101300007044EFF31185502282F3128810330022CB
:1013100073441968013211B1016018680430042A5D
:1013200003F10403F5D10023EDB2036085F31188C6
:101330006444B6010EEBC404BA59236A73B3D3688C
:1013400043F00103D360BDE8F08340790224174FD6
:1013500086080029ABD1A5014FF0020E4FEA840C9C
:1013600057F8058020FA0EF00CEB04050EFA00FE8B
:10137000D8F80C0006EB450520EA0E00DFF830E057
:101380002E1DC8F80C004EF825104EF82620A8E7B0
:10139000012487E70226AEE70126ACE7D36823F0F5
:1013A0000103D360BDE8F083010010005CAC0120B4
:1013B000CC960120F0B5830A4F4C85B0A34200F0D3
:1013C00095804034A34200F08F80B3F5801F01D098
:1013D00005B0F0BD0025AD01484E74597319A04207
:1013E000F6D00446464801394FF0000E076818460B
:1013F00089B2C3F810E0C3F808E0D960C3F814E07C
:101400007451B7FBF2F2013A5A6018F053F93D49B2
:10141000B4F1804F18BF8C420CBF0121002111D0C4
:10142000394B9C420ED003F580639C420AD0374A68
:1014300003F57C439C4218BF944203D003F57053DC
:101440009C42C5D1721900234FF4805792F83C009A
:1014500001930128029303930097B9D07059022792
:10146000DFF8B0E04FF0010C82F83D70876807EAC2
:101470000E0E274FC0F808E0D0F808E00EEA070784
:10148000876082F83C3082F83DC0B9B91E4B9C425F
:1014900014D003F580639C4210D003F580639C4216
:1014A00003D003F578439C4292D17219002392F83D
:1014B0003C200093012A0193029389D0735911486B
:1014C0005A688342996813D000F5806083420FD038
:1014D00022F0700221F08001354400205A609960AA
:1014E00085F83C0005B0F0BD022574E7012572E7E0
:1014F00022F47002ECE700BF010010005CAC012098
:10150000780601200000014000040040000C00406B
:10151000F8FFFEFF8800FEFFF8B506682C4CB30A02
:10152000A3422FD04034A3422AD0B3F5801F00D06D
:10153000F8BD002504463046FFF73CFF254AAB01C5
:10154000022021680127D518D658234A002385F8A0
:101550003D00346821483C43346085F83D7001E02B
:1015600050F8332091420FD001330E2BF8D10020D8
:10157000012126F0C1FF0020BDE8F84017F0B4B803
:101580000225D7E70125D5E7144A012102EBC30361
:101590005C7965B2284626F0AFFF284617F0A4F81C
:1015A0001B2C0AD02E2C11D101212C2026F0A4FFB7
:1015B0000B4B4FF480525A60F8BD0121192026F0E0
:1015C0009BFF074B4FF000721A60F8BDF8BD00BFDB
:1015D000010010005CAC012000000140F8990408F3
:1015E00000E100E0800A084B98420BD0403398425B
:1015F00006D0B0F5801F01D0002070470348704727
:101600000348704703487047010010005CAC01209C
:10161000DCAC01209CAC01202DE9F8434FEA4018D6
:10162000994FA8EB000507EBC5056B68002B66D04A
:10163000DB68002B63D02A7BC0EB40160446934B3B
:1016400042EA410100201B68F6008AB2287328464E
:10165000111181EA1221514001F00F0141EA0211FA
:1016600089B298476A6895F89530D179490748D486
:10167000022B44D095F8953092F80590012B5AD062
:101680001036A8EB0404B919B9F10C0F00F2EF8081
:10169000DFE819F05500ED00ED00ED006800ED0009
:1016A000ED00ED007C00ED00ED00ED000D0007EB1E
:1016B000C407774E774D0346D7F88840BA6D204669
:1016C000E6634032E56417F0B3FABB6DDA6842F4C2
:1016D0008052DA600122196A6F4802FA09F98342DE
:1016E00021EA090119621A6A49EA02021A627ED0E5
:1016F0006A4A93427BD01A6842F001021A60BDE840
:10170000F883022BFBD095F8953092F80590012BC9
:1017100000F0B5801036A8EB0404B919B9F10C0F2C
:1017200000F2A980DFE809F090A7A7A77CA7A7A7E8
:1017300068A7A7A74600022385F89530A0E707EB26
:10174000C407534E534D0346FC6FBA6D2046E66303
:101750003432E56417F06CFABB6DDA6842F400725B
:10176000DA60B7E707EBC407494E4A4D0346D7F89E
:101770008040BA6D2046E6633832E56417F058FAC7
:10178000BB6DDA6842F48062DA60A3E707EBC40756
:101790003F4E404D0346D7F88440BA6D2046E6637D
:1017A0003C32E56417F044FABB6DDA6842F400623B
:1017B000DA608FE707EBC407354E364D0346D7F89E
:1017C0008840BA6D2046E6634032E56417F030FA8F
:1017D000BB6DDA6842F48052DA600422196A02FAB8
:1017E00009F221EA02011962196A0A431A625A6C63
:1017F00042F400425A647EE707EBC407244E254DAD
:101800000346D7F88440BA6D2046E6633C32E5646F
:1018100017F00EFABB6DDA6842F40062DA60DCE7BA
:1018200007EBC4071A4E1B4D0346D7F88040BA6D2C
:101830002046E6633832E56417F0FAF9BB6DDA68E2
:1018400042F48062DA60C8E707EBC407104E114D1E
:101850000346FC6FBA6D2046E6633432E56417F048
:10186000E7F9BB6DDA6842F40072DA60B5E707EBBE
:10187000C407BB6D2EE707EBC407BB6DADE70223C2
:1018800085F8953046E700BF609901205499012002
:101890009D830208AD83020800000140000401405E
:1018A000114B98421ED003F5806398421AD003680A
:1018B00023F04003036059B141F48071002991FA8B
:1018C000A1F3B3FA83F108BF4FF0FF310139C9002A
:1018D000036823F0380319430160036843F04003B1
:1018E000036070474908E2E70038004038B5044615
:1018F00090F85D00002857D104F11405A0694FF459
:101900008071FFF7CDFF636E80226B2128469847D8
:1019100064200EF025FA636E03226821284698475A
:1019200064200EF01DFA636E01226B212846984751
:101930000F200EF015FA94F85720636E1B21032A2E
:1019400028468CBF1A22182298470F200EF008FA5A
:10195000636E18221C21284698470F200EF000FACB
:10196000636E94F856201A21284698470F200EF0EF
:10197000F7F9636E94F85820192128469847642097
:101980000EF0EEF9636E10223721284698470F209B
:101990000EF0E6F92846636E382101229847A069C7
:1019A0001021BDE838407BE70EF0B3FB18B12022D0
:1019B00000238271C371034B214641F8103F2AF086
:1019C0006DFF99E70100010830B44468012B24F44D
:1019D000805444601CDD40F2E93401E0013C35D024
:1019E0008568AD07FAD500293DD031F8024B8481D6
:1019F00040F2E93401E0013C28D08568ED07FAD5D2
:101A0000C468A4B20AB122F8024B023B012BE2DC0B
:101A1000446844F48054446013B340F2E93301E075
:101A2000013B37D08468A407FAD5002936D00B785B
:101A3000037340F2E93301E0013B2BD08168C90711
:101A4000FAD5C368DBB25AB1137009E0144B98425F
:101A50000CD0144B984219D003F57843984217D014
:101A6000012030BC70474FF6FF74C0E723460E4A92
:101A7000D82101FB03239A89013292B29A81988975
:101A800080B2003030BC18BF012070470223EEE75F
:101A90000323ECE7024A9042DBD1E8E7FF23C7E7E4
:101AA00000300140003C004074AD012030B5144CC2
:101AB00083B023781BB90120237003B030BD052209
:101AC00000238DF800208DF8013000BF0D4D2B68EC
:101AD000D8680EF0EEFB2B6801AA6946586802230D
:101AE000FFF772FF2B68D8680EF0E9FB00BF9DF886
:101AF000053003F0010383F00100237003B030BD13
:101B0000D4B001205CAD012070B5064C06462568B6
:101B100003E023685B1BB34203D8FFF7C7FF00282D
:101B2000F7D070BD0C94012070B5034682B0032439
:101B30000E468DF80730190C1B0A062015468DF845
:101B400005108DF806308DF80440FFF7DDFFC8B1B1
:101B500000BF0D4C2368D8680EF0ABFB226801A9CA
:101B6000042350680022FFF72FFF216832462B46DE
:101B700048680021FFF728FF2368D8680EF09FFB14
:101B800000BF284602B070BD5CAD012070B50446B0
:101B900082B0006A0EF08DFB6A4607231049A069E7
:101BA000FFF712FF206A0EF08AFB9DF801309DF8C6
:101BB000021001209DF8036041EA03219DF80420F2
:101BC0009DF805509DF8063042EA0622A4F8401020
:101BD00043EA0523A4F84220A4F8443002B070BDC3
:101BE000F86D040840F2E93300E09BB18268013BE4
:101BF00012F0020F9BB2F8D0017340F2E93300E01B
:101C000043B18268013B12F0010F9BB2F8D0C0686B
:101C1000C0B270470C4A904209D00C4B984211D088
:101C200003F57843984201D0FF2070470323084A08
:101C3000D82101FB03239A89013292B29A819889B3
:101C4000C0B270470223F2E700300140003C004080
:101C500074AD012038B5054600BF084C2368D8682C
:101C60000EF027FB236829465868FFF7BBFF23685F
:101C7000D8680EF024FB00BF38BD00BF5CAD01206A
:101C80002DE9F04FB2F1000A89B00290049103935C
:101C900040F3AD800B46002201EB8A0153F8040BA0
:101CA0008B420244FAD1039B0592002B00F09780EF
:101CB000059B002B6BD0059BDFF858910093504B90
:101CC0001B68DAB200995118B1F5807F8CBFC2F55C
:101CD0008072009A01924B4A92689A426BD9190C11
:101CE0004FF002041A0A06208DF81F308DF81E20CE
:101CF0008DF81D108DF81C40FFF706FF0620FFF73A
:101D0000A9FF0123404A137000BFD9F80030002416
:101D1000049DD868A3460EF0CCFAD9F8002007A994
:101D2000042350682246FFF74FFE029E019F296858
:101D30004FEA8408002201340B4671B1B942D9F848
:101D4000000028D231684068FFF73EFE2A683368F9
:101D5000BF1A13443360C5F800B0A24505F104056D
:101D600006F10406E3D1D9F80030D8680EF0A7FADE
:101D700000BF234B9DE806001B68891A1344204AC4
:101D800000911360039A1AB3009A002A99D105981A
:101D900009B0BDE8F08F029C3B46406854F808103B
:101DA000FFF712FE54F808202B683A44DF1B44F872
:101DB00008202F60D7E705980023009C1349001BDB
:101DC000134A0B7005900598137009B0BDE8F08FA9
:101DD000059B5B1A0593059809B0BDE8F08FFFF7E6
:101DE00065FE00287FF464AF039B0593CFE7039B58
:101DF0001BB90593FFF75AFEC9E700230593C6E711
:101E0000FCB1012040080120D4B0012084B201209F
:101E100000B201205CAD012008B545F20820FFF7B3
:101E200073FE0620FFF716FF064B0122C7201A702B
:101E3000FFF710FF002304480449054A03700B70A4
:101E4000136008BDD4B0012084B2012000B201208B
:101E5000FCB10120F8B504460F4615461E46C06881
:101E60000EF027FA47F080016068FFF7BBFE3346AB
:101E70002A4600216068FFF7A7FDE0680EF01FFA10
:101E80000120F8BD70B504460E461546C0680EF038
:101E900010FA31466068FFF7A5FE29466068FFF733
:101EA000A1FEE0680EF00BFA012070BDF8B5D82352
:101EB000674D684A044603FB00F3E9582B449142FE
:101EC00000F0A380D823661C03FB0453F6B21879F4
:101ED0000EF01FF9074610B11223C6718371D82383
:101EE00003FB045358790EF014F910B11323C67193
:101EF0008371D82303FB045398790EF00AF910B1CB
:101F00001423C6718371D82303FB04539A7B002AE0
:101F10005FD0DA7938464E210EF0C4F9D82606FB98
:101F200004F6AF1978790EF0F4F83A7A2E210EF013
:101F3000B9F9B8790EF0EDF87A7A0E210EF0B2F90F
:101F4000AB5945491A688B4222F040021A605FD0B3
:101F5000424A934266D0424A93426ED03D4A9342EF
:101F60003DD0404A934245D03F4A934209D102F5C1
:101F70006442516A41F400115162516A21F4001126
:101F80005162D822596802FB045441F48051A27B6B
:101F90005960002A196814BF0024022449060FD48E
:101FA0001D6882F00102314831492840024342F461
:101FB000457222431A605A68114041F4E061596049
:101FC000DA6922F40062DA611A6842F040021A60AB
:101FD000F8BDDA7938462E210EF064F99EE702F555
:101FE0008232516A41F400515162516A21F4005128
:101FF0005162C6E702F56842516A41F480115162AC
:10200000516A21F480115162BBE701229A7359E7AA
:10201000184A516A41F480515162516A21F4805149
:102020005162A1E702F50032116A41F48041116268
:10203000116A21F48041116296E702F5FE32116ABD
:1020400041F400411162116A21F40041116298E7E4
:1020500074AD0120003401400030014000380040E0
:10206000003C004000500140005401404000FFFF90
:10207000FBF0FFFF0038024070B5C0EBC0000D4C14
:102080000D4E82B004EB8004306B25692843306329
:10209000366B94F90D003540A1606361910901959B
:1020A000019B26F029FA94F90D0016F01DFB02B0F1
:1020B00070BD00BF80060120003802400A4BC0EB13
:1020C000C00030B403EB8000084C82B0256B03697C
:1020D0001D432563246B0176234042760193019BC7
:1020E00002B030BC704700BF8006012000380240BB
:1020F0000348D0F8AC3113B100F5D27018477047DF
:10210000800601200348D0F8903113B100F5C47067
:1021100018477047800601200348D0F8743113B186
:1021200000F5B67018477047800601200348D0F8C4
:10213000583113B100F5A870184770478006012088
:102140000348D0F83C3113B100F59A701847704736
:10215000800601200348D0F8203113B100F58C70BF
:1021600018477047800601200348D0F804310BB1AE
:10217000FC301847704700BF800601200348D0F8A4
:10218000E8300BB1E0301847704700BF80060120EF
:102190000348D0F8CC300BB1C4301847704700BFAB
:1021A000800601200348D0F8B0300BB1A8301847A2
:1021B000704700BF800601200348D0F894300BB16F
:1021C0008C301847704700BF800601200248836F9B
:1021D0000BB1703018477047800601200248C36D6C
:1021E0000BB1543018477047800601200248036C39
:1021F0000BB1383018477047800601200248436A07
:102200000BB11C30184770478006012002488368D4
:1022100003B11847704700BF80060120014816F03F
:10222000EBBE00BF58930120014816F0A7BE00BFC7
:1022300058930120014816F0DFBE00BFF89201203C
:10224000014816F09BBE00BFF8920120014816F02D
:10225000D3BE00BF98920120014816F08FBE00BF88
:1022600098920120A54A0021A54BA64870B5D2F846
:1022700088404FF00065A44EA4B044F47004C2F846
:1022800088401C6844F001041C6099601C68204070
:1022900018605E60186820F480201860D96095602E
:1022A000BFF34F8FBFF36F8FC2F85012516941F4E3
:1022B00000315161BFF34F8FBFF36F8F196C934A99
:1022C00041F080511964196C01F08051019101991C
:1022D000116841F440411160126802F440420092DA
:1022E000009A9A6802F00C02042A52D09A6802F00E
:1022F0000C02082A4AD0824B854C1A68194642F4CF
:1023000080321A60226803E023689B1A642B3CD851
:102310000B689803F8D57A4B9A6802F00C02082AE9
:1023200033D01A68184622F080721A60226803E0DF
:1023300023689B1A022B28D803689B01F8D447F620
:10234000C07393FAA3F34FF44031B3FA83F291FAD6
:10235000A1F14FF0706191FAA1F10926B1FA81F172
:102360004FF4D8736B4D8E406549934033431D4302
:102370004560036843F08073036022680B689E0128
:102380000BD423689B1A022BF8D9FEE75B685C022A
:10239000B1D55B4B5E4C1B68BDE7086C5B4A40F0F7
:1023A000805013460864096C01F080510291029933
:1023B000116841F48031116021685A68D50305D451
:1023C0002268521AB2F57A7FF7D9FEE71A684F49A8
:1023D00042F400321A60226804E023689B1AB3F5C5
:1023E0007A7FF2D84B689803F7D54FF400164FF078
:1023F00000654FF4C0710722032303A803962295BA
:10240000089109920B9331F04BFD00B1FEE7424A6F
:10241000136803F00F03062B1BD9394B9A6822F07F
:10242000F0029A601A68920166D59A68184641F2DD
:10243000883122F0030242F002029A602268836827
:1024400003F00C03082B10D023689B1A8B42F6D99B
:102450000AE0136823F00F0343F0070313601368C7
:1024600003F00F03072BD8D0FEE72B4A136803F0C5
:102470000F03072B34D8224CA36823F4E05343F412
:10248000A053A360A36823F4604343F40043A36014
:1024900016F0C0FDA368F02292FAA2F2B2FA82F21C
:1024A00003F0F0031D4ED3401D4D33441B7A20FA38
:1024B00003F32B6026F054F800231A4A03A8039272
:1024C0001493159316931793189319931A931B93B8
:1024D0001C931D931E931F9331F0E2FC20B3FEE783
:1024E000136823F00F0343F007031360136803F02E
:1024F0000F03072BB8D1BEE7B6E700BF00ED00E041
:1025000000380240FFFFF6FE10300024007000404B
:102510008092012008004020003C0240F86D040831
:1025200078060120C0FF0300D4F88C3023F08073BC
:10253000C4F88C30D4F88C3043F08073C4F88C30FD
:10254000A36803F00C03042B26D0082B0CD0144BEB
:10255000144A15499268C2F303121644327AD340E2
:102560008B422B601AD0FEE7616862684B0261689B
:1025700002F03F024CBF0D4B094BB3FBF2F3C1F32A
:10258000881203FB02F3074A5268C2F30142013288
:102590005200B3FBF2F3DBE7044BD9E724B070BD84
:1025A0000024F4000038024000E6DF0C00127A003C
:1025B0002DE9F04F2DED028B93B083461BF044FACA
:1025C0008C4B1D7825B113B0BDEC028BBDE8F08FAC
:1025D000894B1B685C05F6D5884BDFF87C821B684D
:1025E0006BB1874AD8F800101368CB1A7C2B06D938
:1025F0008448116003780133037019F0E7FC824BC3
:102600001B78002B6DD0814C814AD4F81031ABEB94
:102610000303934201F2E68294F81891B9F1000F96
:1026200032D17C4F38680DF092FCC0B201280FD92E
:10263000022841F0AC87784E3378002B42F0E580D9
:10264000D4F81C31ABEB0303B3F57A6F82F0A982A7
:10265000D4F82031002B44D094F81831BBB96F4B1B
:10266000012100221B6884F818119B7884F82C2122
:102670001E3B8B4242F24F8238680221043019F02F
:1026800059FC94F8243110E0D4F820314BB3D4F83D
:10269000283140F6B732ABEB0303934221D994F8CB
:1026A0002431002B01F074865A4F013BDBB284F8D1
:1026B0002431002B01F0BC83D4F8206194F82C2144
:1026C00016F8011B94F82D310A4438680133C4F818
:1026D000206184F82C2184F82D310DF03BFCC4F8E6
:1026E00028B14F4BD8F800601B7843B14D4F386884
:1026F00028B14D4B1B78013B012B41F2A8834B4B7A
:102700001B7863B14A4F3B684BB1404CD8F80090FE
:10271000D4F84431A9EB0303632B00F2E780454F63
:102720003B78022B01F014863B4E96F87430032B55
:1027300001F06983404B1B7873B1404D2B685BB14E
:10274000324C0DF065FA44F61F620290D4F8503115
:10275000C31A934200F2A681394B1B78002B7DD11E
:10276000384B1B783BB1294C374BD4F8A02213448B
:102770009B4581F0E281354B1B78002B3FF423AF62
:10278000224E334C06F2C127324D20680DF0DFFB9C
:1027900000283FF418AF20680DF0D3FB2B7880465B
:1027A0005A1E33B120682A700DF0D1FB0028F2D1F7
:1027B00009E703223946781E34F084F996F8C012EE
:1027C0004FF6FF7396F8C12286F8C3821FFA88F885
:1027D0004B409B1A9BB2B8EB132FD6D1DBB296F8C5
:1027E000C2229A42D1D1781E19F0B2F82B7818443F
:1027F0002870CAE74F88012078A9012008380120F5
:10280000783A0120743A01209A3E0120A01E01204E
:102810003F0D0300203A012000000120243A01204E
:102820009C3E012010380120A43E0120AC3E012036
:10283000183A0120A2B30120B43E0120B83E012085
:10284000243F0120353F0120A0860100BE3E01202B
:10285000C43E0120C83E01200C9401207D4C22780A
:10286000A2B17D4B9B7A53B10DF0D2F97B4B1B6823
:10287000C31AA3F57A73B3F5FA6F07D82278784BA9
:10288000784918680DF034FB00232370764C774BA1
:10289000D4F8982213449B45FFF462AF744DC4F8FA
:1028A00098B22B78002B41F0AD86724D2B78002B1F
:1028B00041F00686704994F89C228D5CE80701F18E
:1028C000E987A90701F1A7876A0701F16B872A0742
:1028D00001F11C8794F89C32684A0133117893FB0C
:1028E000F1F201FB123384F89C3239E7644E412047
:1028F00019F0CAFA634AB6F90230029282FB031059
:10290000DB17DFF89CA1C3EBA00080B219F0A0FA9E
:10291000B6F90030029A82FB0310DB17C3EBA0006C
:1029200080B219F095FAB6F90430029A82FB0320BE
:10293000DB17C3EBA00080B219F08AFA9AF80010F6
:1029400038680DF007FB94F8482112F0010601F0F9
:1029500042854D4B1B689B066CD54C4B1B789807EA
:1029600042F1E1804A4E337D042B8CBF03230223C6
:102970000293472019F088FA306819F031FA70682C
:1029800019F02EFAF389434A3868A2FB0323C3F3F4
:102990004713194603930DF0DDFA9AF80010039BD4
:1029A000642032894B4000FB02F08AF8003019F0B5
:1029B00017FA029B367D386843EA8606F6B231463E
:1029C0000DF0C8FA9AF8003038685E4031468AF84F
:1029D00000600DF0BFFA94F848215ABB2E4E4F20EC
:1029E000029219F051FA306819F0FAF9706819F08A
:1029F000F7F9029A104619F0F3F9012138680DF041
:102A0000A9FA224A9AF80030167883F00103386850
:102A100006F001068AF8003031460DF09BFA9AF86C
:102A2000003038685E4031468AF800600DF092FA56
:102A300094F84821531C194AC4F84491DBB2A2FB14
:102A40000312D20802EB8202A3EB420384F848315E
:102A500065E600BF8C3E01200CAB0120E82F012071
:102A6000283F01204C3E0120A01E0120A08601002D
:102A70002C3F01202D3F0120303F0120343F012019
:102A80007C3A012067666666983A01209C3A0120EC
:102A9000A03A01201F85EB51403B0120CDCCCCCC8E
:102AA0001C3A012094F85631002B41F08F84D74A0C
:102AB0004AF60B4748F603404BF60F43126849F6B7
:102AC000074602F0080100294FF0190104BF3B46F8
:102AD000064612F0040F84F8561118BF1E469106E0
:102AE00003D546F4804646F02006C94AC6F30903DA
:102AF0005179002942F081809279002A42F08F8139
:102B0000914664204FF0FF3A00220C930121FE23EE
:102B10000AAF0A960B964FF01F0EADF83690ADF83F
:102B200038A08DF84600ADF83420CDF83A20CDF825
:102B30003E20CDF842206271E171A370B54E84F859
:102B400003E00FCF0FC697E80F0007C61A0C26F850
:102B5000023BC8233146701CA37101F81E2994F86A
:102B6000662182F0F103561C227183EA031384F874
:102B70006661DAB2130983F0E70343EA022383EACA
:102B8000C2031BB283EA0312C3F30723D2B283EA60
:102B9000121343EA022383EAC2031BB283F0C80282
:102BA000C3F3072382EA0212D2B283EA121343EA82
:102BB000022383EAC2031BB283F00106C3F3072298
:102BC00086EA0613DBB282EA131242EA032282EAA1
:102BD000C3021646228011F8013B7340814283EA0A
:102BE0000313DBB24FEA131282EA162242EA0322EF
:102BF00082EAC3031BB29EB22680ECD183F07C0331
:102C0000854F04F1220A83EA031307F5C77CDBB280
:102C10004FEA131E8EEA162E8EEA032E8EEAC30E9C
:102C20000FFA8EFE1FFA8EF35FFA8EFE4FEA13291B
:102C3000238084F827E084F828903868103757F804
:102C40000C1C664657F8082C0CF1100C57F8043C85
:102C500057450FC6F1D13868704ECCF800003B796B
:102C600006F127078CF8043084F8B5E184F8B691B2
:102C700016F8011F28680DF06DF9B742F8D194F8E5
:102C80005711002941F01784654B0A22D8F800003B
:102C90001B78039084F85721002B01F02785614AA7
:102CA000012BB2F800C042F2C680022B568801F018
:102CB000C0879088032B059002F0D480042BB2F8D3
:102CC00006E002F0CA80052BB2F8089002F0C1803D
:102CD000062BB2F80AA002F0B980072B908900D029
:102CE000D18994F8663100274F4A069383F0300368
:102CF0006CF30F07128883EA031366F31F47039EE2
:102D0000DBB2C2EB02220A960493049B474E0B9758
:102D10001F0986FB026C0023059E87F07A07CDF819
:102D20001CC066F30F03079EDDF818C06EF31F4347
:102D300016444FF0000ED2170393049BC2EB662299
:102D4000764669F30F0E47EA03278DF83D2060F3BE
:102D50000F066AF31F4E87EAC303624661F31F46FC
:102D6000CDF834E01BB24FF0C80E01324FF0230A09
:102D700083EA0311C3F30729039B0020C9B284F837
:102D800066210C930AAF89EA111384F804C04FF04E
:102D9000160C84F806E043EA01230E9684F803C07B
:102DA0004FF0FE0983EAC1038DF83C0060711BB24D
:102DB000184E84F807A083EA0E02C3F3072384F8B1
:102DC000029082EA0211C9B283EA111242EA012298
:102DD00082EAC10212B282EA0A03C2F3072E83EA30
:102DE000031C5FFA8CFC0FCF8EEA1C1E0FC64EEA46
:102DF0000C2397E8030083EACC0346F8040BB01CCD
:102E000026F814191946238012E000BF983A0120D1
:102E1000843A0120A81E0120A21E01202F2001209B
:102E2000C8880120507001205830012003082080FC
:102E300016F8012B4A40864282EA0212D2B24FEAC9
:102E4000121383EA112343EA022383EAC20212B275
:102E500091B22180ECD182F0F402DFF8EC9304F21D
:102E60008F1604F2AD1782EA0212D9F8000009F5B4
:102E7000C77CD2B24FEA121E8EEA112E8EEA022EC3
:102E80008EEAC20E0FFA8EFE1FFA8EF35FFA8EFEE6
:102E90004FEA132A238084F81EE084F81FA0D9F893
:102EA0000410D9F80820D9F80C30ACE80F00D9F894
:102EB0001000D9F81410D9F81820ACE8070084F8ED
:102EC000ADA184F8ACE116F8011F28680DF042F8B6
:102ED000B742F8D194F85A31002B41F0DC82D64B3E
:102EE00019221B6884F85A219A0640F1FB82D34BC1
:102EF0001B789B0741F17C86D14E337D042B8CBF20
:102F00004FF0030A4FF0020A0CF082FE338A328936
:102F10004FF47A7103EB83030A900AAF01FB02F2CC
:102F200030685B000E92BE46ADF842304FF00009AB
:102F30000C904FF0FF31F3894FF0C80C327D706870
:102F40008DF844A04FF0180A0D90ADF840308DF880
:102F50004520CDF82C900F910397BA4FBEE80F0093
:102F60000FC79EE80F0007C73A461E20B91CFE2770
:102F700022F81C3994F866E1E0708EF07803A770AF
:102F800084F804E00EF1010E83EA031384F807A02D
:102F900084F80590D8B284F866E184F806C0030985
:102FA00083F0F60343EA002383EAC0031BB283EAFB
:102FB0000310C3F30723C0B283EA101343EA0023CC
:102FC00083EAC0031BB283EA0C00C3F3072380EA41
:102FD0000017FFB283EA171040EA072080EAC70013
:102FE00000B280EA0A07C0F3072387EA0710C0B2DD
:102FF00083EA101343EA002383EAC0031F462380B9
:1030000012F8010B78408A4280EA0010C0B24FEA01
:10301000101383EA172343EA002383EAC00000B2B7
:1030200087B22780ECD180F01800874A04F122098A
:1030300080EA00100592964602F5C77CC0B24FEABE
:10304000101A8AEA172383EA002A8AEAC0000FFAD4
:1030500080FA1FFA8AF35FFA8AF2190A238004922F
:10306000069184F8262084F82710DEF800000EF17F
:10307000100E5EF80C1C67465EF8082C0CF1100C64
:103080005EF8043CCE450FC7EFD1DEF800006F4F6D
:10309000CCF800009DF8103007F12609BA4684F8F4
:1030A000B4319DF8183084F8B5311AF8011F28683A
:1030B0000CF050FFD145F8D10CF0AAFD644BDFF8BD
:1030C00098E14FF47A7CB3F90430002132898EFB09
:1030D000039E4FEAE37933680CFB02F276684FF007
:1030E0001C0C0B93C9EBAE030D92ADF842302123BB
:1030F0000E92FE22DDF80CE00C960A90ADF83C1022
:10310000ADF83E10ADF840106171E371A2704D4E04
:1031100084F803C0BEE80F000FC6C82206F10C03F6
:10312000A271A3F11C0C9EE8070086E8070094F842
:10313000661181F06A02481C217182EA021284F849
:103140006601D1B20A0982F0D50242EA012282EA7E
:10315000C10212B282EA0211C2F30722C9B282EAA4
:10316000111242EA012282EAC10212B282F0C801BF
:10317000C2F3072281EA0111C9B282EA111242EABE
:10318000012282EAC10212B282F02100C2F30721B9
:1031900080EA0012D2B281EA121141EA022181EAE8
:1031A000C201084621801CF8012B42409C4582EA5E
:1031B0000212D2B24FEA121181EA102141EA022131
:1031C00081EAC20212B290B22080ECD182F0680291
:1031D0001D4E04F1220982EA021206F5C77CD2B222
:1031E0004FEA121A8AEA102181EA022A8AEAC20206
:1031F0000FFA82FA1FFA8AF35FFA8AFA1A0A238010
:1032000084F824A0049284F825203068103656F8FB
:103210000C1CE64656F8082C0CF1100C56F8043C31
:103220004E45AEE80F00F0D13388B946094EACF8F0
:1032300000309DF8103011E0983A01209C3A0120AE
:10324000A03A0120A81E0120A21E01202F2001204B
:103250007C3A0120532001206766666684F8B2A19B
:1032600084F8B33119F8011F28680CF073FE4E453D
:10327000F8D194F866110023DFF814E6312681F0C6
:10328000EB020C936371FE20DEF8043082EA021236
:1032900021710131D2B20B93DEF800304FF00C0EE9
:1032A00084F86611C8210A931309E67183F0C503F7
:1032B000DFF8E095A07043EA0223A17184F803E0EF
:1032C00083EAC2031BB283EA0312C3F30723D2B219
:1032D00083EA121343EA022383EAC2031BB283EA9E
:1032E0000102C3F3072382EA0212D2B283EA121365
:1032F00043EA022383EAC203039A1BB25E40C3F38C
:10330000072386EA0616F6B283EA161343EA062373
:1033100007CA83EAC603A9F5C4761BB286E807008C
:10332000267A607A5E40C3F30723A17A86EA0616FE
:10333000E27A94F80CE0F6B294F80DC094F80EA07E
:1033400083EA161343EA062383EAC603E67B1BB22D
:103350005840C3F3072380EA0010C0B283EA101379
:1033600043EA002383EAC003207C1BB25940C3F325
:10337000072381EA0111C9B283EA111343EA012349
:1033800083EAC103617C1BB25A40C3F3072382EA7C
:103390000212D2B283EA121343EA022383EAC2037F
:1033A000A27C1BB28EEA030EC3F307238EEA0E1E25
:1033B0005FFA8EFE83EA1E1343EA0E2383EACE03EE
:1033C00094F813E01BB28CEA030CC3F307238CEAD6
:1033D0000C1C5FFA8CFC83EA1C1343EA0C2383EA7F
:1033E000CC031BB28AEA030AC3F307238AEA0A1A48
:1033F0005FFA8AFA83EA1A1343EA0A2383EACA03C2
:103400001BB25E40C3F3072386EA0616F6B283EAD0
:10341000161343EA062383EAC6031BB25840C3F3DC
:10342000072380EA0010C0B283EA101343EA0023A6
:1034300083EAC0031BB25940C3F3072381EA011199
:10344000C9B283EA111343EA012383EAC1031BB221
:103450005A40C3F3072382EA0212D2B283EA12135C
:1034600043EA022383EAC2031BB28EEA030EC3F3CC
:1034700007238EEA0E1E5FFA8EFE83EA1E1343EACE
:103480000E2383EACE031BB283F02706C3F3072380
:1034900086EA0612D2B283EA121646EA022686EAC3
:1034A000C20636B2B3B25FFA86FA23804FEA132E11
:1034B000059E84F814A084F815E030687168B2683D
:1034C000F368B6F810C0A9E80F0029F803CB84F818
:1034D000A3E184F8A2A117F8011F28680CF03AFDB7
:1034E000B945F8D194F85E21002A40F0DF87DF4E1D
:1034F000052094F866C10DF1280EB6F90270B6F9F0
:1035000000108CF06A0362711E2206EE901A794256
:1035100083EA0313E27107EE901AB6F90410FE2253
:10352000D8F8006007EE101AD9B2A2701C220B095D
:103530000A96E270C82283F0D503F8EEE66AA2711B
:10354000F8EEE77A43EA0123B8EEC77A9FEDC86A3E
:10355000002783EAC10384F85E0166EE866A0E974F
:103560001BB267EE867A27EE067A0F9783EA03117D
:10357000C3F3072310970CF10108C9B2CDED0B6A14
:10358000CDED0C7A83EA11138DED0D7AB94F43EA34
:10359000012383EAC1031BB25A40C3F3072382EA23
:1035A0000212D2B283EA121343EA022383EAC2036D
:1035B0001BB283F01E06C3F3072386EA06195FFADF
:1035C00089F983EA1916BEE80F0046EA09260FC7F3
:1035D00086EAC90607F10C039EE80700A7F1100E62
:1035E00087E8070084F804C0268084F866811EF806
:1035F000012B72409E4582EA0212D2B24FEA1211AA
:1036000081EA162141EA022181EAC20212B296B28F
:103610002680ECD182F02702974F04F1220982EA3A
:10362000021207F5C77CD2B24FEA121E8EEA162E9E
:103630008EEA022E8EEAC20E0FFA8EFE1FFA8EF36B
:103640005FFA8EFE4FEA1328238084F824E084F882
:1036500025803868103757F80C1C664657F8082C38
:103660000CF1100C57F8043C4F450FC6F1D1834EB6
:103670003B8806F12407ACF8003084F8B2E184F806
:10368000B38116F8011F28680CF064FCB742F8D12A
:1036900094F85F91B9F1000F40F00287784B052252
:1036A0001B6884F85F219F0641F12A80754BDFED8E
:1036B000766ADA891B8907EE902A07EE103AF8EE4F
:1036C000E77AB8EE477A67EEA67A94F866610AABB5
:1036D0006E4A4FF0640E86F022011F46B2F90620B2
:1036E00081EA01110393B2F5FA6F604BC9B2DFF8BA
:1036F000A8C1A8BF4FF4FA62B3F904000B09267100
:10370000B2F57A7F06F1010683F05903CDED0B7A0D
:10371000B8BF4FF47A7284F8666143EA01238DEDF5
:103720000C7AA2F57A7283EAC1030EFB02F2DFF88B
:103730006CE11BB28CFB026CD2178EFB001E0021C9
:10374000C2EBAC124B4E83EA031CC3F30723ADF864
:103750003A204A225FFA8CFC0A91E271FE2283EA47
:103760001C130D91A270142243EA0C23C821E270AD
:10377000002283EACC03A1716271C0171BB2C0EBB7
:10378000AE0083EA0102C3F30723ADF8380082EAF2
:103790000212D2B283EA121343EA022383EAC2037B
:1037A0001BB283F04A0EC3F307238EEA0E1C5FFAA6
:1037B0008CFC83EA1C1E0FCF4EEA0C2E3F688EEA6B
:1037C000CC0E0FC6A4F800E0321D46F8107916F8AA
:1037D000013B83EA0E03964283EA0313DBB24FEA0E
:1037E000131181EA1E2141EA032181EAC3031BB2BE
:1037F0001FFA83FEA4F800E0E9D183F014031E4A07
:1038000004F2AB1883EA03131146059204F28F12F7
:10381000DBB20868164601F5C77C1A0937460496DC
:1038200082EA1E2E0E468EEA032E8EEAC30E0FFA91
:103830008EFE1FFA8EF35FFA8EFE4FEA132A238064
:1038400084F81CE084F81DA0F3684968B268ACE80D
:103850000F0030697169338B3E46ACE80300ACF869
:10386000003084F8ABA184F8AAE119E07C3A012089
:1038700088C3E43AA81E0120A21E01202F200120A7
:10388000983A0120A03A01200AD7233C5070012029
:10389000403B012030200120D34D621067666666F0
:1038A00017F8011F28680CF055FBB845F8D1C44B38
:1038B000C44A1B781278013B049612F00101DBB276
:1038C00014BF4FF0C00E4FF0400E172B03D8BE4A66
:1038D000134493F83090BD4B1B889E0700F05F8720
:1038E0004EF0100E002213F4027F18BF022213F0D4
:1038F000100F18BF062213F0200F18BF1022002946
:1039000041F04781032794F8660103230A920021BE
:1039100080F046028DF8303000F10108207182EA13
:103920000212C8208DF82F700927D2B28DF82C9082
:10393000E7704FF0FE0C13098DF82EE08DF82D1076
:1039400083F09203E171617143EA0223A071DFF811
:1039500090E283EAC20384F8668184F802C01BB255
:1039600083EA0312C3F30723D2B283EA121343EAB2
:10397000022383EAC2031BB283EA0002C3F30723D4
:1039800082EA0212D2B283EA121343EA022383EAE2
:10399000C203039A1BB283EA0317C3F30723FFB2E0
:1039A00083EA171343EA072307CA83EAC703AEE88B
:1039B00003001BB2207A617A0EF5C07C5840C3F335
:1039C000072394F80A800EF5C87780EA00108EF875
:1039D0000020E27AC0B294F80CE094F80DA083EADB
:1039E0001013A67B94F8109043EA002383EAC003E7
:1039F000E07B1BB25940C3F3072381EA0111C9B22E
:103A000083EA111343EA012383EAC1031BB288EA64
:103A10000308C3F3072388EA08185FFA88F883EAE3
:103A2000181343EA082383EAC8031BB25A40C3F3BE
:103A3000072382EA0212D2B283EA121343EA022374
:103A400083EAC2031BB28EEA030EC3F307238EEA96
:103A50000E1E5FFA8EFE83EA1E1343EA0E2383EAEC
:103A6000CE031BB28AEA030AC3F307238AEA0A1ABF
:103A70005FFA8AFA83EA1A1343EA0A2383EACA033B
:103A80001BB286EA0302C3F3072382EA0212D2B210
:103A900083EA121343EA022383EAC2031BB25840AB
:103AA000C3F3072380EA0010C0B283EA101343EA8D
:103AB000002383EAC0031BB289EA0302C3F307238E
:103AC00082EA0212D2B283EA121343EA022383EAA1
:103AD000C2031BB283F03202C3F3072382EA02124D
:103AE000D2B283EA121343EA022383EAC2031BB26F
:103AF0009AB2DBB24FEA122E2280637484F812E08D
:103B0000059E30687168B268B6F80C80049EACE817
:103B100007008CF80290ACF8008084F8A0E184F8EB
:103B20009F3116F8011F28680CF014FAB742F8D13B
:103B3000029BC4F85031FEF70FBE94F8A432224A1B
:103B4000C4F8A0B202EB8302926C5AB312AD04F235
:103B5000AB2104F2BD234FF0000E45F8201DA52631
:103B600080211B4F0B9315232846A7F800E084F80B
:103B7000AA3284F8A86204F52A7684F8A91290473C
:103B8000284639880DF06AF80A9D31461148AD1B68
:103B9000152DA8BF15252A4632F089FF0E4A94F844
:103BA000A432157001330D4A82FB0312A2EBE372BB
:103BB00002EB42029B1A84F8A432FEF7DCBD00BF80
:103BC000903001200D720120106E0408603B01202E
:103BD000083E0120A82E0120BD2E01205655555526
:103BE000A81E0120C14A4FF47A71C14B0027D07A38
:103BF000D8F8006001FB00F1D4F814011B88301ADA
:103C0000BC4A5FFA83FE88424FEA132382F81EE023
:103C1000D37782F814E053759770177180F05A8447
:103C2000B5494FF0F40EB54801270B684FF0300945
:103C3000896880FB03C6DB1780FB01C0C917C3EB93
:103C4000A603AF4EC1EBA001AE4813771B1200785C
:103C50004FEA212A53774FF0750C82F82010800725
:103C6000317DA94B82F81AE04FF0780E82F821A03E
:103C70009976D77682F8229082F823C082F824E0E1
:103C800040F1258472680529D6F800C011469F4F7F
:103C90004FEAEC70DFF8889287FB0CE2DFF884A231
:103CA00087FB01E74FEAE17EC0EBA2500291CEEB29
:103CB000A75E09FB00C700EB800009FB0E110EEBAD
:103CC0008E0E07EB470701EB41014FEA47074FEA2A
:103CD000410100EB80000A468AFB07914FEAE77931
:103CE00004904FEAA1410392F0898AFB02A20EEBF5
:103CF0008E0EB6F808A0A1EB090600EBC000CDF8C7
:103D000014E04FEAA242DFF820E23146069076B294
:103D100003980EFB1171049F0AF5FA7A4FEAE079D5
:103D2000069806EB8706A2EB09074FEA80001FFA08
:103D300086F9039E3A464FEADC7C0EFB17671FFAB2
:103D40008AF652B283F809C00396059EDFF8DCC1FB
:103D500002EB860E6E4E6F4A1FFA8EFE83F80A90B3
:103D600082FB00A24FEAE07086FB016A684E049273
:103D70004FEAE17186FB07264FEAE777049AC1EB29
:103D80006A11C7EB6616644FC0EBA210BCF80020A6
:103D9000B7F800A04FEA1929029F83F80B904FEA69
:103DA0001E294FEAD77CC0F3072783F80FE04FEABC
:103DB000262E029783F80EC04FEA212C039F83F82A
:103DC0000DC038BF4FF0320C83F8109028BF4FF071
:103DD000330C19734FEA1729110A5E7483F812E045
:103DE0009DF80C60D8719DF808005E7583F81690F8
:103DF0001872DA74197583F81BC083F81CA0C4F814
:103E000010B1FEF709BCDFF82891D9F800000CF0DA
:103E100092F800283EF48EACD9F8000001210CF095
:103E200087F80222002386F874203B70FEF782BCDC
:103E300094F82C1194F82D314A1C3868013384F819
:103E40002C2184F82D310CF085F8FEF748BC334C5A
:103E50004FF0000ADFF8DC900AE01B2B00F08D82A7
:103E60000D2B00F071814FF0010389F801303868A3
:103E70000CF06DF800285FD038680CF062F8D8F8C4
:103E8000003083B27E2B2AD099F801100029EED1A0
:103E900094F82E21002AE0D07D2B00F0548294F873
:103EA0003CE1BEF1000F04D080F0200384F83C1107
:103EB000DBB2511C2244C9B282F83031092984F89E
:103EC0002E1100F034820829D1D8B4F83A211344D5
:103ED00003EB132303F0FF03A4F83A31C7E784F898
:103EE0002EA184F82FA189F801A0C0E7F83701209E
:103EF00024380120CC3E0120183801206766666610
:103F0000A03A01209C3A0120F83E01206BCA5F6B69
:103F10001F85EB51D34D62104A3B0120A01E0120AA
:103F2000806967FF83DE1B4340420F00483B01204E
:103F300030B401200000012094F83D3133B194F8F1
:103F4000313184F83D01302B00F0038694F82F21A5
:103F5000C74BC8499146DFF848A3DFF848E34A4613
:103F6000002A3EF4CCABD8F80020921B012A24D8BA
:103F700094F83E21002A40F01E8294F83FC133F8A5
:103F80001C00F8B94FF0010284F83F210A68970637
:103F9000E5D59AF800209007E1D5B74E4FF4F363CA
:103FA000B6494FF40360F28903FB02F381FB03215E
:103FB000DB17C3EB611117F0A1FF002384F82F3149
:103FC000FEF79DBB0CF1010CB0F5E06F5FFA8CFCC5
:103FD00084F83FC100F097801AD8B0F5047F00F054
:103FE000878134D8B0F5887F00F07481B0F5007F08
:103FF00000F05A81B0F5807FB1D10A685207AED582
:10400000002117F07BFF002384F82F31FEF777BBE8
:10401000B0F5026F00F015816AD8B0F5E46F00F0DA
:104020008180B0F5006F00F09880B0F5E26F96D116
:10403000934A6423166C118B03FB06F393FBF1F197
:1040400017F05CFF002384F82F31FEF758BBB0F562
:10405000826F00F0D580B0F5C06F00F0C180B0F580
:10406000806F7FF47CAF94F840310133DBB2032BD7
:1040700000F29B8142F2107184F8403101FB03F1A0
:10408000804B1B88002B40F08E8101317E4B1B78CA
:10409000DB077E4B1B8848BF0431DF0748BF0A316E
:1040A000980748BF14311A0648BF2831DF0548BFBA
:1040B0002831580748BF64311A0748BFC8319F05E7
:1040C00048BF01F5C87198064FF4806048BF01F5FC
:1040D0007A71DA0648BF01F5FA615F0648BF01F55B
:1040E0007A6117F00BFF002384F82F31FEF707BB2E
:1040F000B0F5046F1BD0B0F5116F57D0B0F5036F5A
:104100007FF42DAF42E791465D4A6423D66B118B55
:1041100003FB06F393FBF1F117F0F0FE84F82F9107
:10412000FEF7EDBA9146564A6423566CEFE7584BBA
:104130009146B3F9041001EB8101490017F0DEFE4E
:1041400084F82F91FEF7DBBA4FF0010184F830318B
:10415000A4F83A2184F82E1189E60A6897067FF5BB
:10416000FEAE9AF8002090077FF5F9AE1CF0010F23
:10417000414E424900F0DC84726882EAE273002A10
:10418000A3EBE27303EB5303A1FB03314FEAD1012D
:10419000ACBF41F0004141F040414FF4006017F0E6
:1041A000ADFE002384F82F31FEF7A9BA9EF8052052
:1041B000002A3FF4D4AE374A1278002A3FF4CFAE3B
:1041C000354B4FF411601B8803EB8303590091FBBF
:1041D000F2F117F093FE002384F82F31FEF78FBA27
:1041E0009EF80620002A3FF4BAAE2C4B4FF4C06074
:1041F000996817F083FE002384F82F31FEF77FBA09
:104200000A68900640F17681254B40F6B8321A4E86
:104210004FF482601F78317D07F00203002B0ABF44
:1042200000234FF47A734FF4FA6217F0010F18BFAE
:104230001346194417F062FE002384F82F31FEF76D
:104240005EBA0F68BF067FF58AAE9AF800C01CF010
:10425000020F3FF484AE084E64219146338901FB7E
:1042600003F117F04BFE84F82F91FEF748BA00BF18
:10427000106E0408983A0120A03A01201F85EB51E6
:10428000283A01206EB101200D720120603B01200F
:104290007C3A01205B3801202438012018380120A5
:1042A0009C3A0120843A01209EF80620002A3FF41F
:1042B00056AEBF4B4FF40070BE491B6881FB032113
:1042C000DB17C3EBA10117F019FE002384F82F318F
:1042D000FEF715BA0A6852077FF541AE00214FF488
:1042E000887017F00BFE002384F82F31FEF707BA11
:1042F0009EF80520002A3FF432AEAF4A107800281D
:104300003FF42DAEAD4B5B7B002B00F06A84AC4BD1
:104310001B8893FBF0F000EB80014FF40470490020
:1043200017F0ECFD002384F82F31FEF7E8B9B4F85C
:104330003A21C2F1FF0293427FF495AD4FF00103A1
:1043400084F83D318FE54FF0010384F83C318EE570
:104350000BF05EFC9B4A40F6B8331268801A984214
:1043600000F21C81DFF898A29AF804303A2B00F092
:10437000FF8200233B70FEF7DDB938680BF0E7FDE4
:1043800000287FF470AD4FF0010384F82F316EE503
:10439000C4F8203184F8183117F000FE8A4F94F8E1
:1043A0002431FEF782B9023170E6012342F2107126
:1043B00084F8403164E68549062017F069FB002344
:1043C00084F83E0184F82F31FEF799B9013B84F857
:1043D0005631FEF754BC7E4B1B88D90513D4DA0640
:1043E00000F1D583980600F13784590600F13A842C
:1043F0001A0700F13A84D80700F1558413F0020F30
:104400000CBF04260C26734B734A1B78D27803F03A
:1044100001030AB143F0020353201E4317F034FD99
:10442000674B1B8803EB830303EB8303980080B285
:1044300017F00EFD002017F00BFD684B684A1B8833
:104440003868C3EBC3135B0082FB0312D917134414
:10445000C1EB6323DAB2114602920BF07BFD029AA4
:104460009AF800300021386853408AF800300BF089
:1044700071FD314638680BF06DFD9AF800303868F0
:104480007340DBB219468AF800300BF063FD94F8F4
:104490004821FEF7A2BA013B84F85A31FFF722B84F
:1044A00009F1FF3984F85F91FFF742BB013A84F8C4
:1044B0005E21FFF7EDB8013984F85711FEF70ABD08
:1044C00048493A2017F0E4FA2870FEF749B92D223E
:1044D000DA7694E4444BD8F800101B78C4F8141131
:1044E000013B012B3FF69CAB10210223917013710D
:1044F000FFF796BB3D4A1268120600F132832F4A3D
:10450000127B002A3FF42BAD94F84111032900F2ED
:10451000C183DFE801F032281902354B1B68597955
:104520009A7901F14071DB7901EB022101EB034142
:10453000002384F841314FF4826017F0DFFC002340
:1045400084F82F31FEF7DBB82A4B1A68137A5079BA
:104550001B04927803EB002313444A1C03EB016114
:1045600084F84121E7E7234B1A68D37910791B04BB
:10457000527803EB00231344EFE71E4B1A6893793C
:10458000D0781B04127803EB00231344E5E717F0FF
:10459000F5FC194E01233370FEF75AB8174A002173
:1045A000B2F84A3139700133A2F84A31FEF7C2B885
:1045B00018380120676666665B380120F8370120ED
:1045C00024380120A8B30120203A0120F5BE0208BA
:1045D000603B01200D720120A0880120583001208D
:1045E00003082080C5D90208D82D012078A9012010
:1045F000007301206088012000000120A01E01201E
:1046000090B30120C84E0024C84B0AA8A6F13F0170
:10461000C74A00930891C74BC74906F8404C099612
:104620000CF0FFFB089E2920EA21C822731C089386
:104630003470089B5F1C089718700AA8089B5F1CC1
:1046400008971970089B591C08911A702EF03CFFAE
:10465000471C0AA908983A4632F029FADDF820E00A
:104660000122FF210EEB070312A8134408930EF852
:104670000740089B9F1808971C70089B9F18089775
:104680001C70089B9F1808971C70089B9F18089720
:104690001C70089B9F1808971C70089B9F18089710
:1046A0001C70089B9F1808971C70089B9F18089700
:1046B0001C70089B9F1808971C70089B9F180897F0
:1046C0001C70089B9F1808971C70089B9F180897E0
:1046D0001970089B991808911A7050F8283D9B1B77
:1046E000337019F03BF92C70FEF73AB818469A4629
:1046F00099469E4605931E469C461946FEF7F1BA1A
:10470000DFED8E7AB0EE677AFEF7DFBF864B12AD33
:104710008B4E00202F46A3F13D05112103F8400CDC
:1047200047F8205D022503F83F1C384603F83E5C3D
:1047300031680B9303970CF058FA384671680CF007
:1047400054FAF3897F49384603EBC3039B000533D2
:1047500081FB0321DB17C3EBA10189B20CF05BFAEB
:10476000338A384603EB8303590089B20CF053FABD
:10477000754B1B789B0740F13882318901F57A71BE
:1047800089B2039D28460CF046FA0A9B327D2846E2
:10479000591C0A911A7019F0E1F8FEF79BB8012232
:1047A000FFF7A1B8694A00205F4B21211268A3F1ED
:1047B00040070B9303F8400CD300B97040F14082DE
:1047C00003266349634B1B88580500F12F82DA07E3
:1047D00000F14582980701D503265F49DFF88C81F7
:1047E0003246404632F063F906EB0803A8F10202B4
:1047F0000021013312A806F808109A1A40F8203D4B
:104800007A7019F0ABF8FEF762B8C4F81CB186F8FC
:104810000090FDF71DBF444B002712AE4FF00A0C6D
:104820004FF0080EA3F13D004C4903F8407C4C4F7B
:1048300046F8200D304603F83FCC03F83EEC0988DB
:104840000B930CF0E8F93B6830463E49DA1781FBE0
:104850000313C2EBA30399B20CF0DDF9BF681DF09E
:10486000CBFD0A9B390C03F1010E3A0ACDF828E082
:1048700019700A9B591C0A911A700A9B5A1C0A92B9
:104880001F700A9B5A1C0A921870304619F066F87D
:10489000FEF71AB8334F12AE9FED338AB7F90220F4
:1048A00007EE902A204AF8EEE77A02F8403C0B9295
:1048B000A2F14003082267EE887AD91C5A701E22A2
:1048C00046F8201D3046FDEEE77A9A70CDED027A6B
:1048D000BDF808100CF09FF9B7F90030304607EE2C
:1048E000903AF8EEE77A67EE887AFDEEE77ACDED5A
:1048F000027ABDF808100CF08EF9B7F90430304692
:1049000007EE903AF8EEE77A67EE887AFDEEE77AFE
:10491000CDED027ABDF808100CF07DF9304619F0A3
:104920001DF8FDF7CEBF00BF4C3E01205988012085
:1049300060A0040858A004086CA00408000000004F
:10494000A03A0120676666669C3A01206436012021
:104950003CA00408603B012054A004082438012036
:10496000183801207C3A012058A08B410F3E0120CD
:104970009AF80240D4B1013C00235146E4B21A46F1
:104980000134544411F8013B160A53408C4283EA27
:104990000313DBB24FEAC30246EA032682EA13138B
:1049A00086EA0302EED1002A7FF4E3ACBF4A00217D
:1049B000BF4E1288BF4BF261BF4C1A68DFF83093CC
:1049C0009B68F262B4F84A21F066F364D9F80000FB
:1049D000F163F265FBF772FB029000287DF4A5AE4F
:1049E0000221D9F800000BF0A3FA94F84C3104220C
:1049F0009AF80310642B049186F8742040F07C81AF
:104A000094F84D31072B00F0118294F84D31AB4AE8
:104A100006EB031A06930292DAF804100846039193
:104A20002EF052FDDAF808105FFA80FA0846059178
:104A30002EF04AFD069BC0B2039903F00F0E02460A
:104A400023F00F009D4B039252449872039883F811
:104A50000DE002F1080E00EBCA00524683F807E0B1
:104A6000987303F10F0032F022F8954B0AF1090018
:104A70000599039A184432F01AF89049CB7903F15A
:104A8000010AF3B103F1FF3CC81D0023DFF864E223
:104A90005FFA8CFC0CF1080C8C4410F8011B594097
:104AA00084454FEA81034FEAD10283EA410302F0D1
:104AB000180283EA01034EFA02F283EA0203DBB230
:104AC000EBD17F4A04980AF802301AF063F894F8A0
:104AD0004D310022013384F84C2184F84D31029B82
:104AE0009B786BB1DDF808A01AF805100135D9F8EC
:104AF00000000BF02FFA9AF80230EDB2AB42F3D877
:104B000094F84C310322013386F874203A7084F80B
:104B10004C31FFF77AB9022138680BF009FA94F8A2
:104B20002431FDF7C2BD0123664E0293FDF721BF7C
:104B3000326882EAE273002AA3EBE27303EB5303C9
:104B4000A1FB03314FEAD101B8BF41F08041FFF72B
:104B500024BB5D49881F17F041F884F83E01FFF738
:104B6000F5B90026102004230AA98DF828008DF835
:104B700029308DF82A608DF82B608DF82C608DF827
:104B80002D6017F09BF984F82F61FDF7B8BD34262E
:104B900039E44E4BDB78002B0CBF04270527FEF7CA
:104BA000B2BE0123386833700BF0CBF90646386883
:104BB0000BF0C7F9720602D080287DF449AD8A282F
:104BC00056D08E287DF444AD94F81831002B7DF436
:104BD0005BAD3F4A2D23C4F8202184F82431FDF732
:104BE0003EBD324B1888FFF796BB4FF47A71C8E58B
:104BF0004FF0010A334EFEF787B92C4891790288AD
:104C000002EB820202EB82024FEA82091FFA89F963
:104C1000002900F01881274A126803930FFA82FADC
:104C20001DF0EAFB039B40B2FDF76EBF0326294946
:104C3000D4E508468A4689468E460591FEF751B866
:104C4000254B264A1B68264903F4800383420ABF8A
:104C5000114603260426B5E52426FFF7D4BB042617
:104C60002049BBE51026FFF7CEBB2026FFF7CBBBC4
:104C70001D4B1B689B067DF5EBAC94F81831002B9F
:104C80007DF402AD194A2D23C4F8202184F8243183
:104C9000FDF7E5BC4B1C0906DBB2042B84F841315F
:104CA0003FF446AC47E40826FFF7ADBB24380120AB
:104CB0000000012018380120A01E0120986C01205E
:104CC0009E6C0120A03A0120D81F0120A08801205D
:104CD000CC3E012048A0040878A9012040A0040887
:104CE0003CA004084CA00408983A0120F83E01209A
:104CF00030B401200007090E96F875C01CF00F0FA4
:104D000003D10CF1010C5FFA8CFCBCF1070F584B7E
:104D1000059528BF4FF0010C1A46029300234FEA75
:104D20000C1A02F10D0E937206EB0A035FFA8AF277
:104D3000197C504B03920B4493F82420039B012AC7
:104D40000EF1010541EA030106EB0A038EF800109B
:104D5000DB680CD9901E2A46C0B2811C714402F84F
:104D6000013B8A424FEA1323F9D101300544B24492
:104D70000CF1010C23F0600305F1010E9AF81120EB
:104D80005FFA8CFC1343BCF1080F2B7042D00399DF
:104D90004FEA0C1A384B103106EB0A02AEEB030354
:104DA000C9B20391117C334A0A4492F8242098181E
:104DB0001328C3DD059DDBB20298DFF8C8E09A1D19
:104DC000D2B242F0400102F1010AC171D2B1053301
:104DD00002990EF101000022DBB20833CB180393D5
:104DE00010F8011B51408A00CB0882EA410203F00F
:104DF00018034A40214941FA03F35A40039B834276
:104E0000D2B2EDD104980AF80E2086F875C019F0D8
:104E1000C1FE64E6184B059DAEEB0303CBE7184AD1
:104E200089466420B2F900A0FDF76EBE9DF80830F7
:104E300084F84D31E9E508468A4689468E46059153
:104E40000E46FDF74EBF4FF0FF32E6E60846FDF78F
:104E500048BF08468A46FDF744BF08468A46894649
:104E6000FDF73FBF08468A4689468E46FDF739BFA3
:104E7000986C0120106E0408A56C01200007090E33
:104E8000183801209E6C01202DE9F04F95B00C469A
:104E90001646B0F9083000AFDDB20B81442D00F0AA
:104EA0006B84804644D9812D00F0948300F2A28067
:104EB000542D00F0D68040F2E0806E2D00F02A8460
:104EC000802D40F0DD807B4B93F800A00AF1020AB0
:104ED0001AF0FF0A00F0A180774B0A25DFF8048260
:104EE0009A4403F10109754EDFF8FCB117E0322D49
:104EF00001F00D83A5F13C00C0B2132841F20E83EE
:104F000000232268CA4502F1010121601570226860
:104F100002F10101216013707FD019F8015B0A2DA5
:104F2000E5D1BBF80030FF2BA8BFFF23DBB2E8E7D9
:104F3000052D00F00F8420D8022D00F08A8040F269
:104F40002683032D00F0D383042D40F099802A4658
:104F50005B4920460BF03FFE002120460BF07EFE11
:104F60002168012300205437CD181A4625600870A7
:104F700018466281BD46BDE8F08F242D67D040F20F
:104F8000B382282D00F07083382D79D10A68012072
:104F90004FF0050E0A2602EB000C03460025494996
:104FA000C4F800C010700246206800EB030CC4F87F
:104FB00000C080F800E0206800EB030EC4F800E0B9
:104FC00006702068C6182660057020680D78C6181F
:104FD0002660057020684D78C61826600570206828
:104FE0008978C51825600170184654376281BD461E
:104FF000BDE8F08FA02D18D040F29A82B82D00F0B5
:105000007483FE2D3CD1304D05F1080635F8021BA6
:1050100020460BF023FEAE42F8D101231A46184673
:1050200054376281BD46BDE8F08F284B08461968A9
:105030000BF0FEFD264B204619680BF0F9FD254BC1
:10504000196820460BF0F4FD01231A46E7E7224BCE
:10505000F6E70422214920460BF0BDFD01231A4644
:10506000C2E7096801230020CD181A4625600870A0
:105070002168CD1825600870B6E7522D3FF470AF57
:105080002146284606F064FC03460028C5D1742D4D
:1050900000F09382772D29D1D8F80020D8F8041099
:1050A000914240F0768319460D4A20462DF0B6F81D
:1050B000B3E700BF61370120646E0408D07501209A
:1050C0005988012039B501208437012020F4F01FD0
:1050D00024F4F01F28F4F01FE4360120D8A00408BF
:1050E000F914040867666666F8750120F52D01F06D
:1050F0000583762D00F05283472D01F0AD82292DD6
:10510000D8F8006001F07B82392D01F03E82212D1C
:1051100001F04F82D8F804200B3D931BEF2D00F2D5
:10512000878601A151F825F0F15F0108315E010881
:10513000315E0108315E0108315E0108315E01080F
:10514000315E0108315E0108315E0108315E0108FF
:10515000315E0108315E0108315E0108315E0108EF
:10516000315E0108315E0108315E0108315E0108DF
:10517000315E0108315E0108315E0108315E0108CF
:10518000315E0108315E01082B600108315E0108C3
:10519000D75F0108315E0108B55F0108315E010883
:1051A000315E0108315E01083D5F0108315E010892
:1051B000B55E0108315E0108315E0108315E01080B
:1051C000315E0108315E0108A15E0108315E01080F
:1051D0003B5E0108315E0108DD5D0108315E0108BA
:1051E000315E0108315E0108315E01081B50010883
:1051F000315E0108BD5D0108315E0108315E0108C4
:10520000A15D0108315E010831580108315E0108D5
:10521000315E0108315E0108315E0108B1640108A8
:10522000315E0108315E0108315E0108BD6401088C
:10523000315E010815630108315E0108315E010825
:10524000A5620108315E0108315E0108315E010886
:10525000315E0108315E0108315E0108315E0108EE
:10526000C7610108315E010839610108315E01083A
:1052700087600108315E0108E9630108315E0108B9
:10528000B563010899630108315E0108315E0108C8
:10529000315E0108315E0108315E0108315E0108AE
:1052A000315E0108315E0108315E0108315E01089E
:1052B000315E0108315E0108315E0108315E01088E
:1052C000315E0108315E0108315E0108315E01087E
:1052D000315E0108315E0108315E0108315E01086E
:1052E000315E0108315E0108315E0108315E01085E
:1052F000315E0108315E0108315E0108315E01084E
:10530000315E0108315E0108315E0108315E01083D
:10531000315E0108315E0108315E0108315E01082D
:10532000315E0108315E0108315E0108315E01081D
:10533000315E0108315E0108315E0108315E01080D
:10534000315E0108315E0108315E0108315E0108FD
:10535000315E0108315E0108315E0108315E0108ED
:10536000315E0108315E0108315E0108315E0108DD
:10537000315E0108315E0108315E0108315E0108CD
:10538000315E0108315E0108315E0108315E0108BD
:10539000315E0108315E0108315E0108315E0108AD
:1053A000315E0108315E0108315E0108315E01089D
:1053B000315E0108315E0108315E0108315E01088D
:1053C000315E0108315E0108315E0108315E01087D
:1053D000315E0108315E010867630108315E010832
:1053E0009B640108315E0108315E0108315E0108ED
:1053F000315E0108315E0108315E0108315E01084D
:10540000315E0108315E0108315E0108315E01083C
:10541000315E0108315E0108315E0108435D01081B
:10542000ED5C0108AB5C0108315E0108615B0108BD
:10543000F55A0108D95A0108315E0108BF5A01081E
:10544000435C0108195C010887580108915801085C
:10545000315E0108915A0108315E0108315E010890
:105460006F5A01083B5A0108275A0108F3590108ED
:10547000315E0108D15901089B590108315E0108CC
:10548000315E0108315E0108315E0108315E0108BC
:10549000315E0108315E0108315E0108315E0108AC
:1054A000315E0108315E0108315E0108315E01089C
:1054B000315E0108315E010881590108315E010841
:1054C000315E010811590108315E0108315E0108A1
:1054D000315E0108315E0108315E0108315E01086C
:1054E000315E0108F7580108202D7FF4C9AD0B6823
:1054F0000846BC4D591C6A7821601A7023682A78C6
:10550000591C21601A702368AA78591C21601A70EE
:1055100029890BF0A3FB216801236879CE181A466C
:10552000266008702168A879CD18256008705BE5B1
:10553000822D7FF4A5AD0B680846AB4A5E1CAB4DCF
:105540001178A84A2660197011890BF087FBA84BC7
:10555000226820461B88511CFF2B2160A8BFFF2317
:105560001370A96881F3100189B20BF077FB2968E9
:10557000204601F30F0189B20BF070FB21689D4AB0
:1055800001231078CD181A46256008702CE5012DEE
:105590007FF476AD096800262B46242001F1010E28
:1055A0002A46C4F800E00E7021684E1C26600D707B
:1055B00021684D1C2560087016E5D8F80020D8F841
:1055C0000410914240F0E08019468B4A20462CF0AE
:1055D00025FE22E5894B1E78033616F0FF063FF4C0
:1055E0001CAD874B4FF00A09DFF83C821E4403F1E3
:1055F000010A20E0B9F1500F00F08687B9F1320FAF
:1056000000F0A287A9F13C00C0B2132840F2A487A1
:1056100000252946236820465A1C226083F8009002
:105620000BF01CFB294620460BF018FBB2453FF45B
:10563000F4AC1AF8019BB9F10A0FDBD171498B6800
:105640004FF6FF72096803EB830391424FEA43056B
:10565000A8BF1146954221EAE171A8BF154689B25B
:1056600025EAE575ADB2D5E70B68022101254FF0BB
:1056700006085E1C0A22DFF8B491204626601970E5
:105680002368614E5919216083F8008023685919F5
:1056900021601A7023685A1922601D70B9F8001031
:1056A0000BF0DCFAB9F8021020460BF0D7FA2368A9
:1056B0005021002203EB050E2046C4F800E083F8D9
:1056C0000080236803EB050EC4F800E0197023681E
:1056D000591921601A7031880BF0C0FA7188204680
:1056E0000BF0BCFA2B462A467EE4484BA8E4096836
:1056F00001230226002001EB030E1A46C4F800E045
:105700000D702168CD1825600E702168CD182560B8
:10571000087069E4364B08460A681B88511C334DF3
:10572000FF2B2160A8BFFF231370A96881F310012C
:1057300089B20BF093FA364B204619880BF08EFA9B
:105740002968204601F30F0189B20BF087FA012383
:105750001A4649E40B222F4920460BF03CFA082256
:105760002D4920460BF037FA07222C4920460BF032
:1057700032FA01231A4637E4002A3FF44EAC284A95
:10578000012332601A462FE4531CC8F80030117808
:105790001BE7531CC8F80030117885E4D8F80020C6
:1057A000511CC8F800101278002A01F02981102A33
:1057B00001F05E811E461946256820466B1C236059
:1057C0002A700BF035FA314620460BF031FA154BB2
:1057D000204659680BF02CFA002120460BF03EFAC7
:1057E000FFF7BABB843A01205B380120183801204A
:1057F00024380120D82D0120D92004086137012048
:10580000746E040884750120B8750120107301209E
:1058100058300120E0A00408ECA00408F8A0040817
:1058200031B9010864210120C8750120B436012076
:10583000721CDFF820930021B54BC8F800204046C9
:105840003278C9F800101A700BF09EF9D8F80020D1
:10585000D9F80030561CAF490343AF4D4046C9F854
:105860000030C8F8006013780B720BF0A4F92860C0
:1058700040460BF0A0F9686040460BF09CF9A86028
:1058800040460BF098F940460BF095F9FFF7C5BB81
:105890000D2B40F0CD82731CC8F800303578072DF1
:1058A00000F2C6820C26DFF8B092404606FB05F6F1
:1058B0000BF081F909EB0605A88040460BF07BF957
:1058C000E88040460BF077F9D8F800302881404650
:1058D0001A46591CC8F8001012F8021BA972C8F821
:1058E00000205B78EB720BF04FF9012349F80600BA
:1058F0001A46FFF779BB894B1B78DB0700F19882CA
:1059000007F0B4F807F080FA01231A46FFF76CBBE2
:10591000731CC8F8003033780F2B00F28982B51C55
:10592000C3EBC3027E49F01CC8F8005006F1040E18
:1059300075788B188D54751DC8F80000B01DB278AD
:10594000F11D5A7006F10802C8F800E096F803E06D
:1059500083F802E0C8F800503579DD70C8F800001F
:1059600070791871C8F80010B1795971C8F8002021
:10597000F2799A710CF092FD01231A46FFF734BBBD
:10598000684D40460BF017F9E88140460BF013F9DB
:105990000123A8811A46FFF727BB3046731C6249D2
:1059A00006F1030EC8F80030351D10F8022B012354
:1059B0000A701A46C8F8000070784870C8F800E00D
:1059C000B0788870C8F80050F078C870FFF70CBB4A
:1059D000564D40460BF0EFF8288240460BF0EBF8AE
:1059E000688240460BF0E7F80123A8821A46FFF7C9
:1059F000FBBA3146731C4E4AF01CC8F80030012334
:105A000011F802EB474D82F800E01A46C8F8001082
:105A100096F801E0474985F802E0C8F80000B07840
:105A20008870FFF7E1BA444B4E224449186831F0C0
:105A30003EF801231A46FFF7D7BA3246701C404B96
:105A4000F11CC8F80000404612F8025B1D70C8F84F
:105A5000002072785A70C8F80010B2789A700BF073
:105A6000AAF8384A0123D0801A46FFF7BDBA354D4F
:105A700040460BF0A0F8288040460BF09CF8688068
:105A800040460BF098F80123A8801A46FFF7ACBAFD
:105A9000DFF8C89099F80030002B3FF4BEAA2A4ED8
:105AA0000025404601350BF086F80DF03BFA99F8D9
:105AB0000030A6EC010A9D42F3DBFFF7AEBA174BAC
:105AC0001B78D8073FF5A9AA06F0B0FF07F09CF9AC
:105AD00001231A46FFF788BA104B1B78DA073FF507
:105AE0009CAA1A48012301781A4641F0040101706A
:105AF000FFF77ABA094B1B78D9073FF58EAA144AEB
:105B00004FF4C871012311801A46FFF76DBA00BF28
:105B1000903001200CAB0120A88701200D720120DC
:105B2000AC260120C4360120183C01203899012000
:105B300054A90120D436012060880120787304081C
:105B4000BC360120F47401204C7401209C3A0120E1
:105B500052370120E4360120B825012061370120A9
:105B6000092B40F365813346701CDFF84494F11C27
:105B7000321DD9F80050C8F80000701D13F802EB70
:105B800085F800E006F1060EC8F800307378AB70B7
:105B9000C8F80010F11DB378642BA8BF64236B71A3
:105BA000C8F8002006F10802F378642BA8BF64232C
:105BB000AB71C8F8000040463379EB71C8F800E0DB
:105BC0007379642BA8BF64232B72C8F80010B379D3
:105BD000EB70C8F80020F3792B710AF0ECFFD8F8CD
:105BE0000420D8F800306881D11A00290EDD581C35
:105BF000D9F80010121AC8F800001878002A487264
:105C000004DD9A1CC8F800205B784B7014F028FF64
:105C100001231A46FFF7E8B9731CC8F80030307842
:105C2000060600F18F87D04B1B78DD073FF5F5A9FD
:105C3000032828BF002006F0DFFE01231A46FFF7E5
:105C4000D3B9731C4046C8F8003096F800A00AF09B
:105C50009BFF814640460AF097FF064640460AF001
:105C600093FF054640460AF0A6FF40460AF0A3FF10
:105C700040460AF0ABFFBAF1000F00F04E87BAF1D0
:105C8000100F7FF4CAA9B94BC3F800905E600DB144
:105C9000B74B5D60B7490222B74B081F1A701FF05F
:105CA000C5FD01231A46FFF79FB9B44AF31C2136FC
:105CB000106802469D1E591E0332C8F8005013F8A2
:105CC000035C02F8035CC8F8001013F8021C02F829
:105CD000021CC8F80030033313F8041C9E4202F87B
:105CE000011CE7D10CF0CCFFFFF797B9731CA44A55
:105CF000C8F800303378002B00F00A87137843F09F
:105D00000203B11C13709F4D4046C8F80010737811
:105D10009D4E2B750AF038FF286040460AF034FF8C
:105D2000686040460AF047FF288140460AF043FF7A
:105D300031780123E88141F002011A463170FFF702
:105D400053B9C3F34705122D72D8C5B107F15003FB
:105D500007F12A0903EB450A4E46AAF1260A4046F6
:105D60000AF029FF26F8020FB245F8D1874B39F81F
:105D7000022F4E4523F8022FF9D1112D0AD86B00BE
:105D800083480021023B00F12202034423F8021F52
:105D90009342FBD101227F4913460A70FFF724B9D1
:105DA0007D4B06F108020136C8F80060964216F8ED
:105DB000011C03F8011FF6D1FFF72FB93146721C01
:105DC00076480123C8F8002011F8025B1A46857056
:105DD000C8F8001071784170FFF706B90722B3FBCD
:105DE000F2F2C2EBC2055B1B22D1D2B202F1FF3A42
:105DF0005FFA8AFA002A3FF410A90AF101021D464F
:105E0000DFF89CB1114632468A46511C644B4FF074
:105E10000009C8F8001092F9001093F90220083325
:105E20008A4200F0938509F10109B9F1060FF4D116
:105E30004FF0FF331A46FFF7D7B8731CC8F800308D
:105E400031780E29F4D8B31CC8F8003070780328D4
:105E5000EED80623534AF51C06F1040C03FB01F3AC
:105E600006F1050ED1184871C8F80050B51DB0787C
:105E7000D054F01DC8F800C00123F2784A701A46C9
:105E8000C8F800E096F804E081F802E0C8F8005095
:105E90007579CD70C8F80000B0790871FFF7A4B823
:105EA000721C41490123C8F8002030781A46487511
:105EB000FFF79AB8731C3C4D4046C8F80030337861
:105EC0002B720AF078FEA88340460AF074FE2883FD
:105ED00040460AF070FED8F8003068835A1CC8F8B3
:105EE00000201B78EB74D8F804309A1A032A00F3C8
:105EF000CB85D8F800105A1A052A11DD4B1C4046F4
:105F0000C8F800300B78EB720AF03EFED8F800308B
:105F1000E8605A1CC8F800201B782B7498E80A0027
:105F20005B1A002B7FF779A84A1C0123C8F80020D0
:105F30001A46097885F82110FFF756B8731C1B48DC
:105F4000D21AC8F800303378002A03707FF765A8AA
:105F5000B21C0123C8F800201A467178003118BF1E
:105F600001214170FFF740B80D7201207824012013
:105F7000642101207C240120FE3A01206088012058
:105F80009C3A0120A03A0120FC3A0120B2B2012043
:105F9000B4B20120D8B201200BAB0120E0360120C1
:105FA000DCB001201C7301200CAB012090300120DB
:105FB00000730120CB4D40460AF0FDFD28604046AD
:105FC0000AF0F9FD686040460AF0F5FD0123A8607B
:105FD0001A46FFF709B8C44D002340462B600AF06B
:105FE000D3FD2A68012310431A462860FEF7FCBF40
:105FF000102BBE494FF0000228BF10230A604A60F0
:106000008A60CA600A74002B3FF407A8D8F8002001
:10601000013913440132C8F80020934212F8010CF0
:1060200001F8010FF6D1FEF7F8BF731CC8F8003075
:106030003578132D3FF6FCAEB31CC8F800307078ED
:106040002CF026F900283FF4F3AE90F800E0F01CA5
:10605000A74B311D721D03F825E003EB8503C8F83B
:106060000000B578A3485D70C8F80010F1780068AA
:106070009970C8F800203279DA7014F07FFC01239F
:106080001A46FEF7B1BF731C9A4DDFF88492404662
:10609000C8F80030D5F800A0337889F805300AF048
:1060A0008AFDAAF8200040462E680AF084FD98E890
:1060B0000A00F0835A1A072A15DD40460AF07BFDD4
:1060C000A9F80A0040460AF076FD2E68A9F80C00EF
:1060D00040460AF070FD70842E6840460AF06BFD61
:1060E00098E80A00B0845A1A032A0BDD40460AF0E9
:1060F00062FDA9F80E0040460AF05DFD98E80A002E
:10610000A9F810005B1A002B06DD4A1C2B68C8F8A2
:1061100000200A7883F8262006F0B2FC25F0AEFCB9
:10612000754B1B68002B00F0E88428680CF044FADB
:1061300001231A46FEF758BF3346721CDFF8D09190
:10614000F11CC8F80020321D13F8025B404689F8A4
:106150000250C8F80030694D73782B70C8F80010F1
:10616000674DB3782B71C8F80020F378092BA8BFCE
:106170000923AB700AF01FFD98E80A0028805A1A1C
:10618000012A05DD40460AF016FD98E80A00E8817C
:106190008B4208D04B1CC8F800300B78003318BF76
:1061A000012389F8073006F06BFC98E80A008B425F
:1061B0003EF433AF4A1C0123C8F800201A46097880
:1061C000E970FEF711BF40460AF0F5FC05461FF0E6
:1061D00013FCFF283EF421AF3F2D00F277844FEAF5
:1061E000D509002307F1500607F12B0009F1010939
:1061F00087F82B3006F8243D314618F095FB97F8C8
:106200002B305FFA89F905F007054B4505F10105CB
:1062100003D197F82C30AB4203D0294648461FF0F3
:10622000D7FBD8F80030D8F80420D21A012A7EF71C
:10623000F4AE591C002207F15000C8F800101D7878
:1062400000F8252D18F064FB97F82B30AB420AD0EC
:106250002C4B1B683BB19A79AA4204D31B681B697B
:106260000BB128469847D8F8003000223046591C18
:10627000C8F800101D7887F82C2018F03DFB97F81F
:106280002C30AB423EF4C9AE1E4B1B68002B3EF4D3
:10629000C4AE1B685B69002B3EF4BFAE284698472E
:1062A000FEF7BBBE184B1B78012B3EF6B6AEF31CB7
:1062B000701C3146154DD21AC8F8000011F8020BB7
:1062C000012AA870C8F8001096F801E0C8F800305C
:1062D00040F3578440460AF06EFC012328801A469A
:1062E000FEF782BEA8870120E4360120A0360120F7
:1062F00094300120608801208C300120B8360120C4
:10630000389901200452012065B6012068B60120A9
:1063100054A90120731CC8F8003096F80090B9F118
:10632000110F3FF685ADB31CC04D4046C8F8003094
:106330007378192605F8193005EB49050AF03BFC7E
:1063400040F6CA0340F2EE229842A8BF1846012345
:106350009042B8BF10461A46A0F2EE2191FBF6F12A
:106360006970FEF741BE711C3346F21CC8F800107C
:1063700013F8025BC8F800307078C8F80020B178D4
:10638000002D00F0EA83012D7EF447AE24F074FC6A
:106390002B462A46FEF728BEA54B1B7813F00101B9
:1063A0007FF446AD731CC8F80030307824F016FC3A
:1063B000FEF733BE3146731C9E4AF01CC8F800300D
:1063C000012311F802EB9C4D82F803E01A46C8F84D
:1063D000001096F801E0994985F805E0C8F800003A
:1063E000B078C870FEF700BE4046954D0AF0E3FB5A
:1063F00040460AF0E0FB40460AF0DDFB40460AF06A
:10640000E5FBD8F800302A684046194603F1010E32
:10641000DE1CC8F800E011F802EB82F82CE0C8F8A6
:106420000010597882F83610C8F800609B7882F81E
:1064300037300AF0CBFB40460AF0C8FB40460AF072
:10644000C5FB2E6840460AF0B6FB708740462E68B2
:106450000AF0B1FB98E80A0030875A1A012A0BDDCE
:106460004A1C2B684046C8F800200A7883F82E2082
:106470000AF0ACFB98E80A005B1A032B0BDDD5F899
:10648000009040460AF097FB2E68A9F8320040467B
:106490000AF091FBB086286824E40023694D404649
:1064A0002B600AF071FB012328601A46FEF79CBDA1
:1064B000FBF7B2FC01231A46FEF796BD3346721C69
:1064C000614D4046C8F8002013F8022B2A71C8F825
:1064D000003073786B710AF06EFBD8F800302880BA
:1064E00040465A1CC8F800201B78AB710AF063FBC9
:1064F000D8F8001001236880C8181A46C8F80000B0
:106500000978E971FEF770BD5049FFF798B83388F4
:10651000FF2BA8BFFF23DBB2FEF7F3BC15F09EF9FB
:1065200000283EF4EDAC03780A2B2CD8B0F90230E9
:1065300088FB0312DB17C3EBA2039BB2FF2BA8BFA0
:10654000FF23DBB2FEF7DDBCD8F804304FF6FF7254
:10655000D8F80010FFF777B815F080F900283FF45D
:1065600057A803780A2B3FF653A8B0F90430B0F9C6
:10657000061003EB830321EAE17183F3500589B22E
:10658000ADB2FFF747B80023DBE7731CC8F8003053
:1065900033780A2B00F0C08140460AF017FB4046D2
:1065A0000AF014FB40460AF011FB01231A46FEF7DD
:1065B0001BBD3346711C264DF21CC8F80010404626
:1065C00013F8021B6970C8F8003073782B70C8F894
:1065D0000020B378AB700AF0EEFAD8F8001001236F
:1065E0002881CE1808461A46C8F8006010F8026BD9
:1065F0006E71C8F800004978A971FEF7F5BC731CEC
:10660000C8F8003033780A2B00F0E580502B7FF477
:1066100037A9104D40460AF0CEFA288040460AF0CD
:10662000CAFA012368801A46FEF7DEBC80B4012056
:106630000D720120C43601206C3F0120D4360120A8
:1066400060880120107301200C750120BC750120A9
:10665000843A0120B8750120D8F804204046D8F8C3
:1066600000507B62551B0AF08FFA7B6A052D386259
:1066700000F2A28080260125B34620467B6294E882
:106680000600521A396A103A9642C8BF1FFA82FBB6
:10669000C34A92683A61521A396A9345FA6088BFD0
:1066A0001FFA82FB0AF0C4FA7B6A002B40F0958047
:1066B000002D00F08781BA4BD4F800809D683B6ABA
:1066C0005B449D4280F03E813B6AED1A0AF012FE67
:1066D0002A464146386AFBF727FA23688642034474
:1066E00023607EF79AAC002100E0236801305A1C39
:1066F000864222601970F8D1FEF78FBCD8F80030BE
:10670000D8F804209A4240F08081A64BFF221A70EC
:106710004FF00008A44D23F02DFC20224146A34851
:1067200085F8008030F0E8F987F82C80424697F829
:106730002C30072B33D8DFF88892DFF8708297F877
:106740002C3003EB430309EBC3035B7CEBB197F8FD
:106750002C30202103EB430309EBC3035B69A3B196
:1067600097F82C3003EB430309EBC3035B6948F84C
:106770002230184609F099FD2B7858F8230009F0CB
:106780009EFD2A780132D2B22A7097F82C3001335C
:10679000DBB287F82C3097F82C30072BCFD9236841
:1067A000591C21601A70002E3EF437AC804A012338
:1067B00032601A46FEF718BC40460AF0FCF9D8F8D9
:1067C0000020D8F8041083467B6A914240F046814D
:1067D00006461D4651E7774D1CE722680023C7F89F
:1067E00000D0C0B0511D5371C7F808D0F961BBF19A
:1067F000000F00F045813A6A39698A4280F03D8194
:106800007C609A463D6A4FF080091C467B62FB68BB
:106810001C1B634BB4F5807F9B6828BF4FF48074CA
:1068200062199A4288BF5C1B0AF064FDBE68284664
:1068300022463146FBF778F9F96906EB000CB8619E
:106840000C7866457C6132D20CF1FF3C06F1FF3ECC
:106850001EF8013F584A584802EB830210F82350B3
:1068600056880DB300234FF4004205F1FF3816425D
:106870000AF101044FEA520203D0087849EA000005
:1068800008705FEA590906D181F801901FFA84FA6D
:1068900001314FF08009DA4503D3F44536D89845E5
:1068A00034DC01339D42E2D1F445D1D1F9617B6AF8
:1068B000DA45BA6913449BB27B6206D27B6A3A6AB4
:1068C0001C46D5183B699D42A1D37C68B9F1800F65
:1068D00003D00AF101031FFA83FA0AF102012046EC
:1068E000012589B20AF0BAF92368796A20465A1953
:1068F00022601D700AF0B2F922682B4602EB0A01F1
:106900002A462160D7F800D0FEF76EBBFB697C6891
:106910001A463B7D1370D9E7B31C2849F51C301D7E
:10692000C8F80030012396F801E01A4681F800E02B
:10693000C8F80050B5784D70C8F80000F07888703D
:10694000FEF752BB0AF0D6FC5A46C2E60BEBC9066C
:1069500040460135B1700AF02EF9D8F800302BF816
:106960003900AA45194603F1010203F10300C8F8F2
:10697000002003F1040211F802EB86F803E0C8F8E6
:10698000001059783171C8F800009978B171C8F8D1
:106990000020DB7873717FF438AAFEF73EBB00BF9E
:1069A000400801206421012093240120ACB3012080
:1069B000E5160208B4360120846E040839B50120BA
:1069C00078980120594620460AF048F923683A6A27
:1069D000591C5A4421601D70704B26689D68954271
:1069E000C0F0C1800AF086FC5A463146386AFBF78F
:1069F0009BF82268012310441A462060FEF7F4BA7F
:106A0000674B93E84200FEF7D7BE5A1C194665480B
:106A1000C8F8002011F8022B0270042AC8F80010F0
:106A20005B78437003D9FF2A7EF49AAA70E65E4928
:106A30000978994205D8FF2B7EF492AA022A7EF4A7
:106A40008FAA22680123D11821601370002E3EF412
:106A5000E4AA56491A463160FEF7C6BA511C1D46D3
:106A60000646C8F800101378003318BF012304E667
:106A70004F4B93E84200FEF79FBE7B629A462CE79D
:106A8000DA46C7F824B028E740460AF094F8A8840C
:106A900040460AF090F898E80A00E8845A1A032A57
:106AA0007FF729AA0B464A1C4046C8F8002013F875
:106AB000022BAA77C8F800304B7885F820300AF00E
:106AC0007AF898E80A006884FFF715BA07F12C06EF
:106AD00030461EF071FFBB8DAB423FF4A2AB354B8D
:106AE0001B68002B3FF49DAB1B689B69002B3FF498
:106AF00098AB28469847FFF794BB2F4901232F4EA8
:106B00002F4D1A462F48316029600160FEF76CBA9C
:106B1000137803F0FD03FFF7F4B8214B1020C3F8FE
:106B200000905E6021F042FB274A137843F0010396
:106B30001370002D3EF471AA1A4A012355601A46BB
:106B4000FEF752BA00F07F00032828BF002024F08F
:106B5000B1F801231A46FEF747BA0BF0F7FE0123FE
:106B60001A46FEF741BA3B6AED1A0AF0C3FB3146FA
:106B7000386A2A46FAF7D8FF236803442360FEF7F1
:106B80004CBA124A0123B07811881A4611FB0EF153
:106B900091FBF0F12980FEF727BA00BF40080120E1
:106BA000403B012064210120613701203DB90108EB
:106BB000782401200452012019F80108242701201B
:106BC00078270120782B01209C3A0120843601206F
:106BD000444B2DE9F04F2DED0A8B1B7893B0012B20
:106BE000069001F05085404C94F80021002A40F0B6
:106BF000A587072B3D4D01F04185002303936B686A
:106C00003A489847002800F0CA800022B5F8B870CA
:106C100085F85920002F41F09C81B5F944702B6D07
:106C2000B5F94060A7EB030EA86AB5F942108EEAE9
:106C3000EE72301AEE6AA2EBEE726863891BB2F54F
:106C4000804FA96301DC3B462F652A6BDFF8A8B0B3
:106C50009B1A95F85A102648EB630FF007FDDBF8F6
:106C600000309E0040F19D8695ED0E7AD5ED0D7AAF
:106C7000B8EEC78A95ED0F7AD4F8A031F8EEE77A2E
:106C8000F8EEC78A1B4A94ED656A0133D4ED666A53
:106C900094ED677A77EE867A126838EE268A78EE77
:106CA000878AC4F8A0319342C4ED657A84ED668A80
:106CB000C4ED678A02F06E800A4B1F78142F02F031
:106CC00088870023D4F8A8610493062E00F25C861E
:106CD000DFE816F056143614CE134C16C605C3154D
:106CE0001D1500BF803701206C21012068A1012003
:106CF0009CA10120F430012078A90120CE4E00276C
:106D0000DFF8AC9306F2DC68DFF8A8A3CB4B1B7866
:106D1000172B01F01C8096ED007A082BD5ED097A2F
:106D2000B8EEC78A28EE278A07D1B0EE480A049346
:106D30002DF0BCFD049B2AF81700DBF80020900022
:106D40000BD5002F04F01A85B0EE480AD5F87C3731
:106D500008F170009847B0EE408AB0EE480AD5F8C6
:106D60009C36A8F170009847D5F80C3740469847F4
:106D7000B24BB0EE408A1B78032B00F0F887013746
:106D8000D6F85C06B0EE480AD5F8BC309847032F19
:106D900008F1240806F10406A9EC010AB6D1A74BB4
:106DA0001E78072E01F0918194F8B831002B40F045
:106DB0002686A34B5B79002B40F0378501239F4A41
:106DC00084F8B8311278072A01F0B68700230993B6
:106DD0009C4BF7EE007ADFF8E082002693ED007A14
:106DE000994B3546D4ED709AD3F800A008F16803AA
:106DF00077EEE98A954F0893954B68EE878ADFF81E
:106E0000BC920393934BD4ED6FBAC8FEE78A049308
:106E1000914BDFF8ACB207939FED909A904BDFED6A
:106E200091AA9FED91BA9FED91AA0593904B98ED91
:106E3000008A3344D3ED007AF5EE407AF1EE10FA91
:106E400017D08C4B3344D3ED006A38EE667AB0EE3F
:106E5000C76AF4EEC67AF1EE10FA08D5B5EEC07A3C
:106E6000F1EE10FACCBF37EEA68A36EEE78A83ED54
:106E7000008A049B1A8891073BD0022D39D07E48A6
:106E80009AF82E1030F91500089B07EE901A07EEBD
:106E9000100A68003344B8EEE76AB8EEC77AD3ED5B
:106EA000006A4B42A6EE267A07EE903AF8EEE77AB1
:106EB000B4EEE77AF1EE10FA05D407EE901AF8EE88
:106EC000677AC7FEC77A6D4BD2076D490344085EE7
:106ED000B3F90C30A0EB030007EE100AB8EEC77A46
:106EE000E7EE497A40F19385664B93ED008A27EEF1
:106EF000888A059B94F8D0213344D3ED01CA38EE3B
:106F00006CCA002A3BD0D4F8D4215F4B06991B6889
:106F10008A1A9A4233DD9AF84830022B02F0248014
:106F2000022D04F0A983594B1B689B0740F1F6869C
:106F3000524B534903EB4500DFF848C131F915E0E6
:106F4000B0F90C009CED008AA0EB0E0E504828EE24
:106F5000098A87ED00BA07EE90EA0068F8EEE77A52
:106F6000904227EE888A38EE6CCAC1F2C681F7EEED
:106F7000007AF4EEE79AF1EE10FA01F19581454BB3
:106F8000022D334493ED000A039B2BEE800A20EE82
:106F90000C0AA3EC010A039304F09183079ADBED3A
:106FA000006AD2ED007A3C4B66EEA77A97ED006A54
:106FB000334467EEA87A93ED007A384B67EE877A10
:106FC000D3ED005AB0EE467AF1EE656AACEE277A60
:106FD000B4EEE67AF1EE10FA01D4C7FE656AF7EE78
:106FE000007A94ED707AB4EEE77AF1EE10FAACBF65
:106FF0000123002343B1B0EEC66AF0EEE67AF4EE68
:10700000C67AF1EE10FA01D5C7ED006A022D00F044
:10701000A180234AB0EE6C0A224B52F825001B686F
:107020009847214A214B52F825001B6898479AF847
:107030003730002B4BD045E09CA101208037012048
:1070400054A90120CC2B0120608801204030012070
:1070500034300120603B012078000120CDCCCC3DB4
:1070600068A90120AE47813F000000000000C8422F
:10707000C02B012030230120FC220120C436012036
:107080007C3A0120A82B0120D42B0120983A012022
:10709000D02B01207C2B0120882B0120F02B0120FC
:1070A00028270120242701207C2701207827012080
:1070B0006CA9012084370120702201204C3001206E
:1070C00020270120049B1B88002B00F0F784B0EEE2
:1070D0004B8AD84B38EE400A9BED007A334493ED4F
:1070E000008A83ED000A30EE480A9AF84830C0EE74
:1070F000077A2BB3D04B1B78D90721D5B7EE007A8E
:10710000F4EEC79AF1EE10FA04DB94F8D031002BBC
:1071100000F0D886D4F8D431069AD31AC74A126838
:107120009A420DDDC64BB0EECCCA93ED007AB4EEB8
:10713000C7CAF1EE10FA41F1FC80002384F8D03187
:10714000C04B334493ED007A2BEE877A67EE277AB3
:10715000C9ED007A94F8E03133B9039B87ED00BAAA
:1071600003ED01BA89ED00BA013508F104080437CE
:1071700009F10409032D06F104067FF457AEB24B62
:107180001B78072B01F09D82012B01F0DA85002688
:1071900094F8E831002B40F08B85AC4AAC4B116879
:1071A0001B6893F82C2011F48053039340F0E5857D
:1071B000A8480123408B84F8003207EE900AA64BC2
:1071C000A648B8EEE77AD3ED037AA54BD0ED006A76
:1071D00093ED006A77EEC77AA24B76EE665AC4ED5D
:1071E0007E6A93ED007AC4ED7C6AC4ED7B5A84ED2F
:1071F0007F6A9D4BC7EE875ADFED9C4A93ED006A8C
:107200009B4BD3ED007AB7EE005A9A4B36EE276AC5
:10721000DFED997A93ED004A984B36EE046A93EDD0
:10722000007A26EE246AF1EE476AC5FEC55AC5FE0D
:10723000A75AB4EEE66AC4ED815AF1EE10FA01F1F4
:10724000878086FE476A884BD3ED017A884B93EDA1
:10725000015A884B77EE857A9FED845AD3ED014A27
:1072600077EEA47A67EE857AF4EEE76AF1EE10FA2B
:1072700001DCC7FE676A7C4B9FED7C5AD3ED027A36
:107280007B4B93ED027A7E4B77EE877A93ED007A13
:1072900067EE857AF1EE473AF4EEE37AF1EE10FA12
:1072A00001D4C7FEC73A774B5B780BB9F1EE633A6E
:1072B000002A41F08183B7EE004A734D2A78002AF4
:1072C00002F06B84714BDFED6C4A93ED025A93ED43
:1072D000017A26EE855AD3ED037AA6EE075AA3EE7D
:1072E000A75A24EE055AB4EEE45A85FE647A8DED71
:1072F0000A5AC5FE247AF1EE10FA88BFB0EE647A1D
:10730000012A02F0C285D3ED064AD3ED052A66EEC6
:10731000A44A93ED073AE6EE224AE3EE834A64EE8E
:10732000244AF4EEE74ACDED0B4AC4FEA77AC4FE28
:10733000C74AF1EE10FA98BFB0EE647A022A00F064
:10734000DF80D3ED0A4AD3ED092A66EEA44A93ED15
:107350000B3AE6EE224AE3EE834A64EE244AF4EE68
:10736000E74ACDED0C4AC4FEA77AC4FEC74AF1EE47
:1073700010FA98BFB0EE647A032A00F0C180D3ED12
:107380000E4AD3ED0D2A66EEA44A93ED0F3AE6EECF
:10739000224AE3EE834A64EE244AF4EEE74ACDED56
:1073A0000D4AC4FEA77AC4FEC74AF1EE10FA98BF90
:1073B000B0EE647A042A00F0A380D3ED124AD3ED34
:1073C000112A66EEA44A93ED133AE6EE224AE3EE62
:1073D000834A64EE244AF4EEE74ACDED0E4AC4FE39
:1073E000A77AC4FEC74AF1EE10FA98BFB0EE647AED
:1073F000052A00F08580D3ED164AD3ED152A66EEF6
:10740000A44A93ED173AE6EE224AE3EE834A64EE8D
:10741000244AF4EEE74ACDED0F4AC4FEA77AC4FE33
:10742000C74AF1EE10FA98BFB0EE647A062A67D028
:107430002EE000BF442301200D720120D42B012037
:10744000E02B0120942B01208037012078A9012016
:10745000608801200CAB01205C3801200C35012034
:107460009C360120FC740120343001206F12833AD5
:10747000403001204C30012000000000F42B01209E
:10748000F82B012090300120613701206C7401201D
:10749000D3ED1A4AD3ED192A66EEA44A93ED1B3AAE
:1074A000E6EE224AE3EE834A64EE244AF4EEE74A2B
:1074B000CDED104AC4FEA77AC4FEC74AF1EE10FA19
:1074C00098BFB0EE647A072A1AD0D3ED1E4A93ED26
:1074D0001D3A66EEA46AD3ED1F4AE6EE036AE4EEB7
:1074E000A36A66EE846AF4EEE76ACDED116AC6FE21
:1074F000A77AC6FEC76AF1EE10FA98BFB0EE667AB8
:1075000077EEC77AF7EE006AC4ED707AF4EEE67AA9
:10751000F1EE10FA43F36A8586EEA77ADDED0B7A79
:10752000022A27EE055A67EE877A8DED0A5ACDEDCD
:107530000B7A2DD0DDED0C7A032A67EE877ACDED3C
:107540000C7A25D0DDED0D7A042A67EE877ACDED31
:107550000D7A1DD0DDED0E7A052A67EE877ACDED26
:107560000E7A15D0DDED0F7A062A67EE877ACDED1B
:107570000F7A0DD0DDED107A072A67EE877ACDED10
:10758000107A05D0DDED117A27EE877A8DED117A2C
:10759000A94B1B6813F0805B01F08E80F6EE005A59
:1075A000C4ED815A002A02F0EF82D4ED7F7A01F017
:1075B0001007A24B01F48001FDEEE77A94ED7E5AAC
:1075C00093F803E094F900329D4806EE903A17EEE6
:1075D000903AFDEEC57A0078DFF870A2F8EEE66A20
:1075E000DFF86C9200F00100DFF86882DFF868C213
:1075F000049117EE901A9AF800A0D9ED007AB8F924
:107600000680BCF81AC094ED7B6A94ED7C7ABEF1DA
:10761000000F41F00B82002F41F09C80DFF83CE22C
:107620009DED0A5ADEED007A864F65EEA77AE6EE0A
:10763000857AB0EE475AA6EE275AFDEEC57A17EEC8
:10764000908A17EE90CA9845A8BF9C464145C8BF8E
:107650008C46012A07EE90CAF8EEE77AC7ED007A69
:1076600000F0DC80DEED047A9DED0B5A65EEA77A22
:10767000E6EE857AB0EE475AA6EE275AFDEEC57AB9
:1076800017EE908A17EE90CA9845A8BF9C464145D0
:10769000C8BF8C46022A07EE90CAF8EEE77AC7ED1B
:1076A000017A00F0BB80DEED087A9DED0C5A65EEA4
:1076B000A77AE6EE857AB0EE475AA6EE275AFDEE97
:1076C000C57A17EE908A17EE90CA9845A8BF9C46D7
:1076D0004145C8BF8C46032A07EE90CAF8EEE77A08
:1076E000C7ED027A00F09A80DEED0C7A9DED0D5A1E
:1076F00065EEA77AE6EE857AB0EE475AA6EE275AEF
:10770000FDEEC57A17EE908A17EE90CA9845A8BF8D
:107710009C464145C8BF8C46042A07EE90CAF8EE45
:10772000E77AC7ED037A79D0DEED107A9DED0E5A37
:1077300065EEA77AE6EE857AB0EE475AA6EE275AAE
:10774000FDEEC57A17EE908A17EE90CA9845A8BF4D
:107750009C464145C8BF8C46052A07EE90CAF8EE04
:10776000E77AC7ED047A59D0DEED147A9DED0F5A11
:1077700065EEA77AE5EE267AB0EE475AA7EE865A6E
:10778000FDEEC57A17EE908A17EE90CA9845A8BF0D
:107790009C464145C8BF8C46062A07EE90CAF8EEC3
:1077A000E77AC7ED057A39D0DEED187A9DED105AEB
:1077B00065EEA77AE5EE267AB0EE475AA7EE865A2E
:1077C000FDEEC57A17EE908A17EE90CA9845A8BFCD
:1077D0009C464145C8BF8C46072A07EE90CAF8EE82
:1077E000E77AC7ED067A19D0DEED1C7A9DED115AC5
:1077F00065EEA75AE6EE855AA6EE257AFDEEC77A23
:1078000017EE90EA7345A8BF73467145C8BF0B4693
:1078100007EE903AF8EEE77AC7ED077A002840F0D5
:107820005482002A40F04C824FE2074B1B78013B08
:10783000DBB2FFF7C4BA00BF64360120A088012084
:107840000D7201206C300120B83601205C990120B6
:1078500048740120507001200CAB01206C74012091
:10786000A14B1A78D4F8ACE1DFF8C4C24FEACE00DD
:107870009FED9E7A0CEB000383ED007A002A78D00E
:10788000B0EE476A9A49F0EE476A00230133F1EC03
:10789000017A05EE903A67EEA77A9342F8EEE55A40
:1078A00087FE277A76EEA76AA7EEA56AEED1F5EEF7
:1078B000C06A0CEB000383ED007AF1EE10FA58DD9C
:1078C000C6EE265A8B4A8C4BD2ED007A1A88B7EE58
:1078D000000A75EEC05A65EEA77AFDEEE77A17EE5C
:1078E000903A812B42F311849342A8BF134607EECE
:1078F000903AF8EEE77A00EB0E01804B03EB810340
:1079000093ED007A93ED056A93ED015AA7EE276A8D
:10791000D3ED066A93ED047AE5EE276AD3ED034AC8
:1079200093ED025A27EE467ABDEEC64AE6EE646A49
:10793000A5EE277A14EE101A8129C3ED056A83EDAE
:10794000067A42F3E6838A42A8BF0A4607EE902AE7
:10795000F8EEE77AFCEEE77ACDED057ABDF8143063
:107960000CEB00029380BEF1000F02D1132F03F045
:107970003183152F41F0D5856044DFF8B881D4F804
:10798000A861838828F81E3001365D4A82FB0632E2
:10799000F3173244C3EBA203C3EBC303F61AC4F8D4
:1079A000A861584B1B78002B7FF4A8A9564FDFF82D
:1079B000889107F24C7607F5F768F7EC017A3046C4
:1079C00095ED090AF8EEE77AD5F87C3727EE800ABC
:1079D0009847A6F1E000D5F89C369847A6F17000CC
:1079E000D5F80C3724369847D7F85806D5F8BC3068
:1079F0009847B045A9EC010ADFD1FFF7D0B9013BA8
:107A000084F8B83113B0BDEC0A8BBDE8F08FB1F942
:107A10000020B1F9021082EAE27394ED5E7AD4EDAF
:107A20005F6AA3EBE27381EAE17286FE876AA2EBEA
:107A3000E17236499342B8BF13460A7807EE103A0E
:107A4000B8EEC77A27EE097A002A40F0D981304B88
:107A5000D3ED005AF4EEEA5AF1EE10FA41F1FD804E
:107A6000B7EE005ADFED2B6ADFED2B4A36EEC77A10
:107A70002A4B35EE655AD3ED006A25EE245AE5EE21
:107A8000075A65EEA65AF5EEC05AF1EE10FA40F22A
:107A90000F86CAEE256AB7EE007AF0EE475AE6EE98
:107AA000665AC5FEC76AC6FE8B6A1D4B93ED007A07
:107AB00067EE877AA7EEA68AFFF71BBA194BF7EE97
:107AC000006A194A3344D2ED007A93ED007A174BDD
:107AD00067EE277A93ED007AC7FEE67A67EE877A3B
:107AE00027EE888AFFF7F5BAFA300120000000007F
:107AF0006C210120FC300120F830012030330120BE
:107B000093244992EC3001209CA10120B42B012048
:107B1000BC2B012000003443610BB63BB02B01208D
:107B2000AC2B0120E4220120A42B0120A02B01205A
:107B300018330120843701206CA90120072B02F0A3
:107B400058800027DFF874B3C24DDBF800305905C8
:107B500001F1E880C04B1B78002B40F0DE81BF4E66
:107B600094F8123123B1BE4A1288920741F0CD87B2
:107B700094F81831002B41F07580B27F002A00F094
:107B80000184022A01F0B587032A01F05683B54A21
:107B90005188F27F0232D2B2002901F0A087002B77
:107BA00001F09D87B0480068B1FBF0F10FFA81F950
:107BB000A4F84891B2B307EE909AF7EE005AAB4999
:107BC000012AB8EEE76AD4ED576AD1ED007A85EE66
:107BD000867A77EEE67A67EE877AC4ED537A21D01B
:107BE000D1ED017A022AD4ED586A77EEE67A67EE93
:107BF000877AC4ED547A15D0D1ED027A032AD4EDF8
:107C0000596A77EEE67A67EE877AC4ED557A09D03D
:107C1000D1ED037AD4ED5A6A77EEE67A67EE877A89
:107C2000C4ED567A92490978092903F01182B9F115
:107C3000000F40F3AA83002A02F02B8594ED577AB7
:107C4000012AD4ED537A894977EE877AC4ED577AC1
:107C5000C1ED007A21D094ED587A022AD4ED547AFD
:107C600077EE877AC4ED587AC1ED017A15D094ED9C
:107C7000597A032AD4ED557A77EE877AC4ED597A8A
:107C8000C1ED027A09D0D4ED5A7A94ED567A77EEA6
:107C9000877AC4ED5A7AC1ED037A013A022AB8BF55
:107CA0000222D2B2002B0CBF96464FF0020E72E3B6
:107CB000704B714D1B78DA0700F128822A7822B1C7
:107CC00092006E496E482EF0F2FE6E4B1B68002B40
:107CD00040F042836C4B1B789BB1287870B1DFF881
:107CE000A0810027DFF8D891F8B2D9F80030B8ECBD
:107CF000010A0137984728788742F5DB634B1B68F8
:107D000098475B4B1B78072B00F0F084012384F825
:107D1000003113B0BDEC0A8BBDE8F08F5C4B87EDF2
:107D200000BA1B689342BFF622A95A4A0023128860
:107D300084F8D031002A41F0C086574A574B117859
:107D4000186881F0010108F0BFFAFFF718B996ED45
:107D5000007A05EB4702D5ED097AB8EEC78AB2F88A
:107D600040202AF8172028EE278AFEF7E6BF2CF0DD
:107D70009DFD2AF81700FFF702B83E4B1B78DB0782
:107D800003D4364B1B8BA4F8F431454B37481B8882
:107D900090ED037A07EE903AF8EEE77AB4EEE77AE0
:107DA000F1EE10FA41F236813E48008807EE900A63
:107DB000F8EEE77AB4EEE77AF1EE10FAC1F2A980B4
:107DC00077EE677A384BBCEEC77A3848D3ED006A55
:107DD00017EE103A90ED007A0120C4ED7E6A37EE7E
:107DE000666AA4F8F431324BC4ED7C6A84ED7F7A84
:107DF00084ED7B6A84F8000293ED007AFFF7F9B90D
:107E00002C4BD3ED005AF5EEC05AF1EE10FA40F3C8
:107E10004F84294B93ED005AB5EEC05AF1EE10FA9B
:107E200040F3468426EE4A6A35EE477AF7EE004A7A
:107E3000C6EE256A87EE056A76EEA46A86FE646A57
:107E400086FE0B6A66EE266AC6FEE46AC6FE8B6A8A
:107E50002BE600BF68A10120B00001200CAB01207F
:107E6000603B0120C88801208C3001205C38012053
:107E7000803701200D720120613701204C740120F0
:107E80006C3001201C27012064A101205899012099
:107E9000D02B0120A4960120A6960120A8960120AF
:107EA0000075012002750120EC7401209C36012030
:107EB00008750120B02B0120B82B012078A90120E2
:107EC00050990120864AB0EEE77AD2ED006AB4EE0E
:107ED000E67AF1EE10FA7FF71DA9824AB0EECC7A6D
:107EE000D2ED006AB4EEE67AF1EE10FA7FF712A94D
:107EF00098ED007A7C4AB0EEC77AD2ED006AB4EE13
:107F0000E67AF1EE10FA7FF505A90122069984F8C8
:107F1000D021C4F8D411FFF701B9744B744EB3F9F2
:107F20000620738B9A423FF71BAE724B1B78012BD6
:107F300001F0BD87192B01F0BA87082B3FF410AE72
:107F40000E2B3FF40DAE00236B49C4F80C318B604F
:107F500006E66A4B4FF47A71694805931B68DFF8AF
:107F6000A881684E90F801A03678B8F90600B1FBF8
:107F7000F3F3C3EB431903EB89034FEAC3091FFA79
:107F800089F94F4502F0C880D5F88C10B5F940E06A
:107F90002B6F4A1C07EE90EA7344012AF8EEE77A49
:107FA000C5F88C202B6702F0C28095ED1F5A07EEB2
:107FB000102AD5ED216A012F77EEC55AB8EEC76AAF
:107FC00085EE867A37EE057A77EEC77A85ED207AE8
:107FD00085ED1F7AE7EEA56AF0EE667AC5ED226AB6
:107FE000C5ED216A02F0C084D5F8A010B5F942E0D1
:107FF0006B6F4A1C07EE90EA7344012AB8EEE77AE9
:10800000C5F8A0206B6702F0AB8095ED245A07EE0F
:10801000902AD5ED266A012F77EE455AB8EEE76A29
:10802000C5EE867A77EE857A37EE677AC5ED257AE2
:10803000C5ED247AF0EE667AE7EE257AC5ED277A6B
:10804000C5ED267A02F0B884D5F8B410B5F944E04D
:10805000AB6F4A1C07EE90EA7344012AB8EEE77A48
:10806000C5F8B420AB6702F0948095ED295A07EE6D
:10807000902AD5ED2B6A012F77EE455AB8EEE76AC4
:10808000C5EE867A77EE857A37EE677AC5ED2A7A7D
:10809000C5ED297AF0EE667AE5EE877AC5ED2C7AA1
:1080A000C5ED2B7A02F05484A8F80600B5F8B83074
:1080B000144A013B1678A5F8B83000230599072E1D
:1080C0004B608B60CB607EF46FAE07F0A1FD039B2D
:1080D000DFF83480C01AA8F80000FEF765BE00BFC4
:1080E000E42B0120E02B0120E82B0120507001201F
:1080F0000CAB0120903001205C38012068A90120E0
:1081000054A9012080370120843701202B78002BCF
:108110003FF4DBADD4ED5F3AF3EE046A94ED5E4AD2
:10812000D4ED7C7AF4EEC43A8D4A77EEA64A94ED0B
:108130007B7A92ED005AF1EE10FAD4ED5C5A94ED90
:108140005B6ADFF83CE2874F00F1C8879EED026A68
:10815000B0EE674A26EE656AA6EE074AB4EEE44A38
:1081600034EE666AF1EE10FA48BFB0EE456A012BB4
:1081700087ED006A3FF4A9AD9EED066AB0EE674A4E
:1081800026EE656AA6EE074AF4EEC44A34EE666A45
:10819000F1EE10FAC8BFB0EE456A022B87ED016A16
:1081A0003FF493AD9EED0A6AB0EE674A26EE656A2B
:1081B000A6EE074AB4EEE44A34EE666AF1EE10FA2F
:1081C00048BFB0EE456A032B87ED026A3FF47DADF0
:1081D0009EED0E6AB0EE674A26EE656AA6EE074A85
:1081E000F4EEC44A34EE666AF1EE10FAC8BFB0EE9F
:1081F000456A042B87ED036A3FF467AD9EED126A72
:10820000B0EE674A26EE656AA6EE074AF4EEC44A67
:1082100034EE666AF1EE10FA88BFB0EE456A052BBF
:1082200087ED046A3FF451AD9EED166AB0EE674AE1
:1082300026EE656AA6EE074AB4EEE44A74EE666A74
:10824000F1EE10FA48BFF0EE456A062BC7ED056A5D
:108250003FF43BADDEED1A6AB0EE674AB3EE046A56
:1082600066EEE56AA6EE874AF4EEC44A74EE466A04
:10827000F1EE10FAC8BFF0EE456A072BC7ED066AAB
:108280003FF423ADDEED1E6A66EEE55AE5EE877A31
:10829000F4EEE74A77EEC67AF1EE10FAC8BFF0EED8
:1082A000457AC7ED077A10E5059A2F4BD2ED017A92
:1082B00093ED007AF0EEE77AF4EEC77AF1EE10FA79
:1082C0007EF55DAED2ED027AF0EEE77AB4EEE77AB3
:1082D000F1EE10FA7EF753AED2ED037AF0EEE77AC4
:1082E000B4EEE77AF1EE10FA7EF749AE1F4B1B6849
:1082F00098077FF51AAD1E491E4BB3F90C20B1F952
:1083000000E01D48AEEB020E00688EEAEE72A2EBB2
:10831000EE728242BEF633AEB3F90E30B1F90220EE
:10832000D21A82EAE273A3EBE27398427EF727AE99
:10833000FBE498ED007A114BB0EEC77AD3ED006AFA
:10834000B4EEE67AF1EE10FA7EF7FAAEFEF7F5BE7D
:10835000B0EE666AFEF777BF09F0F8FCBAE400BF3A
:10836000487401206C300120DC2B0120983A012058
:108370007C3A0120C4360120D82B0120E82B0120B3
:108380006C7401209146A4F84821002B00F0508124
:108390004FF0020ED949DA4BB0EE007ADFEDD96A20
:1083A0001A68D94B1878137807EE903A9378F8EE5C
:1083B000E77A67EEA67AF4EEC77AF1EE10FA40F3A8
:1083C000228337EEC77ADFEDD16AB0EE676AA7EE97
:1083D000266AF0EE466A9FEDCE6A91ED007A27EEAE
:1083E000067AB0EEC76A84ED5B7A84ED5E6A9BB173
:1083F00005EE903A9FEDC34A67EE074AB8EEE55A9C
:10840000F7EE005A64EE864A25EE045A75EEC55A18
:10841000E4EE855A27EE257ADFEDBE5A92F805C0C4
:1084200066EEA56A26EE877ABCF1000F19D09FEDA3
:10843000B55A06EE90CADFEDB85AF8EEE66A26EEB7
:10844000056A26EE266AB4EEE56AF1EE10FA00F34C
:108450000886F7EE005A35EEC66AC5EE866A27EE44
:10846000267A0C2800F0B3859FEDAC8ADFEDAC6A6C
:1084700087FE488A88FE268A84ED418ABEF1000F75
:1084800000F0CB80B0EE007AF4EEC77AF1EE10FA8D
:1084900005DD37EEC77ADFED9D6AE7EE267A91EDCE
:1084A000017ADFED9B6A27EE267AB0EEC76A84ED8B
:1084B0005C7A84ED5F6A9BB106EE903ADFED914AFB
:1084C00027EE075AF8EEE66AF7EE005A25EE065A4E
:1084D00066EEA46A75EEE65AE5EE265A27EE257A90
:1084E000DFED8C6A937967EEA67A67EE877AABB197
:1084F00007EE103ADFED835AF8EEC76A9FED867AF1
:1085000066EE866A66EEA56AF4EEC76AF1EE10FAC8
:1085100040F3AB859FED837A67EE877A0C2800F0F5
:108520003E85DFED7E6ABEF1010F9FED7D7AC7FECD
:10853000E67AC7FE877AC4ED427A6EDD5378B0EEF4
:10854000007ADFED706A07EE903A537AF8EEE77A38
:1085500067EEA67AF4EEC77AF1EE10FA05DD37EE93
:10856000C77ADFED6A6AE7EE267A91ED027ADFEDEF
:10857000686A27EE267AF0EEC75A84ED5D7AC4ED7C
:10858000605A9BB106EE903ADFED5E4A27EE075A3D
:10859000B8EEE66AF7EE006A25EE255A26EE246A62
:1085A00076EEC66AE6EE056A27EE267ADFED596AB0
:1085B000D37967EEA67A67EE877A0BB307EE103AA7
:1085C0009FED506AF8EEC76A9FED537A66EEA56A92
:1085D00066EE866AF4EEC76AF1EE10FA0CDCF5EE90
:1085E000C06AF1EE10FA01F17682B7EE006A76EE1B
:1085F000666A86EE267A01E09FED4A7A67EE877A10
:108600000C2800F0C284DFED456A9FED457AC7FE75
:10861000E67AC7FE877AC4ED437A092800F0988489
:1086200096F82160002E40F04284002384F818312F
:108630003D4B1B689A0609D53C4B1B8803F0300361
:1086400023B13B4B1B78DB0701F1AE871BF026FD06
:10865000002840F08B81374B1B7823B9364B9B7831
:10866000002B41F04D82284B1B78072B00F0C7846C
:108670000022072B84F800217EF4BFAA07F0C8FA75
:108680000390FEF7BCBA2D4A2D4B12682D4CDFF833
:10869000C080D2691B8894F80001A8F80020A8F8CF
:1086A000023000287FF44DAA0390274DFEF7A7BAA9
:1086B000DFED266AFFF7F9B94F023EF56FAFFEF71F
:1086C00071BF07F0A5FA099BDFF88480C01A0E4B32
:1086D0001B78A8F80200012B00F03583072B7EF4ED
:1086E00056AD07F095FA0646FEF752BD07F090FA30
:1086F000174B801BD880FFF709BB00BF5C380120F7
:10870000007301200AD7233C80370120D7A368419A
:108710006F12033B00004843A4707D3F00C0F94442
:1087200000C0F9C40000C842983A0120603B012013
:108730009C3A01204F88012068B60120843F012027
:10874000DC2D01206C21012068A101200000000027
:1087500084370120002841F0B183DFF8CCE29DEDA1
:108760000A5ADEED007AA94F65EEA77AE5EE267A81
:10877000B0EE475AA7EE865AFDEEC57A17EE90CABC
:1087800017EE900A9C45A8BF18466145C8BF084629
:10879000012A07EE900AF8EEE77AC7ED007A3FF477
:1087A0008FAADEED047A9DED0B5A65EEA77AE5EE11
:1087B000267AB0EE475AA7EE865AFDEEC57A17EE36
:1087C00090CA17EE900A9C45A8BF18466145C8BFDD
:1087D0000846022A07EE900AF8EEE77AC7ED017A1A
:1087E0003FF46EAADEED087A9DED0C5A65EEA77A8D
:1087F000E5EE267AB0EE475AA7EE865AFDEEC57A28
:1088000017EE90CA17EE900A9C45A8BF184661451E
:10881000C8BF0846032A07EE900AF8EEE77AC7EDCC
:10882000027A3FF44DAADEED0C7A9DED0D5A65EE0D
:10883000A77AE5EE267AB0EE475AA7EE865AFDEE05
:10884000C57A17EE90CA17EE900A9C45A8BF184645
:108850006145C8BF0846042A07EE900AF8EEE77A99
:10886000C7ED037A3FF42CAADEED107A9DED0E5A87
:1088700065EEA77AE5EE267AB0EE475AA7EE865A5D
:10888000FDEEC57A17EE90CA17EE900A9C45A8BF78
:1088900018466145C8BF0846052A07EE900AF8EE5B
:1088A000E77AC7ED047A3FF40BAADEED147A9DED6A
:1088B0000F5A65EEA77AE5EE267AB0EE475AA7EE94
:1088C000865AFDEEC57A17EE90CA17EE900A9C45BF
:1088D000A8BF18466145C8BF0846062A07EE900A99
:1088E000F8EEE77AC7ED057A3FF4EAA9DEED187AEB
:1088F0009DED105A65EEA77AE5EE267AB0EE475A5E
:10890000A7EE865AFDEEC57A17EE90CA17EE900ACA
:108910009C45A8BF18466145C8BF0846072A07EE10
:10892000900AF8EEE77AC7ED067A3FF4C9A9DEEDC2
:108930001C7A9DED115A65EEA75AE6EE855AA6EE11
:10894000257AFDEEC77A17EE900A8342A8BF034648
:108950008142C8BF0B4607EE903AF8EEE77AC7EDC2
:10896000077A002A7FF4ACA9FFF7AFB9284E1BF0B5
:108970003BFA7378022B01F04181032B7FF46BAE3D
:1089800041F2B813F35C002B42F0A78141F2A4033B
:10899000F35C002B42F09C8141F2E803F35C002B76
:1089A00042F0A08141F22C13F35C002B3FF453AE54
:1089B000184828F027FD4EE6174B5A79002A3EF456
:1089C0007AAC164A1278002A3EF475AC1B7807EE92
:1089D000902AB7EE005ADFED124A07EE103A114B1B
:1089E000F8EEE77AB8EE477A1B8867EE277A07EE4B
:1089F000103AB8EE477A87EE874A84FE644A84FECE
:108A0000054AFEF75ABCF0EE676AE4E46C300120D8
:108A1000745A0120A06B0120843A01205B380120A8
:108A2000713DAA3F243801206C740120002F00F012
:108A30000E84002841F0EC87DFF84CE3BAF1000F18
:108A400041F04486FDEEE77A9DED0A5AC64F17EED7
:108A5000901ADEED007A65EEA77AE5EE267AB0EEA2
:108A6000475AA7EE865AFDEEC57A17EE90CA17EE62
:108A7000900A9C45A8BF18466145C8BF0846012A10
:108A800007EE900AF8EEE77AC7ED007A3FF418A9EE
:108A9000DEED047A9DED0B5A65EEA77AE5EE267AB7
:108AA000B0EE475AA7EE865AFDEEC57A17EE90CA89
:108AB00017EE900A9C45A8BF18468C45B8BF0846DB
:108AC000022A07EE900AF8EEE77AC7ED017A3FF442
:108AD000F7A8DEED087A9DED0C5A65EEA77AE5EE73
:108AE000267AB0EE475AA7EE865AFDEEC57A17EE03
:108AF00090CA17EE900A9C45A8BF18468C45B8BF8F
:108B00000846032A07EE900AF8EEE77AC7ED027AE4
:108B10003FF4D6A8DEED0C7A9DED0D5A65EEA77AEE
:108B2000E5EE267AB0EE475AA7EE865AFDEEC57AF4
:108B300017EE90CA17EE900A9C45A8BF18468C45C0
:108B4000B8BF0846042A07EE900AF8EEE77AC7EDA8
:108B5000037A3FF4B5A8DEED107A9DED0E5A65EE6E
:108B6000A77AE5EE267AB0EE475AA7EE865AFDEED2
:108B7000C57A17EE90CA17EE900A9C45A8BF184612
:108B80008C45B8BF0846052A07EE900AF8EEE77A4A
:108B9000C7ED047A3FF494A8DEED147A9DED0F5AE8
:108BA00065EEA77AE5EE267AB0EE475AA7EE865A2A
:108BB000FDEEC57A17EE90CA17EE900A9C45A8BF45
:108BC00018468C45B8BF0846062A07EE900AF8EE0C
:108BD000E77AC7ED057A3FF473A8DEED187A9DEDCC
:108BE000105A65EEA77AE5EE267AB0EE475AA7EE60
:108BF000865AFDEEC57A17EE90CA17EE900A9C458C
:108C0000A8BF18468C45B8BF0846072A07EE900A49
:108C1000F8EEE77AC7ED067A3FF452A8DEED1C7A4B
:108C20009DED115A65EEA75AE6EE855AA6EE257A15
:108C3000FDEEC77A17EE900A8342A8BF0346814231
:108C4000D8BF194607EE901AF8EEE77AC7ED077A13
:108C5000002A7FF435A8FFF738B8444BD3ED005A0B
:108C6000FEF711BF424A44F620604249D2F8EC2098
:108C700009688242A8BF0246B2F57A7FB8BF4FF4B6
:108C80007A7211F0100FDBF8001092B2A4F81A21DA
:108C900001F03682C90400F1D3863749D1F800E0EB
:108CA000BEF93200DFF8E4804FF0640C3349A8FBD2
:108CB0000282D4F81C81D1ED037A910908F10102F6
:108CC000BDEEE77A04EB4808C4F81C219CFBF1F1E7
:108CD000142917EE109AA8BF1421A8F820918A42EF
:108CE00003DB00210A46C4F81C1104EB4202B2F96E
:108CF000202107EE102AB8EEC77A77EEC77AFDEE8C
:108D0000E77ACDED037ABDF90C1081EAE172A2EBAE
:108D1000E172824202F34F814FF07E5218490A609D
:108D2000FEF72BBFAB68002B3EF414AF05F15401E6
:108D300028469847FEF70EBF06F06AFF0990FEF737
:108D400047B8DFF84C8006F063FFD4F8E4310D4AF1
:108D50000646C31AC4F8E4011268A8F804309B1A46
:108D6000A8F80630FEF714BA6C300120B02B0120B1
:108D7000B800012064360120608801205C380120A1
:108D8000780001208C3001206C740120D34D6210DA
:108D90008437012007EE103ABB4BF7EE006A002241
:108DA0001B78B8EEC77ADFF83083132BC4F8A02104
:108DB00086EE879AB8F90400B4F8A47195ED090A13
:108DC00001F07C83B14BB24A67EE897AD3ED006A39
:108DD00029EE088A93ED053A69EE288A93ED097A1F
:108DE00093ED0E5AA6EEA73A93ED176A02EB8701B0
:108DF000D3ED126AA7EE085AD3ED063A0E4693ED6C
:108E0000017AA6EEA86AD3ED0A5AD3ED0F4AE7EE2F
:108E1000273AD3ED186A93ED137AE5EE884A93ED7D
:108E2000044AE7EE286AD3ED0D5A93ED167A24EE44
:108E3000434A93ED032A65EEC55AD3ED022A27EE85
:108E4000467AD3ED0C1AE2EE433AA2EEA74A93ED2E
:108E50000B2AD3ED152AE1EEC54AD3ED147AE2EEE2
:108E6000085AE2EEC66A81ED003AA7EEA87A002120
:108E7000C3ED053A83ED064AC3ED0E4A86ED205A4E
:108E8000C3ED0F5A86ED406AC3ED176A83ED187A79
:108E9000C4F89411C4F89811C4F89C117B1CA8F86C
:108EA000040003F01F03A4F8A431FDF705BF1E2141
:108EB000784808F012FA00283FF4B7AB764B1B88CD
:108EC00059063FF5B2AB94F88431B34242F01281B7
:108ED000724BD4ED627AD3ED016A94ED435A28EED9
:108EE000277ADFED6F5A67EEC57A9FED6E6AA5EEC1
:108EF000267AE8EE267A87FE657A87FE067A84ED82
:108F0000437AC7FEE57AC7FE867AC4ED417AFFF759
:108F10008CBBB4F8F401984240F29E85624B01206C
:108F2000624D93ED007AD5ED007A614B77EE676A7A
:108F3000C4ED7E7AC4ED7C7A84ED7F7AC4ED7B6AE1
:108F400084F80002DFED5B7A93ED007AFEF751B909
:108F5000FDEEC87ADFF88081A8F8049017EE903A09
:108F6000A8F80630FFF75CBB534B1B88002B40F082
:108F70009285524A524B1178186807F0A5F9D4F837
:108F8000D421069B9A1AFDF7CBBFBDEEE77ADFF836
:108F9000488117EE103AA8F80430FFF734BBBDEE55
:108FA000E77ADFED3F6ADFF83081BEF1010FC7FEDF
:108FB000E67A17EE103A9FED3B7AA8F80230C7FE2A
:108FC000877AC4ED427A3FF7B9AAFFF729BBFDEED5
:108FD000C76A9FED338ADFF8008187FE488A16EE64
:108FE00090CADFED306AA8F800C088FE268A84EDBA
:108FF000418ABEF1000F7FF445AAFFF711BB06F0CE
:1090000007FEDFF8D480C01B1F4BA8F804001B78B4
:10901000FFF72EBB2B4B2C48D3ED006A2B4B90ED6A
:10902000006A1B78C4ED7E6A84ED7F6A002B40F0F5
:109030000F8576EEC65AF0EE466ABCEEC76AFF2090
:10904000234B77EEC77AC4ED7B5A16EE105AC4ED67
:109050007C6A84F80002A4F8F45193ED007AFEF7DC
:10906000C8B8DFED1C6AFFF7FAB9F5EEC06AF1EE99
:1090700010FA00F12C85B7EE006A76EE666A86EE8D
:10908000267AFFF749BA00BF803701209C330120C0
:109090001831012064360120603B01207800012056
:1090A00000C0F94400C0F9C49C360120EC740120D2
:1090B0000875012000000000A4960120A69601205A
:1090C000A89601200C350120F07401205C99012044
:1090D000047501200000C84284370120DEED015AEA
:1090E000B0EE674A65EEC65AA5EE874AF4EEC44A6A
:1090F00074EE665AF1EE10FAC8BFF0EE455A012B35
:10910000C7ED005A3EF4E1ADDEED055AB0EE674A18
:1091100065EEC65AA5EE874AF4EEC44A74EE665A66
:10912000F1EE10FAC8BFF0EE455A022BC7ED015A16
:109130003EF4CBADDEED095AB0EE674A65EEC65A95
:10914000A5EE874AF4EEC44A74EE665AF1EE10FAC0
:10915000C8BFF0EE455A032BC7ED025A3EF4B5AD39
:10916000DEED0D5AB0EE674A65EEC65AA5EE874AA7
:10917000F4EEC44A74EE665AF1EE10FAC8BFF0EE8F
:10918000455A042BC7ED035A3EF49FADDEED115A4C
:10919000B0EE674A65EEC65AA5EE874AF4EEC44AB9
:1091A00074EE665AF1EE10FAC8BFF0EE455A052B80
:1091B000C7ED045A3EF489ADDEED155AB0EE674AAC
:1091C00065EEC65AA5EE874AF4EEC44A74EE666AA6
:1091D000F1EE10FAC8BFF0EE456A062BC7ED056A3E
:1091E0003EF473ADDEED196AB0EE674AF3EE045A51
:1091F00066EEC66AA6EE874AF4EEC44A74EE656A65
:10920000F1EE10FAC8BFF0EE456A072BC7ED066A0B
:109210003EF45BADDEED1D6A26EEC66AE6EE077A29
:10922000F4EEE47A77EEE57AF1EE10FAB8BFF0EEFC
:10923000457AC7ED077AFEF748BD96F82020C2EBC5
:10924000421102EB8101C90089B2FEF7A2BCDFF82E
:1092500024E3BAF1000F40F0E787FDEEE77A9DEDD9
:109260000A5AC14F17EE901ADEED007A65EEA77A22
:10927000E5EE267AB0EE475AA7EE865AFDEEC57A9D
:1092800017EE908A17EE90CA9845A8BF9C464145B4
:10929000C8BF8C46012A07EE90CAF8EEE77AC7ED00
:1092A000007A3EF4BBAADEED047A9DED0B5A65EE22
:1092B000A77AE5EE267AB0EE475AA7EE865AFDEE7B
:1092C000C57A17EE908A17EE90CA9845A8BF9C46BB
:1092D0008845B8BF8C46022A07EE90CAF8EEE77AB6
:1092E000C7ED017A3EF49AAADEED087A9DED0C5A9C
:1092F00065EEA77AE5EE267AB0EE475AA7EE865AD3
:10930000FDEEC57A17EE908A17EE90CA9845A8BF71
:109310009C468845B8BF8C46032A07EE90CAF8EEF3
:10932000E77AC7ED027A3EF479AADEED0C7A9DED7C
:109330000D5A65EEA77AE5EE267AB0EE475AA7EE0B
:10934000865AFDEEC57A17EE908A17EE90CA9845B8
:10935000A8BF9C468845B8BF8C46042A07EE90CA31
:10936000F8EEE77AC7ED037A3EF458AADEED107AFC
:109370009DED0E5A65EEA77AE5EE267AB0EE475AD5
:10938000A7EE865AFDEEC57A17EE908A17EE90CAC0
:109390009845A8BF9C468845B8BF8C46052A07EE6D
:1093A00090CAF8EEE77AC7ED047A3EF437AADEED0C
:1093B000147A9DED0F5A65EEA77AE5EE267AB0EEA7
:1093C000475AA7EE865AFDEEC57A17EE908A17EE39
:1093D00090CA9845A8BF9C468845B8BF8C46062AC7
:1093E00007EE90CAF8EEE77AC7ED057A3EF416AAC2
:1093F000DEED187A9DED105A65EEA77AE5EE267A35
:10940000B0EE475AA7EE865AFDEEC57A17EE908A5F
:1094100017EE90CA9845A8BF9C468845B8BF8C46B1
:10942000072A07EE90CAF8EEE77AC7ED067A3EF40F
:10943000F5A9DEED1C7A9DED115A65EEA75AE6EE10
:10944000855AA6EE257AFDEEC77A17EE90EA7345A7
:10945000A8BF73467145D8BF194607EE901AF8EEBB
:10946000E77AC7ED077A00287EF42FACFEF7D9B96A
:10947000DFF80491D4ED017AB0EE006AD4ED005A21
:10948000F6EE006A77EEA77AB9F80000D9F8142052
:109490000138B0EE664AB0EE677A1032D5EE867AC1
:1094A00004EBC003A5EE867A083B67EEA67A27EEAA
:1094B000267AC4ED217A84ED207A2C4CA64604F15C
:1094C000800193ED036A0138DEED036AA3F108031E
:1094D00093ED047A0EF1080E76EEC65ADEED007AB0
:1094E00012ED015A76EE266A77EE674A12ED026AAD
:1094F00077EE277A02F10802B0EE657A01F10801F1
:10950000E6EE247AA5EE247AE5EE267AA6EE667AD1
:1095100067EE847A27EE047AC1ED007A81ED017A54
:10952000CFD1142F7EF430AA06F072FB049BDFF833
:109530004C80C01AD4F8A861A8F80200FEF724BA3B
:10954000DFF834900948D9F80820B9F80C1029F050
:1095500051FF074B1F78142F01F06585D4F8A861DF
:109560000136C4F8A86185E76C3001206C21012028
:10957000803701206C7401200031012084370120E4
:10958000DFF8E493B9F80010D9F804E04FEA510C81
:1095900004EB81084FEA8C02C90804EB020600F0D4
:1095A000A0800131103206F11003E44806EB0117E8
:1095B00042440EF1100608F1100151ED047A103307
:1095C00010ED047A103613ED085A103052ED041ADB
:1095D00037EE271A12ED032A77EE670A51ED034A98
:1095E00075EE218A51ED023A71EEC51A12ED026A4A
:1095F000103112ED017A103251ED055A53ED072A60
:1096000053ED066A53ED057A32EE828A10ED074A71
:1096100036EE860A10ED063A72EE622A10ED055A11
:1096200034EE249A00ED081A74EE644A33EE231ADD
:1096300037EE874A00ED079A35EE252A00ED061A27
:1096400077EE677A33EE631A00ED052A76EE666AE6
:1096500003ED054A75EE655A43ED088A03ED078A66
:1096600003ED060A9F4216ED077A16ED086A64EECE
:10967000873A27EE603A26EE624A21EE865AA4EE39
:10968000863AF0EE634AA2EE875AE0EE864AB0EEE2
:10969000446A01ED073AA1EE876A41ED084A02EDFE
:1096A000075A02ED086A16ED057A16ED066A65EEB0
:1096B000873A27EE414A66EE674A26EE865AA5EEBD
:1096C000864AE1EE063AE6EE874AA7EE875A41ED72
:1096D000063A01ED054A42ED064A02ED055A7FF4CD
:1096E0006CAF1FFA8CF672469548314623F014FF92
:1096F0003146D9F80420404623F00EFF914B1B78E9
:10970000142B3FF411AFD4F8A861FEF73DB9D4F89B
:10971000ACC1B4F8A4A18C4BCAF120090AEB4C1ED1
:109720005FFA89F903EB8E0E5FEA990001F0668417
:1097300001300EF1100385490001804A0EEB00084C
:1097400013ED025A103311ED027A103253ED075A1D
:10975000103151ED077A25EE075A13ED056A13ED26
:10976000087A65EEA75A51ED056A984551ED087AD9
:1097700066EE266A02ED065A67EE277A42ED075A30
:1097800042ED056A42ED087ADAD110387049864414
:109790000A18204419F0030309D0BEEC017A013BFA
:1097A000F2EC017A67EE277AE0EC017AF5D1BAF1B2
:1097B000000F3FF4B6AE4FEA890E634B5FEA9A00A2
:1097C00001EB0E0803EBCC1CA64401F04D860130E2
:1097D0000CF1100308F110010EF110024FEA00190C
:1097E0000CEB090013ED025A103311ED027A10321E
:1097F00053ED075A103151ED077A25EE075A13ED54
:10980000056A13ED087A65EEA75A51ED056A98428C
:1098100051ED087A66EE266A02ED065A67EE277A5F
:1098200042ED075A42ED056A42ED087ADAD1A9F114
:109830001000844408EB000186441AF0030A3FF448
:1098400070AEBCEC017ABAF1010AF1EC017A67EE74
:10985000277AEEEC017AF4D163E6D4F8AC913D4A74
:109860004FEAC9083C4B9FED3D7A4244D3ED008A54
:10987000C8443B4B9288F8EE688A03EB8808A2F153
:10988000640308EE102A68EE878AC82BF8EE487A3F
:10989000B8EEC89AA8BFC82368EEA78A782BB8BFCD
:1098A0007823B0EE680A07EE903AB8EEE78A2BF01C
:1098B00049F8F0EE409AB0EE680A2AF0A5FF78EE7B
:1098C000097A79EE486A142F28EE098AB7EE006A01
:1098D00066EEA76AF8EE007A88EE267A60EE277ABE
:1098E00077EE076A89EEA67A77EE065A36EE477A61
:1098F000C6EE256A67EEA67AC8ED006A27EE267ADC
:10990000C8ED026AC8ED017A88ED047AC8ED037AE1
:1099100001F0C18309F10109124B0136094A83FBA9
:10992000093C1778ACEBE97CC4F8A8610CEB4C0C53
:10993000A9EB0C0CC4F8ACC1EBE600BF7C21012004
:109940006C2101208037012018310120A83201202C
:10995000983201201833012068A9012027D4D2367B
:10996000E8A801205655555500310120DFF898939D
:1099700099F800205FEA920E01F09A840EF1010836
:10998000CC484FEA481800F12003A0F1700100EB29
:10999000080C53ED077A203353ED0D6A103113EDA7
:1099A0000B7A27EEA76A53ED097A66EEA66A53EDA5
:1099B000105A27EE077A67EEA77A53ED0E4A13ED99
:1099C0000C5AA5EEA56A53ED0A5AE4EEA46AA5EE78
:1099D000057A9C45E5EEA57AF1EEC65AB1EEE66A47
:1099E000F1EEC76AB1EEE77A41ED085A01ED076A78
:1099F00041ED066A01ED057ACBD1A8F1200804EB10
:109A00000E13804412F0030E12D008F1080151ED3C
:109A1000017ABEF1010E11ED027A01F1080167EE43
:109A2000A77AE7EE077AB1EEE77AA3EC017AEED1F6
:109A3000142F01F0CC830136C4F8A861FDF712BFE2
:109A40009D49D1F800E0BEF832004008FFF72AB97E
:109A500076EE665AFFF7F1BA984B9948D3ED007A43
:109A6000984B90ED007A1B78C4ED7E7A84ED7F7A76
:109A7000002B01F09A8277EE676AFF20924BC4EDCB
:109A80007C7AC4ED7B6A84F80002DFED907A93ED76
:109A9000007AFDF7AEBB8E494B69002B3DF440AA1E
:109AA0008C484FF0010E8C4B008893FBF0F00B6854
:109AB000186081F811E0FDF733BA85494A69002A38
:109AC0003DF45DAA0A6813604B74FDF758BAB7EE0F
:109AD000007AFEF721BDB7EE007AFEF78FBDB4F82D
:109AE000489109F1FF390FFA89F9A4F84891FEF776
:109AF0009EB8B4F81A1101F57A7189B2FEF749B827
:109B000006980DF083FBFEF7AEBD744ADFED747A64
:109B100092ED080A0393B4EEE70AF1EE10FA40F270
:109B200013872AF059FFD4ED457A20EE270A2AF050
:109B3000BDFEB0F5617F039B01F3A08007EE900AA4
:109B400007EE103AF8EEE76ADFED667AB8EEC77A0C
:109B500066EEA76AFDEEE67A17EE903A2033402BC8
:109B600041F2B3839FED590A2AF0A0FE00B207EE3E
:109B7000900AB8EEE77A5C49D1ED037A77EE877AFE
:109B8000C1ED037AFDF7F4BF584B187800F00100DF
:109B900000287EF49AA8FDF744BE554BDFED557AB8
:109BA0001B68C4ED707A13F0805B40F07585480245
:109BB00001F17E80B6EE007AF4EEC75AF1EE10FAAB
:109BC000CCBF01230023002B41F072809B46FDF7A0
:109BD000E9BC06F01DF8484B04901F78D4F8A86142
:109BE000142F7DF472A8DFF82481A8F80060FDF737
:109BF0006CB806F00DF80746FDF7A4BFB3784FF038
:109C0000010B072B3EF627ADDFE813F082001A01A7
:109C10000E019B00A6003E0048000800032373705D
:109C2000FEF719BD33690622652BB27036D932783A
:109C3000653B032A15BF6FF0FF016FF07F014FF402
:109C4000807280220B4001339A42336126D2D8F8C9
:109C50000020D6F80C80023203EB0809914502D3AC
:109C600026F0A2FB3369254A0520C6F80480D16F8F
:109C7000C6F808904902C2F80080B07003FB01F3F7
:109C800042F81C3C42F8183CB26801201C4927F0FD
:109C900001F9012841F05B850623B37000211948C2
:109CA00026F098FC012841F05285B3780133DBB2ED
:109CB000B370A6E7EC210120608801200C3501205B
:109CC000F07401205C99012004750120000000005F
:109CD000AC960120C496012020A1070098720120B3
:109CE0008FC2753CD06D393A5C3801200D7201206D
:109CF000643601200000008080370120086C0120BC
:109D0000785A0120E46B0120FA30012084370120C9
:109D100000230DF1280909224946184619F042FE90
:109D200001287EF498AC0A9B93F8FE21552A01F095
:109D3000128341F2B41202210123B1547370FEF771
:109D40008ABC41F27013F35C002B3EF484ACE04813
:109D500027F058FBFEF77FBC3278337D032ADFF80B
:109D60008C83DFF88CA314BF4FF480794FF0800907
:109D7000002B44D0012BFBD1D64B4FF0FF3E706837
:109D800000211A68D8F80030520203F1020CBEFB21
:109D9000F2FE10EB0E024FF0020041F10003002131
:109DA0009942CD4908BF944538BF624619F036FF45
:109DB000032801F2CD8201A353F820F05786010851
:109DC000CD9D010857860108CD9D0108D6F808E011
:109DD00072683369AEEB0201994201D9F2603161D8
:109DE00003283FF41FAF0EF10103B3FBF9F209FBA7
:109DF00012320AB14B449B1A002273603275D8F8B4
:109E0000002051460020023219F008FF032801F219
:109E10009F8201A353F820F0578601087F9E010816
:109E200057860108259C0108AC49032030230522F0
:109E30000091B070AA49A64826F09AFFFEF70BBC25
:109E40000DF1280941F2FC1849460023092256F871
:109E5000080019F0A7FD01287EF4FDAB00230A9A43
:109E60003370B2F80B30B3F5007F01F0908341F20C
:109E7000B41203210123B1547370FEF7ECBB736875
:109E800086F814B00133B36076E777EEC77AB7EEA1
:109E9000007AC4ED707AF4EEC77AF1EE10FA41F36D
:109EA000A58085EE277A8DED0A7AFDF771BB8D4A84
:109EB000927B002A7DF454AEFEF73FB80398DFF89A
:109EC00034E2002800F05C87DEED007A9DED0A5A4E
:109ED00065EEA77A844FE5EE267AB0EE475AA7EEF4
:109EE000865AFDEEC57A17EE90CA17EE900A9C4589
:109EF000A8BF18466145C8BF0846012A07EE900A68
:109F0000F8EEE77AC7ED007A3DF4DFAEDEED047AD5
:109F10009DED0B5A65EEA77AE5EE267AB0EE475A2C
:109F2000A7EE865AFDEEC57A17EE90CA17EE900A94
:109F30009C45A8BF18466145C8BF0846022A07EEDF
:109F4000900AF8EEE77AC7ED017A3DF4BEAEDEED99
:109F5000087A9DED0C5A65EEA77AE5EE267AB0EE0A
:109F6000475AA7EE865AFDEEC57A17EE90CA17EE4D
:109F7000900A9C45A8BF18466145C8BF0846032AF9
:109F800007EE900AF8EEE77AC7ED027A3DF49DAE4F
:109F9000DEED0C7A9DED0D5A65EEA77AE5EE267A98
:109FA000B0EE475AA7EE865AFDEEC57A17EE90CA74
:109FB00017EE900A9C45A8BF18466145C8BF0846E1
:109FC000042A07EE900AF8EEE77AC7ED037A3DF42B
:109FD0007CAEDEED107A9DED0E5A65EEA77AE5EEC9
:109FE000267AB0EE475AA7EE865AFDEEC57A17EEEE
:109FF00090CA17EE900A9C45A8BF18466145C8BF95
:10A000000846052A07EE900AF8EEE77AC7ED047ACB
:10A010003DF45BAEDEED147A9DED0F5A65EEA77A46
:10A02000E5EE267AB0EE475AA7EE865AFDEEC57ADF
:10A0300017EE90CA17EE900A9C45A8BF18466145D6
:10A04000C8BF0846062A07EE900AF8EEE77AC7ED81
:10A05000057A3DF43AAEDEED187A9DED105A65EEC4
:10A06000A77AE5EE267AB0EE475AA7EE865AFDEEBD
:10A07000C57A17EE90CA17EE900A9C45A8BF1846FD
:10A080006145C8BF0846072A07EE900AF8EEE77A4E
:10A09000C7ED067A3DF419AEDEED1C7A9DED115A3E
:10A0A00065EEA75AE6EE855AA6EE257AFDEEC77A4A
:10A0B00017EE902A9342A8BF13468A42A8BF1946BA
:10A0C00007EE901AF8EEE77AC7ED077AFDF7FDBDC7
:10A0D000E46B0120846C01207C5A01201D030408DC
:10A0E00004A10408A89701206C3001207C6C012099
:10A0F000785A01206C740120000002430000000027
:10A10000C8003EF5C7ADFDF738BD5FED057AFDF738
:10A11000F2BB8223FDF724BCB5F940100123AA62EB
:10A1200007EE901A2967C5F88C30F8EEE77A00231D
:10A13000012FC5ED207AC5ED1F7AC5F8843001F0F6
:10A14000BC804F457DF450AFB5F942100022012389
:10A1500007EE901AEA626967B8EEE77AC5F8A030B0
:10A160000023012F85ED257A85ED247AC5F89830F6
:10A1700001F0A7804F457DF467AFB5F94430002268
:10A1800007EE903AAB6701232A63B8EEE77AC5F889
:10A19000B4300023012F85ED2A7A85ED297AC5F8A0
:10A1A000AC307DF481AF1FED2B8A032E36D0BAF18F
:10A1B000000F09D007EE90AAF8EEE77AF4EEC87A1D
:10A1C000F1EE10FA01F1DD81AB6F0021B64A03EB2D
:10A1D0005903A8F80600126894F8B00193FBF9F34C
:10A1E0002B6391621163D16230B1B04B1B8823F4B1
:10A1F0000063002B7DF45AAFAD4B1B6813F40033A2
:10A2000041F04E801946AB48C25C0C33012A00F085
:10A210006E8501311529F7D1FDF748BFB0EE480A28
:10A220002AF044FB00B2C2E7FDEEE74A9DED0A4A80
:10A23000A14F14EE901ADEED004A65EEA44AE4EE5A
:10A24000264AB0EE474AA4EE864AB4EEC45AF0EE6F
:10A25000444AF1EE10FA88BFF0EE674AFDEEE44A98
:10A2600014EE90CA14EE908A9C45A8BF98466145AA
:10A27000C8BF8846012A04EE908AF8EEE44AC7ED8A
:10A28000004A3DF4CBAADEED044A9DED0B4A65EE93
:10A29000A44AE4EE264AB0EE474AA4EE864AB4EE5B
:10A2A000C45AF0EE444AF1EE10FA88BFF0EE674A65
:10A2B000FDEEE44A14EE90CA14EE908A9C45A8BFC5
:10A2C00098468C45B8BF8846022A04EE908AF8EE7C
:10A2D000E44AC7ED014A3DF4A1AADEED084A9DED2E
:10A2E0000C4A65EEA44AE4EE264AB0EE474AA4EED4
:10A2F000864AB4EEC45AF0EE444AF1EE10FA88BF32
:10A30000F0EE674AFDEEE44A14EE90CA14EE908A2D
:10A310009C45A8BF98468C45B8BF8846032A04EEE2
:10A32000908AF8EEE44AC7ED024A3DF477AADEEDE2
:10A330000C4A9DED0D4A65EEA44AE4EE264AB0EEC5
:10A34000474AA4EE864AB4EEC45AF0EE444AF1EE0F
:10A3500010FA88BFF0EE674AFDEEE44A14EE90CAA8
:10A3600014EE908A9C45A8BF98468C45B8BF884695
:10A37000042A04EE908AF8EEE44AC7ED034A3DF45D
:10A380004DAADEED104A9DED0E4A65EEA44AE4EEBC
:10A39000264AB0EE474AA4EE864AB4EEC45AF0EE1E
:10A3A000444AF1EE10FA88BFF0EE674AFDEEE44A47
:10A3B00014EE90CA14EE908A9C45A8BF98468C452E
:10A3C000B8BF8846052A04EE908AF8EEE44AC7ED45
:10A3D000044A3DF423AADEED144A9DED0F4A65EED2
:10A3E000A44AE4EE264AB0EE474AA4EE864AB4EE0A
:10A3F000C45AF0EE444AF1EE10FA88BFF0EE674A14
:10A40000FDEEE44A14EE90CA14EE908A9C45A8BF73
:10A4100098468C45B8BF8846062A04EE908AF8EE26
:10A42000E44AC7ED054A3DF4F9A9DEED184A9DED71
:10A43000104A65EEA44AE4EE264AB0EE474AA4EE7E
:10A44000864AB4EEC45AF0EE444AF1EE10FA88BFE0
:10A45000F0EE674AFDEEE44A14EE90CA14EE908ADC
:10A460009C45A8BF98468C45B8BF8846072A04EE8D
:10A47000908AF8EEE44AC7ED064A3DF4CFA9DEED36
:10A480001C4A9DED114A65EEA45AE6EE845AA6EEEA
:10A49000257AB4EEC75AF1EE10FAD8BFF0EE477A3B
:10A4A000FDEEE77AFEF7D1BF843F01206EB10120B7
:10A4B00010730120349404086C3001207A4E67EE4A
:10A4C000897ADFF8049229EE088AD6ED006A69EEEF
:10A4D000288A96ED057A09EB8703D6ED015AA6EE98
:10A4E000A77A96ED066AD6ED046AA5EEA76A96ED00
:10A4F000035AD6ED025A66EEC76A83ED007A20EE63
:10A50000070AA5EE476AE5EEA76A86ED056AC6ED7D
:10A51000066A2AF0CBF996ED097A96ED0E5A09EB08
:10A520008703D6ED127A00B2D6ED175AA7EE085A75
:10A53000D6ED0A6A9946E8EEA75A96ED0F6AD6ED6F
:10A54000137A96ED187AA6EE886AD6ED0D6AA8EE13
:10A55000A77AD6ED167A66EEC56A96ED0C3A67EEE6
:10A56000E57AD6ED0B3A96ED154AD6ED144AA3EEF0
:10A57000456AE3EE886A83ED205AA5EEC47A00238B
:10A58000E8EEA47AC9ED405AC4F89431C4F8983181
:10A5900086ED0E6AC6ED0F6A86ED177AC6ED187A5B
:10A5A000C4F89C31FEF77ABC404B414AB3F9043001
:10A5B000DFED407A82FB0312DB17C3EBA2031BB271
:10A5C00008EE103AB8EEC88A28EE278AB0EE480A9C
:10A5D00006F0B0FDF0EE408AB0EE480A06F032FD1B
:10A5E000354BD978002900F09A83344E44F25060FC
:10A5F000B4F98E31B6F90220D21A824240F31F8597
:10A60000A2F50C42A03A4842904200F3FC848A42F0
:10A61000A8BF0A461344B6F90020B4F98C6144F28D
:10A62000506E1BB2921BA4F88E31724540F3EE843B
:10A63000A2F50C42A03A904203DC9142A8BF114619
:10A640000846304407EE903A9FED1D6A03B2B8EE1B
:10A65000E77A07EE903AA4F88C31F8EEE77A67EEE5
:10A66000E86A60EE277AE0EE076AE8EE877A26EE7F
:10A67000867A67EE867ABDEEC77AFDEEE77A17EE48
:10A68000102A17EE903AA4F89021A4F89231FDF721
:10A69000DDBF0C49FDF706BBB7EE007A77EE677AAF
:10A6A000C5FEE75AFCF77CBF9C3301207C3A0120B1
:10A6B0006766666635FA8E3C9C3B0120F83B0120BC
:10A6C000CDCCCC3D5C38012018310120FDEEE74AAD
:10A6D0009DED0A4ACC4F14EE901ADEED004A65EE6D
:10A6E000A44AE4EE264AB0EE474AA4EE864AB4EE07
:10A6F000C45AF0EE444AF1EE10FA88BFF0EE674A11
:10A70000FDEEE44A14EE900A14EE90CA9842A8BFF7
:10A710009C468142C8BF8C46012A04EE90CAF8EEDE
:10A72000E44AC7ED004A3DF4CBAADEED044A9DEDB4
:10A730000B4A65EEA44AE4EE264AB0EE474AA4EE80
:10A74000864AB4EEC45AF0EE444AF1EE10FA88BFDD
:10A75000F0EE674AFDEEE44A14EE900A14EE90CA59
:10A760009842A8BF9C468842B8BF8C46022A04EE95
:10A7700090CAF8EEE44AC7ED014A3DF4A1AADEED25
:10A78000084A9DED0C4A65EEA44AE4EE264AB0EE76
:10A79000474AA4EE864AB4EEC45AF0EE444AF1EEBB
:10A7A00010FA88BFF0EE674AFDEEE44A14EE900A14
:10A7B00014EE90CA9842A8BF9C468842B8BF8C4607
:10A7C000032A04EE90CAF8EEE44AC7ED024A3DF4CB
:10A7D00077AADEED0C4A9DED0D4A65EEA44AE4EE43
:10A7E000264AB0EE474AA4EE864AB4EEC45AF0EECA
:10A7F000444AF1EE10FA88BFF0EE674AFDEEE44AF3
:10A8000014EE900A14EE90CA9842A8BF9C46884263
:10A81000B8BF8C46042A04EE90CAF8EEE44AC7EDAD
:10A82000034A3DF44DAADEED104A9DED0E4A65EE59
:10A83000A44AE4EE264AB0EE474AA4EE864AB4EEB5
:10A84000C45AF0EE444AF1EE10FA88BFF0EE674ABF
:10A85000FDEEE44A14EE900A14EE90CA9842A8BFA6
:10A860009C468842B8BF8C46052A04EE90CAF8EE92
:10A87000E44AC7ED044A3DF423AADEED144A9DEDF7
:10A880000F4A65EEA44AE4EE264AB0EE474AA4EE2B
:10A89000864AB4EEC45AF0EE444AF1EE10FA88BF8C
:10A8A000F0EE674AFDEEE44A14EE900A14EE90CA08
:10A8B0009842A8BF9C468842B8BF8C46062A04EE40
:10A8C00090CAF8EEE44AC7ED054A3DF4F9A9DEED79
:10A8D000184A9DED104A65EEA44AE4EE264AB0EE11
:10A8E000474AA4EE864AB4EEC45AF0EE444AF1EE6A
:10A8F00010FA88BFF0EE674AFDEEE44A14EE900AC3
:10A9000014EE90CA9842A8BF9C468842B8BF8C46B5
:10A91000072A04EE90CAF8EEE44AC7ED064A3DF471
:10A92000CFA9DEED1C4A9DED114A65EEA45AE6EE74
:10A93000845AA6EE257AB4EEC75AF1EE10FAC8BFD3
:10A94000B0EE677AFEF774B99FED307AFFF713B96E
:10A95000012A7FF728AC07EE101AB8EEC77AC7EEC7
:10A96000876AB1EEE68A20E4012A40F3A68407EE66
:10A97000101AB8EEC77AC7EE876AB1EEE68A032EE0
:10A9800014D0BAF1000F09D007EE90AAF8EEE77ADA
:10A99000F4EEC87AF1EE10FA00F1F3852B6F03EBB9
:10A9A000590393FBF9F3AB62FFF7CBBBB0EE480A58
:10A9B00029F07CFF00B2E4E7012A40F3828407EE2D
:10A9C000101AB8EEC77AC7EE876AB1EEE68A032E90
:10A9D00014D0BAF1000F09D007EE90AAF8EEE77A8A
:10A9E000F4EEC87AF1EE10FA00F1CB856B6F03EB51
:10A9F000590393FBF9F3EB62FFF7BCBBB0EE480AD7
:10AA000029F054FF00B2E4E76C30012000000000A0
:10AA10000399002900F0FD83DFF860E39DED0A4A09
:10AA2000DEED004A65EEA44AE4EE264AB0EE474A5F
:10AA3000A4EE864AF0EE444ABAF1000F06D0B4EE16
:10AA4000445AF1EE10FAC8BFF0EE674AFDEEE77A1D
:10AA500017EE901AFDEEE47A04EE901A17EE900AC3
:10AA6000814200F371859842A8BF184607EE900A0C
:10AA7000F8EEE77AB74F012AC7ED007A3DF425A931
:10AA8000DEED047A9DED0B4A65EEA77AE4EE267AB8
:10AA9000B0EE474AA7EE864AF0EE447ABAF1000FCC
:10AAA00000F0D784B4EEC45AF1EE10FA40F3D1842A
:10AAB00008469842A8BF184607EE900AF8EEE77AD3
:10AAC000022AC7ED017A3DF400A9DEED087A9DED7A
:10AAD0000C4A65EEA77AE4EE267AB0EE474AA7EE76
:10AAE000864AF0EE447ABAF1000F00F0A784B4EE83
:10AAF000C45AF1EE10FA40F3A18408469842A8BF68
:10AB0000184607EE900AF8EEE77A032AC7ED027AB4
:10AB10003DF4DBA8DEED0C7A9DED0D4A65EEA77ADB
:10AB2000E4EE267AB0EE474AA7EE864AF0EE447A83
:10AB3000BAF1000F00F07784B4EEC45AF1EE10FAC7
:10AB400040F3718408469842A8BF184607EE900A61
:10AB5000F8EEE77A042AC7ED037A3DF4B6A8DEEDF5
:10AB6000107A9DED0E4A65EEA77AE4EE267AB0EEF5
:10AB7000474AA7EE864AF0EE447ABAF1000F00F099
:10AB80004784B4EEC45AF1EE10FA40F3418408460B
:10AB90009842A8BF184607EE900AF8EEE77A052A11
:10ABA000C7ED047A3DF491A8DEED147A9DED0F4ACD
:10ABB00065EEA77AE4EE267AB0EE474AA7EE864A1B
:10ABC000F0EE447ABAF1000F00F01784B4EEC45AE4
:10ABD000F1EE10FA40F3118408469842A8BF1846D7
:10ABE00007EE900AF8EEE77A062AC7ED057A3DF4FB
:10ABF0006CA8DEED187A9DED104A65EEA77AE4EEBA
:10AC0000267AB0EE474AA7EE864AF0EE447ABAF1C9
:10AC1000000F00F0E883B4EEC45AF1EE10FA40F3EE
:10AC2000E28308469842A8BF184607EE900AF8EE5D
:10AC3000E77A072AC7ED067A3DF447A8DEED1C7ACD
:10AC40009DED114A65EEA75AE4EE265AA5EE867AE6
:10AC5000BAF1000F00F0BF83B4EEC57AF1EE10FA3E
:10AC600040F1B9830A469A42A8BF1A4604EE902AD8
:10AC7000F8EEE44AC7ED074AFDF727B807EE903A29
:10AC8000DFED356AB8EEE77A66EEA65A9FED335AE5
:10AC90009FED336ADFED337AA5EE856A26EEA55A7D
:10ACA000E5EE867AE5EE276A26EE870AFEF75CBFB8
:10ACB0004FF0000BB6EE007A67EE877AF4EEE57A95
:10ACC000F1EE10FA7FF7E8ACF0EE675AFCF768BCDB
:10ACD000254826F097FBFDF75FBE244826F092FB3F
:10ACE000FDF754BE224826F08DFBFDF75BBED4F87D
:10ACF000B4214B003AB156785A1800EB82025278D0
:10AD0000B242BDF4D3A90B44002200EB8300A4F8A7
:10AD10000822C4F80C22C4F8B401FDF7C7B9154BDA
:10AD20009FED156AB3F90020B3F9023007EE902ABF
:10AD300006EE903AF8EEE77AF8EEE66A27EEE87A61
:10AD400060EE277AA0EE267AE8EEA67A27EE067A5B
:10AD50008FE400BF6C30012084F9223F92E741B9B3
:10AD60009730083C15A82ABE186B01202C6C0120D6
:10AD70005C6B0120F83B0120CDCCCC3D6C740120F4
:10AD80009EED005ADDED0A4A25EE855AA4EEA65A3C
:10AD9000F0EE474AE5EE064ABDEEE45A15EE100A1B
:10ADA000814200F333829842A8BF184605EE100A8C
:10ADB000B8EEC55ABBF1000F00F02E85BD4F012A39
:10ADC00087ED005A3CF481AF9EED045ADDED0B4A4D
:10ADD00025EE855AA4EEA65AF0EE474AE5EE064A5D
:10ADE000BDEEE45A15EE100A814200F30C8298423F
:10ADF000A8BF184605EE100AB8EEC55ABBF1000F01
:10AE000000F00085022A87ED015A3CF45EAF9EED0A
:10AE1000085ADDED0C4A25EE855AA4EEA65AF0EE4E
:10AE2000474AE5EE064ABDEEE45A15EE100A8142A5
:10AE300000F3E6819842A8BF184605EE100AB8EE66
:10AE4000C55ABBF1000F00F0FB84032A87ED025ABC
:10AE50003CF43BAF9EED0C5ADDED0D4A25EE855AD4
:10AE6000A4EEA65AF0EE474AE5EE064ABDEEE45AD5
:10AE700015EE100A814200F3C0819842A8BF18461F
:10AE800005EE100AB8EEC55ABBF1000F00F0CE84F3
:10AE9000042A87ED035A3CF418AF9EED105ADDEDFD
:10AEA0000E4A25EE855AA4EEA65AF0EE474AE5EE84
:10AEB000064ABDEEE45A15EE100A814200F39A816B
:10AEC0009842A8BF184605EE100AB8EEC55ABBF165
:10AED000000F00F07884052A87ED045A3CF4F5AEA3
:10AEE0009EED145ADDED0F4A25EE855AA4EEA65AC2
:10AEF000F0EE474AE5EE064ABDEEE45A15EE100ABA
:10AF0000814200F374819842A8BF184605EE100AEA
:10AF1000B8EEC55ABBF1000F00F04B84062A87ED4E
:10AF2000055A3CF4D2AE9EED185ADDED104A25EEDE
:10AF3000855AA4EEA65AF0EE474AE5EE064ABDEE63
:10AF4000E45A15EE100A81426ADC9842A8BF1846FE
:10AF500005EE100AB8EEC55ABBF1000F00F00184EF
:10AF6000072A87ED065A3CF4B0AE9EED1C5ADDED83
:10AF7000114A65EE855AE6EEA45AA6EE257ABDEE94
:10AF8000C77A17EE102A914203DC9A42A8BF1A46EC
:10AF9000114607EE101AB8EEC77ABBF1000F00F0A9
:10AFA000278487ED077AFCF790BE77EEC76AF0EE4C
:10AFB000477AFEF762BDBEF834209FED3F7A07EE78
:10AFC000902A3E4AF8EEE77A67EE877AC2ED007A79
:10AFD000FCF7D3BD9FED3A0ADFF8048125EE800A25
:10AFE00029F064FCA8F80600FEF78DBB354B1B6802
:10AFF00013F0805B7FF45EAEFEF7D9BD3249334873
:10B000000A46FEF7C7BB0246FFF704BBDFF8C4E001
:10B010007245BFF610AB02F50C42A032FFF70BBB36
:10B0200005EE101A96E704F0F3FD049BDFF8B080FC
:10B03000C01A274BA8F802001F78FEF78FBA2548E0
:10B040008242BFF6E0AA02F50C42A032FFF7DBBA5B
:10B050002149039391ED000A049229F027FC1F492E
:10B06000DFF880E0D1F8EC10DFF874808EFB013E51
:10B07000C917A8F80000C1EBAE11039B049A07EEB4
:10B08000901AF8EEE77AFDEEE77A17EE901AA8F834
:10B090000210FCF7CCBD04F0BBFD049BDFF8408040
:10B0A000C01AD4F8AC91D4F8A861A8F80200FEF751
:10B0B00031BC00BF6C3001206F12833A7800012050
:10B0C0000000C84264360120983201206C21012022
:10B0D00080370120B0B9FFFF5C380120B8000120A3
:10B0E00084370120D34D621035FA8E3CDB0FC93F07
:10B0F0000000000007EE906A1FED057A5FED056A1B
:10B10000F8EEE77A84F8846167EE877A37EEA67AFC
:10B11000BDEEC76A16EE103A2033402B40F2CE81C6
:10B120005FED0D6ABDEEE77AD24BC3ED016A17EE13
:10B13000103A2033402B00F29A819FEDDA7AF4EE38
:10B14000C77AF1EE10FA40F3F682DFEDD35A9FEDA5
:10B15000D16AF4EEC67A37EEE57AF1EE10FAF0EE47
:10B16000477AF6DCDFEDD47AB4EEE77AF1EE10FA46
:10B1700040F1DE82DFEDC85A9FEDC86AB4EEC67AB0
:10B1800077EE257AF1EE10FAB0EE677AF6D49FEDFD
:10B19000C47AF4EEC77AF1EE10FA40F3D9819FED4C
:10B1A000C17A77EE677A67EEA75A9FEDBF5A9FED97
:10B1B000BF6A9FEDBF7AA5EE856A27EEA55AA5EE78
:10B1C000867AE5EE077AC4ED627AFDF786BE04F072
:10B1D0001FFD049BDFF8B482C01AA74B99F800202A
:10B1E000D4F8A861A8F804001F78FEF724BC05EE87
:10B1F000101A8DE605EE101A67E605EE101A41E604
:10B2000005EE101A1BE605EE101AF5E505EE101A0C
:10B21000CEE50AA8FDEEE74A984F00EB8202DFF880
:10B2200070E214EE901A0394914652469A465B4699
:10B23000D34605E0484507F11007EEEC014A2CD053
:10B24000D7ED004AB0EC014A65EEA44AE6EE844A26
:10B25000B0EE474AA6EE244A32B1B4EE445AF1EEBB
:10B2600010FAC8BFB0EE674ABDEEC44A04EE901AA9
:10B2700014EE10AA514504DCDA45A8BFDA4604EE04
:10B2800090AAF8EEE44A002BD4D1049C002CD1D132
:10B29000E045B8BFF0EE674ACCE7039CFCF715BD6C
:10B2A000774B1B78032B00F0DD810023FEF7AABF4C
:10B2B000744B03F18008FEF7A5BB9FED738AFFF77F
:10B2C0005EBB9FED718AFFF782BBDFED767AF4EE0D
:10B2D000E76AF1EE10FA40F34E82DFED6F5A9FED10
:10B2E0006D6AF4EEC66A76EEE57AF1EE10FAF0EEEB
:10B2F000676AF6DCDFED706AF4EEE67AF1EE10FADA
:10B3000040F16F82DFED645A9FED646AF4EEC67A15
:10B3100077EEA56AF1EE10FAF0EE667AF6D4DFED7C
:10B32000607AF4EEE76AF1EE10FA04DDDFED5D7AA3
:10B3300077EEE66AA8E4DFED5F7AF4EEE76AF1EE15
:10B3400010FA7FF5A1ACDFED5C7A77EEE66A9BE45C
:10B35000337DFEF70DBD93F8FF21AA2A7EF4E9ACF8
:10B36000D3F8C62142B193F8C21101F0F7000628C4
:10B370002AD00B39012927D9D3F8D62142B193F825
:10B38000D21101F0F70006281ED00B3901291BD974
:10B39000D3F8E6214AB193F8E211A1F10B0001289C
:10B3A00012D901F0F70106290ED0D3F8F621002AB0
:10B3B0003EF4BFAC93F8F23103F0F701062903D055
:10B3C0000B3B012B3EF6B5AC41F2FC110123725050
:10B3D000B370FEF737BDFDEEC77A17EE902A8A42AA
:10B3E000FFF646AC3FE4FDEEE77A17EE900A88429E
:10B3F000BFF618AC07EE901A19E4FDEEE77A17EEE7
:10B40000900A8842BFF6E9AB07EE901AFFF7EABB55
:10B41000FDEEE77A17EE900A8842BFF6B9AB07EE69
:10B42000901AFFF7BABBFDEEE77A17EE900A884252
:10B43000BFF689AB07EE901AFFF78ABBFDEEE77AFD
:10B4400017EE900A8842BFF659AB07EE901AFFF745
:10B450005ABBFDEEE77A17EE900A8842BFF629AB99
:10B4600007EE901AFFF72ABB4146FEF7E6B9DFED7B
:10B47000067AA8E678000120803701206C7401204C
:10B48000D82D01206C21012000000000843701200C
:10B490006C300120E4CB1641DB0FC940E4CB16C170
:10B4A000DB0FC93FDB0F494092E741B99730083CB9
:10B4B00015A82ABEDB0FC9BFDB0F49C0F4EEE67A40
:10B4C000F1EE10FA40F3D2805FED0D5A1FED0F6AD6
:10B4D000B4EEC67A77EE656AF1EE10FAB0EE667AEF
:10B4E000F6DC1FED0B7AF4EEC76AF1EE10FA40F1CC
:10B4F000C0805FED175A1FED176AF4EEC66A36EE8C
:10B50000A57AF1EE10FAF0EE476AF6D45FED1C6A08
:10B51000B4EEE67AF1EE10FA27DD5FED1E6A36EE44
:10B52000C77A67EE075A1FED205A1FED206A5FEDBC
:10B53000206AA5EE856A27EE255AE5EE866AA5EE15
:10B54000267AF0EE476AEDE507EE901AFFF790BA1B
:10B550001FED287AF4EEC77AF1EE10FA7FF523AEEC
:10B560001FED2B7A77EE677A1DE65FED2E6AB4EE5B
:10B57000E67AF1EE10FAD4D55FED316A36EEC77A8D
:10B58000CFE7A8F80600A5F8B890FCF796BD137CA5
:10B59000022B7EF46CAC92F8FE31552B7EF467AC36
:10B5A00092F8FF31AA2B7EF462ACB2F80EC041F2E1
:10B5B000102156F80800A74B0CEB0008C3F80080D8
:10B5C00092F80DE00EF1FF3346F801E07F2B3EF6D6
:10B5D0004EACCEF100033EEA03037EF448AC4FEAE2
:10B5E0004E2341F21821013B7350D08A00B9506AB2
:10B5F00041F204239849F050B2F811305B0103F294
:10B60000FF135B120B60B2F8131001B9116A40000E
:10B610009C4440F6F47941F2082A8444A1EB0C01E1
:10B62000B1FBFEF1494546F80A1040F2D6804FF6CC
:10B63000F47E714540F2D88003213170D26A4344D0
:10B64000864941F20C2E18440B7841F21C2146F831
:10B650000E0072500BB928F0AFFFB3780133B3700E
:10B66000FCF7F9BF1CF052FCFCF720BDF0EE476A76
:10B6700037E7B0EE667A49E7DFED797AF4EEE7CAAC
:10B68000F1EE10FA5ADCDFED777AF4EEE7CAF1EE6C
:10B6900010FA53D4744B93ED007AF1EE477AB4EE7E
:10B6A000E7CAF1EE10FA4FD48CFE47CA6F4B87ED14
:10B6B00000BA1B689342BBF65AACFCF717BE6C4A43
:10B6C0006C4B10681B689847079BDBED007A93ED85
:10B6D000007A694B27EE277A97ED006A334427EE0C
:10B6E000287AD3ED007A654B67EE277AD3ED005ABE
:10B6F000B0EE467A624BF1EE656A83ED020AA7EE80
:10B700008C7AB4EEE67AF1EE10FA1AD55D4B1B781E
:10B71000012B02D0192B7BF462ACDFED5B7AB4EE27
:10B72000E7CAF1EE10FACCBF01230023FBF762BC9D
:10B73000F0EE477A2BE5B0EE677A13E59FED53CA3A
:10B74000B4E7C7FE656AE1E7B0EE67CAAEE7022874
:10B750007CF481AF012341F2B4127370B354FCF74F
:10B760007ABF049800287FF4FBABE045B8BFB0EE89
:10B77000675AFFF7F5BBF0EE667ABBE5132B05D1F0
:10B78000B0EE480A29F092F8AAF80000B0EE480A94
:10B79000D5F87C373E4898473E4BB0EE408A1B7840
:10B7A000132B7BF4DAAA29F081F8AAF80200FBF740
:10B7B000D4BA049800287FF4B1ABE045B8BFB0EE2E
:10B7C000675AFFF7ABBB049800287FF484ABE045D1
:10B7D000B8BFB0EE675AFFF77EBB01233370FEF7A8
:10B7E00046BBF0EE676A9AE502210022317026E737
:10B7F000049B002B7FF4D5ABE045B8BFB0EE677A71
:10B80000FFF7CFBB049800287FF4FCAAE045B8BF3F
:10B81000B0EE675AFFF7F6BA049800287FF4CEAA74
:10B82000E045B8BFB0EE675AFFF7C8BA04980028E1
:10B830007FF42EABE045B8BFB0EE675AFFF728BBE8
:10B84000049800287FF401ABE045B8BFB0EE675A1A
:10B85000FFF7FBBA746C0120946C0120546C01203A
:10B8600000C0F84400C0F8C4EC2B0120D02B01200C
:10B87000642B0120782B0120882B0120F02B012044
:10B8800034300120B4250120000096420000000061
:10B89000E8A801208037012038B50B4C23688BB114
:10B8A0005A680546821A002A04DA0CE05A68AA1A75
:10B8B000002A07DB9A6818461B68226098472368AD
:10B8C000002BF3D138BD38BDB02F012000210B4B28
:10B8D00010B40A460124017202E007290BDC9C79AE
:10B8E000A40702F1010202D51C7944540131042A53
:10B8F00003F11803F1DD5DF8044B70474C9904081F
:10B9000039230370704700BF012333213222417174
:10B91000C27003700371837010B4312444705DF8F9
:10B92000044B70471F22032302704370704700BF0F
:10B9300008B507F079FBF5F7D3FB00BF024A034BCC
:10B94000127819781AF064B8642101206521012069
:10B95000A0F10A032DE9F04F0C462DED028B89B0C2
:10B96000E72B00F2EA86DFE813F01C01E806E806A0
:10B97000E806E806E806E806E806E806E806E80657
:10B98000E806E806E806E806E806E806E806E80647
:10B99000E806E806E806E806E8066F04E806E806B2
:10B9A000E806FB03E806E806E806F303E806AF034B
:10B9B000E806E806E806E806E8067F03E80653031B
:10B9C000E8064003E806E806E8063A033303E8061B
:10B9D0002603E806E8061F03E806F702E806E8067D
:10B9E000E806DB02E806E806E806E8065305E8068E
:10B9F000FC00E80697057305E806E806E806E80691
:10BA0000E806E806E8065906E8062A06E806B30648
:10BA1000E806C005E8061506E806E806E806E806B2
:10BA20004B0411040A04D304E800570222027B02EB
:10BA30001802E806E001C201E806E806E806E806A2
:10BA4000B701E806E8069601E806E806E806CC0233
:10BA5000B502A102E806E806E806E8069202BC0480
:10BA6000E8069C04E806E806E806E806E806E806B4
:10BA7000E806E806E806E806E806E806E806E80656
:10BA8000E8064B04E806E806E806E806E806E806E5
:10BA9000E806E806E806E806E806E806E8062D01F6
:10BAA000E806E806E806E806E806E806E806E80626
:10BAB000E806E806E806E806E806E806E806E80616
:10BAC000E806E806E806E806E806E806E806E80606
:10BAD000E806E806E806E806E806E806E806E806F6
:10BAE000E806E806E806E806E806E806E806E806E6
:10BAF000E806E806E806E806E806E806E806E806D6
:10BB0000E806E806E806E806E806E806E806E806C5
:10BB1000E806E806E806E806E806E806E806E806B5
:10BB2000E806E806E806E806E806E806E806E806A5
:10BB3000E806E806E80691046401A64E337853B19E
:10BB4000A54F002537F8021F204605F087F801357C
:10BB50003378AB42F6DC012009B0BDEC028BBDE8C6
:10BB6000F08F9C4E3378002BF5D09C4F0025B846C3
:10BB70002368204617F815200135591C08F10208E2
:10BB800021601A7018F8011C01EB810101EB8101A1
:10BB900001F2EE2189B205F061F83378AB42E7DCBF
:10BBA000D9E78F4D284627F08FFC0028D3DD2B46A0
:10BBB0000544226813F8011B501C9D42206011703F
:10BBC000F7D1C8E70B68DFF84CC2591C9CF800207D
:10BBD00021601A709CF80030002BBCD0814E0023ED
:10BBE000814D824882492268013316F8017F02F1B3
:10BBF000010EC4F800E01770226815F8017F02F109
:10BC0000010EC4F800E01770226810F8017F02F1FD
:10BC1000010EC4F800E01770226811F8017F02F1EC
:10BC2000010EC4F800E017709CF800209A42DADC9C
:10BC300091E7704B03F170052268073313F8071C76
:10BC4000501C20601170226813F8061C501C2060E4
:10BC50001170226813F8051C501C206011702268B6
:10BC600013F8041C501C20601170226813F8031C88
:10BC7000501C20601170226813F8021C501C2060B8
:10BC8000117013F8011C9D42226802F1010020602E
:10BC90001170D1D15FE7584D05F16006A9882046A3
:10BCA00004F0DCFFE988204604F0D8FF298920460B
:10BCB00004F0D4FF2368AA7A2046591C21601A7028
:10BCC0002368EA7A591C21601A7055F80C1B04F09D
:10BCD000AFFFAE42E2D13EE7522348492268501CF2
:10BCE0002060137011F8013F002BF7D133E70023D8
:10BCF0004348226803EB430105680133561C6D5C21
:10BD00000A2B26601570026825680A4405F10106B1
:10BD1000527826602A70026825680A4405F10101FC
:10BD2000927821602A70E4D115E7364D00230A6825
:10BD30002968501C09782060117029682268897868
:10BD4000501C206011702A6821681A440133481C75
:10BD50005279032B20600A70F5D1236820462A68A7
:10BD6000591C127A21601A7023682A68591CD278EB
:10BD700021601A7023682A68591C127921601A7090
:10BD80002B68598904F06AFF2A6823680120527AD7
:10BD9000191821601A702A6814E10021204604F065
:10BDA00047FF2046002104F059FF0120D4E6164B3E
:10BDB0000846198804F052FF144B2046198804F0F5
:10BDC0004DFF134B226801201B781118034021609E
:10BDD0001370C1E6C88801204E70012080B4012094
:10BDE000A0360120333C0120433C0120633C01206C
:10BDF000533C0120AC260120B8250120887204089C
:10BE00006088012000730120483B01204A3B01204B
:10BE1000FC3A0120313C0120974B08460A681B7808
:10BE2000511C964D03F002032160137023682A7D94
:10BE3000591C21601A70296804F0FAFE69682046CE
:10BE400004F0F6FE2989204604F008FFE98920461F
:10BE500004F004FF2046298A04F000FF01207BE65D
:10BE6000874D0846298804F0F9FE6988204604F0C9
:10BE7000F5FEB5F90430834A2046D91782FB032327
:10BE8000C1EBA30189B204F0E9FE012064E67E4D16
:10BE90000846298A04F0E2FE698A204604F0DEFEA4
:10BEA0002046A98A04F0DAFE012055E60B6801203D
:10BEB000764A1E187649157826601D7023688978A1
:10BEC0001D18744A2560197023689278191821602A
:10BED0001A7041E60A6808466F4B561C6F491D7878
:10BEE0002660157022685D78561C266015702268E1
:10BEF0009B78551C25601370C98804F0AFFE0120A3
:10BF00002AE6664D0846298804F0A8FE698820467E
:10BF100004F0A4FE2046A98804F0A0FE01201BE640
:10BF2000F5F7C4FD236800285D4D03F101012046AB
:10BF30000CBF0222032221601A70298804F078FEC7
:10BF4000A968204604F074FE05F060FA0146204618
:10BF500004F06EFE0120FFE50B680846514A5E1CA6
:10BF6000514D1178514A26601970116804F060FE35
:10BF700023684F4A2046591C127A21601A7029887A
:10BF800004F06CFEA988204604F068FE298920464A
:10BF900004F064FE0021204604F060FE20460021EB
:10BFA00004F05CFE0120D7E508460822404904F071
:10BFB00012FE0120D0E50B6801203E4A1D18917841
:10BFC0002560197023685278191821601A70C3E52A
:10BFD0000B6801229918104621601A70BCE50846CA
:10BFE000002104F025FE0120B6E5334D334E05F166
:10BFF000300795F90210324B93F9062008338A4234
:10C0000000F09E83B342F7D10835AF42F1D1A2E5EB
:10C010002C4B03F15A052268063313F8011C501CFF
:10C0200020601170226813F8061C501C20601170EB
:10C03000226813F8051C501C20601170226813F848
:10C04000041C501C20601170226813F8031C501C43
:10C050002060117013F8021C9D42226802F1010059
:10C0600020601170D7D176E50B680120104A1918AD
:10C07000527D21601A706FE59C3A0120A03A0120A0
:10C080007C3A0120676666663899012054A9012030
:10C09000C4360120D4360120BC360120F4740120BE
:10C0A0004008012090300120A8870120E4360120BB
:10C0B0000CAB0120E0360120DCB00120E8AA012011
:10C0C000B8AA01201C730120BA4D08460B682A7AD1
:10C0D000591C21601A70A98B04F0C0FD298B2046E1
:10C0E00004F0BCFD698B204604F0B8FD2368EA7CAF
:10C0F0002046591C21601A70A98C04F0AFFDE98C10
:10C10000204604F0ABFD2368AA7F2046591C21601D
:10C110001A70236895F82020591C21601A70698CC8
:10C1200004F09CFD2368EA7A2046591C21601A70AD
:10C13000E96804F07DFD236801202A7C191821603C
:10C140001A70236895F82120191821601A7003E5E8
:10C150000B680120984A1D1811782560197031E785
:10C16000964D0846298804F079FDA988204604F0F8
:10C1700075FD2046298904F071FD0120ECE4084694
:10C1800010228F4904F027FD0120E5E48D4B1B8B25
:10C19000B3F5006F00F2A483B3F5806F00F2C383A0
:10C1A000B3F5007F34BF01270227874D05F10C0648
:10C1B00055F8041B204691FBF7F189B204F04EFDBF
:10C1C000B542F5D1814D824F05F10C06B5EC010A5F
:10C1D000D7ED097A80EE270A28F068FB81B2204665
:10C1E00004F03CFDAE42F1D17A4D05F10C0655F854
:10C1F000041B204689B204F031FDB542F7D1AAE410
:10C2000000238146DFF8F08101211D464FF6FF7AB9
:10C21000DFF8E8B1049306930593079305E0013531
:10C220000B2D00F0AA8218F9011F4F1C4AFA05F3E2
:10C23000F5D0DE07F3D5BBF800302B41D807EED59B
:10C2400006A805F03BF8EAE7634D05F150062878AB
:10C25000043526F037F82368027A591C21601A70D9
:10C26000236815F8032C591C21601A70236815F8EF
:10C27000022C591C21601A7015F8012CAE4223685B
:10C2800003F1010121601A70E1D164E4534D0846C5
:10C29000E98904F0E3FC2046A98904F0DFFC0120D1
:10C2A0005AE40B684E4F591C3A7821601A703B785B
:10C2B000002B3FF450AC0025EEB2013530460FF0B4
:10C2C000CDFA236842783046591C21601A700FF06D
:10C2D000C5FA0189204604F0C1FC3B78AB42EBDC97
:10C2E00039E40A6801203F4B151819782560117050
:10C2F00022685978151825601170226899781518E8
:10C30000256011702268DB7811182160137023E416
:10C31000354D364E05F12007DFF8E480DFF8E49074
:10C320009FED338ADFF8E0B0DFED328ADFF8DCA082
:10C330000DE0FCEEE77ACDED017ABDF8041004358E
:10C34000204604F08BFC1836BD423FF404AC717CEF
:10C350000029F4D098F80030D5ED007A012BE8D10F
:10C36000D9F80030DB0440F1A782F5EE407AF1EE17
:10C3700010FA00F0BE82F4EEC87AF1EE10FA00F185
:10C38000B882F4EEE87AFDEEE77AF1EE10FA17EEF5
:10C39000903A00F2D3826FF4F972303B02FB03F360
:10C3A0008AFB0312D9171344C1EB632101F2DB515D
:10C3B00089B2C4E70CAB012090300120A88701208E
:10C3C0005C300120283A0120643A01206CA9012048
:10C3D00068A101206875012094300120C436012035
:10C3E00061370120183C01206C3001207898012031
:10C3F0000000404200E08244B8720408603B012023
:10C400005C99012078A90120DB9B914121053483AF
:10C410000B680846A24D591C2A7921601A702368BE
:10C420006A79591C21601A70298804F017FC236866
:10C43000AA792046591C21601A70698804F00EFC04
:10C4400023680120EA79191821601A70FFF784BB6C
:10C450000B680125934E5A190A601D700B68B2785B
:10C46000591921601A700AF0BBFE23688E4A5F19C1
:10C470008E4927601870B1F90010B2F9000004F07D
:10C4800073FD23685A19226018702046318804F021
:10C49000E5FB2846FFF760BB0A68012693190B608D
:10C4A000167018F0C5F8002840F01C820346804D35
:10C4B000804A216841F2B41741F27816204601F112
:10C4C000010EC4F800E00B702368D15D5F1C27608B
:10C4D00019709159890A04F0ABFBA96A20464908F2
:10C4E00004F0A6FB0120FFF737BB0021204604F033
:10C4F000B5FB00212046704D0E4604F0AFFB2046F0
:10C50000314604F0ABFB236820465A1C22601E70A3
:10C5100023682A68591C92F82C2021601A7023681D
:10C520002A68591C92F8362021601A7023682A68FC
:10C53000591C92F8372021601A7023685A1C226017
:10C540001E7023685A1C22601E7023685A1C2260C9
:10C550001E702B68598F04F081FB2B682046198FC1
:10C5600004F07CFB23682A682046591C92F82E2090
:10C5700021601A7023685A1C22601E702B68598E25
:10C5800004F06CFB2B682046998E04F067FB0120B9
:10C59000FFF7E2BA0B680120484A1E184849D578CF
:10C5A00026601D70236849791D18464A2560197058
:10C5B0002368D278191821601A70FFF7CDBA424E5D
:10C5C000F378002B00F080810B6801220821981875
:10C5D000206019702368991821601A70236820461A
:10C5E0003A4D591C2A7921601A702368AA78591C7F
:10C5F00021601A70298804F031FBE989204604F093
:10C600002DFB23680120F279191821601A70236824
:10C61000EA78191821601A70FFF79EBA19F0ECF940
:10C62000FF28064600F0688108A900250DF10D00DD
:10C6300001F8125D8DF80D5012F076F908A800F897
:10C64000115D12F065F908A800F8105D12F054F9B8
:10C6500008A820F8085D19F0AFF9236820465A1C95
:10C6600022601E7023689DF80D20591C21601A70ED
:10C6700023689DF80E20591C21601A7023689DF8CC
:10C680000F20591C21601A7023689DF81020591C36
:10C6900021601A70BDF8181004F0E0FAFFF75BBAD9
:10C6A0000C75012068B60120843601208C360120EB
:10C6B000246F0120745A012060880120C4360120B3
:10C6C0006C3F0120D436012054A901203899012063
:10C6D000AE4E08460B687279AD4D591C21601A7038
:10C6E0002B68198C04F0BAFA2B682046D98B04F019
:10C6F000B5FA7189204604F0B1FAB189204604F0F8
:10C70000ADFA2B682046598C04F0A8FA2B68204615
:10C71000998C04F0A3FAF189204604F09FFA318A3B
:10C72000204604F09BFA2A682368012092F826200C
:10C73000191821601A70FFF70FBA0020FFF70CBA22
:10C74000236820465A1C22601970298804F086FA52
:10C750002368EA78591C21601A7023682A79591CC9
:10C7600021601A702368AA79591C21601A70236805
:10C770006A79591C21601A7046E40025DFF840A24E
:10C780004FF008080135C5F12002A5F12003252D41
:10C790002AFA05F608FA02F228FA03F310D0164333
:10C7A0001E43002306F001021343EBD0E8B20EF063
:10C7B000DFF80028E6D0294606A804F07FFDE1E76F
:10C7C000744B1B78DA0700F19E800025724E2F46CD
:10C7D00002E00135252D0DD02946304604F07DFDBF
:10C7E0000028F6D0294606A804F077FD00285ED17F
:10C7F0000137EEE7694B2046694DB3F8501004F05D
:10C800002DFA684B2046198889B204F027FA664B46
:10C81000204619684A01C1F34003C1F3800EC1F3F9
:10C82000C00602F020021343C1F3401201F01001D0
:10C8300043EA4E0343EA860343EAC203194304F082
:10C840000DFA04A90422204604F0C5F923682978CA
:10C8500020465E1C554A2660197011886429A8BFBD
:10C86000642104F0FBF9B9F1960F51D00021204664
:10C8700004F0F4F9B7F11903256805A9204648BF6B
:10C88000A7F112036E1CA3F3C40326601A462B7093
:10C8900004F0A1F923681021454A5D1C204625605B
:10C8A0001970118804F0C4F90120FFF755B9394611
:10C8B00004A804F003FD9BE7F4EEC87AF1EE10FA49
:10C8C0004CDA4FF47A713AE50B68B178581C394A62
:10C8D0002060197023681278591C21601A707DE657
:10C8E000082762E4344D95F82430F3B93346334ACF
:10C8F000DFE540F2DC5122E5236801201A182260AE
:10C900001E70FFF729B9069B43F0010306935CE70D
:10C9100023680322591C21601A7023686A78591C05
:10C9200021601A70A6E704273FE4244A51780229BF
:10C9300026D003290CBF04233346BAE540F2F31294
:10C94000A3F5836302FB03F38AFB0312D917134495
:10C95000C1EB632101F2DD5189B2F0E4FDEEE77A2B
:10C9600040F2E73217EE903A303B02FB03F38BFBC9
:10C970000312D917C1EB622101F2E93189B2DEE479
:10C98000042B34BF0223032393E500BF54A90120E5
:10C99000608801200D7201201CB50120B800012023
:10C9A0005488012004940120983A0120DC2D0120B4
:10C9B0006EB10120B8360120246F0120745A012085
:10C9C00090E33FF408B50121022003F0B5FC094BC8
:10C9D0001B7803F00503052B08D00021012003F08C
:10C9E000ABFC0021084603F0A7FCFEE714F04CFE68
:10C9F000F3E700BF608701200228094B094928BFDF
:10CA0000022000EB8002C0EBC20230B4064D441C91
:10CA100003EB42032870E0B20B6030BC1BF0AEBBEE
:10CA20004CB50120608801205488012038B503F0FE
:10CA300043FE094C094B002209490A480A4D1A7065
:10CA40005A702560086022F0BFFD03F095FEBDE836
:10CA5000384022F0A1BD00BF608801205488012029
:10CA600000730120648801204CB5012008B522F034
:10CA7000ABFD03F081FEBDE8084022F08DBD00BF94
:10CA8000434B99895A89914210B501D300225A81AA
:10CA9000198ADA89914201D30022DA81DA78072AE9
:10CAA00018BF002A3B4A3CD092F85B2001213A4C47
:10CAB00000200A2A99702170D8715FD00C2A5BD1AE
:10CAC000364CDFED377AA278062A3DD92179DFEDA1
:10CAD000356A002940D19B782F4A07EE103A117829
:10CAE000B8EEC77A27EE277A07EE901AF8EEE77AC3
:10CAF00067EE877AF4EEE76AF1EE10FA3BDDC6EEF8
:10CB0000877AFDEEE77A17EE903A102BA8BF102334
:10CB1000012BB8BF0123DBB28B4238BF0B46137029
:10CB200010BD92F85B200A2A2BD00C2ADA792CD17E
:10CB3000DFED1D7A002A9FED1B7A18BFF0EE477AD1
:10CB4000164CA278062AC1D8184901EB8201D1ED12
:10CB50000F6A21790029BED0013A032A0BD8B7EE1B
:10CB6000000A80EE260A27F0A1FE2388984228BFFB
:10CB70001846208010BD10BD0A2AA1D1DFED0C7A25
:10CB8000DEE7DA79DFED0B7AD4E7DFED0B7AD1E778
:10CB900054A9012068A10120B8360120389901204C
:10CBA0006F12833A6F1203380AD7A33988720408C8
:10CBB0000F506E3A5304E9386F1203392DE980485B
:10CBC0000A2385B001308B4D02938B4FC3B28B4C3F
:10CBD0008B4E03931CF0D0FA4FF4FA7ADFF82492CC
:10CBE0004FF0100C4FF47A70D9F80430C3F30803F7
:10CBF000002B40F0C180EFF31183002B40F0BC808C
:10CC00002968A26800BF2B689942F9D1D7F800E0E3
:10CC100000FB0EF39B1AB3FBFEF300FB01314FF058
:10CC2000010E0191D9F80430C3F30803002B40F042
:10CC30008780EFF31183002B40F082802B68A1687E
:10CC400000BF2A689342F9D1D7F800B000FB0BF27D
:10CC5000521AB2FBFBF200FB0323019A9B1AB3F5B5
:10CC60007A7FDFD3BAF1010ABED1039B002B40F0DB
:10CC7000BD804FF47A7ADFF88C914FF0100C50465B
:10CC8000D9F80430C3F30803002B40F09280EFF38F
:10CC90001183002B40F08D802968A26800BF2B68AB
:10CCA0009942F9D1D7F800E000FB0EF39B1AB3FBD1
:10CCB000FEF300FB01314FF0010E0191D9F8043071
:10CCC000C3F3080303BBEFF31183EBB92B68A1682F
:10CCD00000BF2A689342F9D1D7F800B000FB0BF2ED
:10CCE000521AB2FBFBF200FB0323019A9B1AB3F525
:10CCF0007A7FE3D3BAF1010AC2D1029B013B0293CE
:10CD00007FF468AFF4F7DAF9EFF311888CF3128847
:10CD1000A1682368DB0302D5C6F800E0A1682B6890
:10CD20005FFA88F8326888F31188D7F800801A44CF
:10CD300000FB08F35B1AB3FBF8F300FB0233D4E704
:10CD4000EFF311888CF31288A1682368DB0302D506
:10CD5000C6F800E0A1682B685FFA88F8326888F3AB
:10CD60001188D7F800801A4400FB08F35B1AB3FB64
:10CD7000F8F300FB023370E7EFF311828CF31288B3
:10CD8000D4F808E02368D90303D501233360D4F82D
:10CD900008E02B68D2B2316882F311883A681944EE
:10CDA00000FB02F3A3EB0E03B3FBF2F300FB013134
:10CDB00035E7EFF311828CF31288D4F808E023688A
:10CDC000D90303D501233360D4F808E02B68D2B22D
:10CDD000316882F311883A68194400FB02F3A3EB2F
:10CDE0000E03B3FBF2F300FB013164E718461CF0BD
:10CDF00029F83EE70C9401201094012010E000E097
:10CE00000894012000ED00E02DE9F047B54F22F035
:10CE1000DBFBB54EBE421ED2DFF85883DFF85893D5
:10CE20004446258862197DB14A450DD2052D0BD99E
:10CE300033886188C3F30B03994200F0F8801446ED
:10CE400025886219002DEFD171683046143603F041
:10CE50000FFCBE42E4D3A54A1378A3F117010229BF
:10CE600014D9A34911F83300002800F03581D80007
:10CE70000C186468002C00F031810144497829B114
:10CE80009C4911F833300BB9182313709A4C63780E
:10CE9000022B01D9002363702378022B00F2E88073
:10CEA000964B9A78042A00F0EA8022B91A88B2F5E3
:10CEB000F07F00F20D81924D924A2B681A40002AB1
:10CEC00000F05C81D80700F1E780590400F1EB80A5
:10CED0001A0700F1EF809B0400F1F3808A4D2B6864
:10CEE000998C5A8C914201D300225A84FFF7C8FDD5
:10CEF0001FF0E6F9002800F0CB804FF4007003F03B
:10CF0000FDFB4FF4803003F0F9FB4FF4802003F079
:10CF1000F5FB4FF4001003F0F1FB4FF0007003F04D
:10CF2000EDFB4FF0806003F0E9FB6378022B06D83D
:10CF300003EB4303754A764902EB83030B602378C6
:10CF4000022B07D803EB8301724AC3EBC10302EB48
:10CF500043032B600DF084FD002130226E4829F040
:10CF6000CBFD286805F012FD6C4B2D6803F15001D4
:10CF700002E00433994279D01A78002AF9D19C78DA
:10CF8000D8788442F5D266492846664B0A701D60FF
:10CF900018F0AAFC644AC823644864211579002269
:10CFA000634C11FB0531634F634B30F8066C634DE6
:10CFB000A46B596038602E809A60DA601A615A61F9
:10CFC0009A61DA6183F8202083F821200CB109F0FE
:10CFD000C9FB5B4B9FED5B5A1B885B4A06EE903AA0
:10CFE0009FED5A6A1388F8EEE66A557907EE103A13
:10CFF00053881479C5EE265A07EE903A544B55499A
:10D00000554A5648B8EEC77A1D72F8EEE77A5C7258
:10D01000106027EE067A67EE867ABDE8F04783ED6A
:10D02000017AC3ED007AC1ED005A22F0B5BA6379F6
:10D030009B077FF404AF7168304694F804A003F0B6
:10D0400017FB3388BAEB133F04D01436BE42FFF40B
:10D05000E7AE00E77388AA1FA11D7068C3F30B0336
:10D060009A42A8BF1A4629F022FDEEE701228AE77C
:10D0700000232370214B9A78042A7FF416AF9A8AF2
:10D08000B2F57A7FBFF417AF4FF47A729A8212E743
:10D09000334819F0DDFE30E7324803F02FFB2B68F0
:10D0A00059047FF515AF304803F028FB2B681A07A9
:10D0B0007FF511AF2D4803F021FB2B689B047FF512
:10D0C0000DAF2B4803F01AFB402003F017FB05E7D8
:10D0D0004FF4F0721A80EEE6D800CEE617241470F2
:10D0E000CBE600BF3C060008C801000890300120D4
:10D0F00018890408E0730408548801203899012035
:10D10000E436012009600002608801206488012063
:10D11000007301204CB501204024012094300120EF
:10D12000B0000120742401200C750120CA360120B2
:10D13000283A0120F4B40120A08801202C340120D9
:10D140007C220120C0C9FB488023012017B7D138B9
:10D15000C072012080220120E47201203661023D6C
:10D16000DCB001200860000209200002016000021A
:10D1700009400002028000080000010843F0080393
:10D180002B609FE608B522F01FFA03F0F5FA22F0B3
:10D1900003FAFFF739FE0120BDE808401AF0EEBFA0
:10D1A00044F620631A469C4B2DE9F04F82182DED72
:10D1B000028B93B011461C780892984A0490116033
:10D1C000002C00F0D486964A04991268914240F2ED
:10D1D0008B80944A013C944917681C7007F480576F
:10D1E000924CDFF888B205920391002F40F08980BD
:10D1F000039B5B7D002B40F04086059B1B681D0454
:10D2000001F154818A4B049A9A429BF8023000F251
:10D210001385002B40F01485864B0693059B1F68F1
:10D2200017F4805940F0CD85039BB4F906605B8B01
:10D230009E42B4BF002601267F4B1B6813F080532B
:10D2400069D0069A127812F001026AD00399498CCB
:10D2500007EE901A7949F8EEE77A91ED037A049196
:10D26000B4EEE77AF1EE10FA81F2D881002E60D1A7
:10D27000734D95F8A01000295BD1724800257249C2
:10D2800000680D6090F82D004D608D606F4900289A
:10D2900050D10870002A51D0F9064FD56C4A127847
:10D2A000D2064BD4B9F1000F48D1002B46D17B02F6
:10D2B00044D4684B1B78002B01F0DB87664B9B78CE
:10D2C000002E42F0AB803BB1644A654B12681B688C
:10D2D0009B1A002BC2F264801020594D1AF034FEC4
:10D2E000012385F8A13029E04E4B4F4A1F68059372
:10D2F00007F4805703924D4CDFF870B1002F3FF4D4
:10D3000077AF00214C4803F0E8FF00287FF470AFAE
:10D310001CF06CFE6CE7780293D4069A127802F047
:10D3200001020021464D85F8A01044490491002EC9
:10D33000A3D0464901200870002AADD1494B197885
:10D34000002952D1039AB4F900E0578B908B7745AE
:10D35000B4BF80220022B4F90250B4F904C042F0F4
:10D3600040037045D8BF1346B4F906E09B0843F06C
:10D370008002AF42B8BF134643F04002A842D8BF74
:10D380001A462F4D920895F8A29042F08003674507
:10D39000B8BF1A4642F040036045D8BF13469B0809
:10D3A00043F08002BE45C8BF134643F040028645A5
:10D3B000ACBF18461046814501F011830B46A5F815
:10D3C000A41085F8A610234A85F8A2001778002F2C
:10D3D00001F0AB825F2801F0DB826F2801F09E81B3
:10D3E000069B1B78D90741F13D81059B1B6803F023
:10D3F0000403002B40F0D28700221B4D0DF14008A2
:10D4000040F6330AC8F8042005F15009192740F204
:10D41000833610922FE000BFE0B30120B0B20120AC
:10D42000DCB3012078A901200CAB01205070012051
:10D43000404B4C000D720120643601205C38012005
:10D440009023012060880120403001204C230120DE
:10D450009C3A0120B0000120E03601200C9401200C
:10D46000709701206DB1012094300120A088012027
:10D4700004354D4520D0AA78EB7817FB02619A421B
:10D48000F6D26A7817FB0363043234F9122052454E
:10D49000A8BF5246B2F5617FB8BF4FF461728A42AD
:10D4A000E6DD9A42E4DC29782429E1D804354046B7
:10D4B00003F004FF4D45DED1644A654B177898E8C8
:10D4C000030083E80300002F00F0C486614B08933B
:10D4D00001215F4803F001FF002840F0AD829BF876
:10D4E0000330002B40F0A8825B4B07935B4E3388E0
:10D4F0001DB225F00105AFB2BB42378001F03E807E
:10D50000574D4FF002084FF014094FF0FF0A0E205C
:10D5100085F8008085F8019085F802A01AF014FDC6
:10D5200041464B48378803F0D8FE002800F09E8221
:10D5300027F0010292B2BA42328009D00E2085F85B
:10D54000008085F8019085F802A01AF0FDFC37886C
:10D55000BB0741F1FC80434BBD07434A1978506833
:10D5600008BF81F0020109930A92C1F3400102F061
:10D57000ABFE2421364803F0B0FE30B9069A13788A
:10D58000590702D523F004031370079B196811F0A3
:10D590000A0F1DD005212E4803F09FFE002801F040
:10D5A0000D8035886B0741F14E810621284803F034
:10D5B00094FE002800F0EF876F0641F13C810721BF
:10D5C000234803F08AFE002840F07A84079B1968FC
:10D5D000880600F1858437880C211D4803F07DFE04
:10D5E000002800F00A8347F48073BB42338009D0DF
:10D5F0001B4B02201421FF2218700E2059709A70C4
:10D600001AF0A2FC194B1B780E2B00F00283082B9A
:10D6100000F0FF82059B1B68580560D5144B1B79F1
:10D62000002B00F026811421094803F056FE002843
:10D6300040F0248110F008FA01201AF0C5FB002503
:10D64000DFF830A04FF0CC0917E000BF4F88012071
:10D650006436012000730120983A0120603B0120CC
:10D660001475012094960120989601209030012095
:10D67000F8370120C06C0120DDB209FB05F86B1CF6
:10D6800068B3022D2BD85AF80870002FF4D1C37854
:10D690004FF0030ED1493A4690F9020051F8233079
:10D6A00001210197CDF800E019F0FEFB0346CC22E2
:10D6B00005EB45003946079353B100EB00100135E7
:10D6C0000AEB800029F018FA079BEDB24AF80830FF
:10D6D00020F0DAFA09FB05F86B1C0028D1D1069B73
:10D6E0001D7815F0010500F0F481BD4B01221A7080
:10D6F000089B4FF0010EB4F906101868B94F428923
:10D7000087F800E0914280F2CA814FF07E52B64B1A
:10D710001A60B64A039BB4F900E01F8B92F90430FB
:10D720001078002BAEEB070392F801C014BF012262
:10D730004FF0FF32002BB8BF5B42B3F5FA7FA8BFB2
:10D740004FF4FA73984280F2A7811B1A07EE903AC1
:10D75000F8EEE77A049BBE45C3ED007A03DAF1EEFA
:10D76000677AC3ED007AB4F902E0AEEB0703002B51
:10D77000B8BF5B42B3F5FA7FA8BF4FF4FA73984283
:10D7800080F287811B1A07EE903AF8EEE77A049B45
:10D790007745C3ED017A03DDF1EE677AC3ED017AD7
:10D7A000B4F90400C31B002BB8BF5B42B3F5FA7F8A
:10D7B000A8BF4FF4FA736345CCBFA3EB0C0300235F
:10D7C000B84202FB03F3049A07EE903AF8EEE77AC8
:10D7D000C2ED027A03DAF1EE677AC2ED027A059BB6
:10D7E0001A6812F4805200F0E581B1F5FA6F804BAF
:10D7F000A8BF4FF4FA611878B1F57A7FB8BF4FF43B
:10D800007A71A1F57A71002840F0ED8179484FEAEC
:10D81000E17C794C6FF0630380FB018ECCEB6E1CD6
:10D820000CF1010E03FB0C1334F91C1034F91E40EB
:10D83000641A03FB04F380FB0340DB17C3EB6013A4
:10D840000B441BB207EE903A049BB8EEE78A83EDD7
:10D85000038A002A40F0D08433885A0624D4002D4D
:10D8600040F0AE800DF0E3FA13B0BDEC028BBDE8E2
:10D87000F08F069B1B78D9077FF5DCAE3C2011F0BA
:10D88000FDF800283FF42BAF15F052FE3C2011F0BC
:10D8900097F800283FF423AF15F04AFE3C2011F022
:10D8A0008FF80028F0D11AE7544B554AB3F90430E9
:10D8B000544982FB0302DB170988C3EBA203DFEDA7
:10D8C000526A9FED527A5B1A1BB207EE903AF8EE5D
:10D8D000E77A67EEA67A77EE876ABDEEE66A16EE1D
:10D8E000103A2033402B40F2BA87DFED496ABDEE93
:10D8F000E77A17EE103A2033402B00F2AC879FED09
:10D90000457AF4EEC77AF1EE10FA41F33883DFED91
:10D91000425A9FED426AF4EEC67A37EEE57AF1EEAE
:10D9200010FAF0EE477AF6DCDFED3D7AB4EEE77AF6
:10D93000F1EE10FA41F13F83DFED375A9FED396A7E
:10D94000B4EEC67A77EE257AF1EE10FAB0EE677A89
:10D95000F6D49FED2E7AF4EEC77AF1EE10FA00F3CA
:10D9600074869FED317AF4EEC77AF1EE10FA03D5A2
:10D970009FED2B7A77EE677A67EEA75A9FED2B5AC9
:10D980009FED2B6A9FED2B7AA5EE856A27EEA55AAF
:10D99000A5EE867AE5EE077A049A92ED016AD2ED59
:10D9A000005A27EEC67A65EEA77AA5EEA67AE6EECD
:10D9B000267A82ED007AC2ED017A002D3FF452AF53
:10D9C000099B19780A9B01F00101186802F07CFCA0
:10D9D00013B0BDEC028BBDE8F08F00BFB887040820
:10D9E0000E7201208422012028230120BC36012050
:10D9F000287601201F85EB51383701207C3A012021
:10DA0000676666666C97012035FA8E3CDB0FC93F6E
:10DA100000000000DB0F4940DB0FC940E4CB16419A
:10DA2000DB0F49C0E4CB16C1DB0FC9BF92E741B998
:10DA30009730083C15A82ABEBC4B07931B68990772
:10DA40007FF554ADBA4E3788FA070FD447F001037B
:10DA50009F4233800AD0B74B02201421FF22187056
:10DA60000E2059709A701AF06FFA378827F0020367
:10DA70009BB2BB4233803FF46EADAE4B1421FF220C
:10DA800002250E2059701D709A701AF05DFA3788C1
:10DA900061E5DFEDA97A7AE6DFEDA77A5AE6B1F51E
:10DAA000FA6F80F2A2848B1A007AC2F5FA6203FB45
:10DAB00000F393FBF2F3C3F1640307EE903AF8EE40
:10DAC000E77A9FED9E7A9E4B67EE877AC3ED007AE8
:10DAD0001FE69C4B1B780793002B7FF409AEDFF801
:10DAE000A0A2DFF8A09251461AF8030CAAF103078E
:10DAF00099F800800CF014FF002800F07D84079B4B
:10DB0000B8F1000F53D107F1080178790CF008FF44
:10DB1000002841F0C4828C49B87A0CF001FF00283B
:10DB200000F07E84B8F1020F41F094828749F87BBF
:10DB30000CF0F6FE002841F090828549387D0CF00B
:10DB4000EFFE002800F07E84B8F1040F41F0A182BE
:10DB50008049787E0CF0E4FE002841F09D827E49E9
:10DB6000B87F0CF0DDFE002800F07E84B8F1060FCF
:10DB700041F07682794997F823000CF0D1FE002815
:10DB800041F01580764997F828000CF0C9FE00286E
:10DB900000F07E84B8F1080F41F01A80714997F8BF
:10DBA0002D000CF0BDFE00283FF4A2AD09231A465B
:10DBB00000F0FFBF039B588B8142C0F21384B1F584
:10DBC000FA6FD4BFC0EB0101C0F5FA614FF47A736C
:10DBD00003FB01F1644BC0F5FA601C78B1FBF0F176
:10DBE000002C3FF413AE5B78604801FB03F380FB2D
:10DBF0000301DB17C3EB611108E627F480739BB2C6
:10DC0000BB4233807FF4F4AC594B1B780E2B7FF46E
:10DC1000FEAC328822F040039BB29A4233803FF43C
:10DC2000F9AC444B02201421FF2218700E205970C9
:10DC30009A701AF089F9EDE413B901238BF80230D8
:10DC40004C4B1B209BF821601D4606930CF090FE68
:10DC5000012E2F78824607F0010900F0958607F023
:10DC6000020304939BF82030DFF81C81424D052B02
:10DC700000F29A80DFE813F08A004E000600DB0015
:10DC8000FF00BD00012E00F0AE84B9F1000F00F0DE
:10DC90005981039B0022B8F80000B3F9181013460D
:10DCA000364F61F30F0261F30F0360F31F4261F31C
:10DCB0001F4339686260DBF8142023608A42C1F098
:10DCC0007783012E41F0E08303229BF820300492F9
:10DCD000CDE70CF079FE012808D1284F6421B8F86F
:10DCE00002303A6801FB0323CBF81030BAF1000F81
:10DCF00004D098F80630002B40F09080012E53D0CD
:10DD00001E4FDBF810203B689A42C0F0EA860123E0
:10DD10008BF82030012E6CD098F80730012B00F0E2
:10DD20001B8114F0C3F89BF82030A0E7983A01203B
:10DD3000603B012014750120000000000AD7233C3D
:10DD4000282301200E720120107401201574012077
:10DD50001A7401201F7401202474012029740120E9
:10DD60002E74012033740120287601201F85EB5189
:10DD7000903001200D7201206EB101200C94012021
:10DD800006740120800001200C750120B9F1000FFC
:10DD90009FD14FF48060BAF1000F00F0F9831AF0C0
:10DDA0001DFA0023CBF81030049B002B3FF436AA59
:10DDB00004981AF0C9F8059B1F6817F480593FF4BE
:10DDC00033AA1D218B4803F088FA00287FF42CAA7F
:10DDD000894A039BD2881B8BB4F90660991A8E423C
:10DDE00040F3748613449E42B4BF00260126FFF719
:10DDF00023BA824F39686420B8F80230002200FB51
:10DE000003134FF480608BF82020CBF810308BF890
:10DE100003201AF0CBF99BF8203028E714F046F8DD
:10DE200003224FF47A738BF82020CBF81C30734F09
:10DE30002B8843F002032B801CF0D8F83A680421A9
:10DE4000DBF81C308BF820101344CBF81830012E6F
:10DE500040F03F863B68DBF818209A42A4D2684B1A
:10DE6000187818B90CF084FD00289DD12B8823F078
:10DE700002032B80BEE7614FE9E7039A013BD27DA5
:10DE800034F913301AB140F6B832D21A13B2A3F5EE
:10DE90007A739FED5C7A5C4AB3F57A7FA8BF4FF442
:10DEA0007A7323EAE37307EE903AF8EEE77A67EEC7
:10DEB000877AFCEEE77A17EE903A1380FFF7A2B963
:10DEC000524B534AB3F90430079982FB0302DB1724
:10DED00050480968C3EBA203038088067FF57BAB3B
:10DEE0004D4B1B78990706D5DFF8508198F8143010
:10DEF000042B00F20186378817F0300F3FF46CAB2B
:10DF000010201AF053F920201AF050F9434B002248
:10DF100037881A7000214248424B434A0160116021
:10DF20004248434A19600023416081610360836075
:10DF30004361C36113605160936053619161D36128
:10DF4000FFF74ABB2D4F3B6847F230520323CBF813
:10DF50001C208BF820306BE713F0A8FF032240F65B
:10DF6000B833264F8BF82020CBF81C3060E7314FB8
:10DF70003B78002B6AD0DFF8C8804FF47A79DFF85D
:10DF8000C4B02D4B4546DFF8C0A05E46039326E0A3
:10DF9000039A115D9847032C02B219DC0246B8B10E
:10DFA00038F824E040F6CA016B88A0EB0E02A3EB20
:10DFB0000E0040F2EE2309FB02F292FBF0F202F5B2
:10DFC0007A728A42A8BF0A469A42B8BF1A4612B26B
:10DFD00001343B782AF8022F04359C4238DA072CAA
:10DFE0003046DBF80430E1B2D2DD3046984702B269
:10DFF000EEE700BF64360120F47401200C94012088
:10E00000B0000120AAF1823F583001207C3A012063
:10E01000676666666C9701209C3A0120FE3A0120F3
:10E02000FC220120F8220120F83B0120A83B01201E
:10E03000D03B012034B401200CAB0120A03A0120D8
:10E040004CB40120C88801208E230120BC4A0392D1
:10E05000BC4A42F2010CBC4904980591A2FB002B7A
:10E060000A6812EA0C0C4FEA9B1B00F0D382B748F7
:10E07000B74990F80080B74C0878B74984F8008019
:10E080000870B8F1000F04D0B34991F8008088F00F
:10E090000108B24D0F2185F82410002B00F02584D3
:10E0A000AF4B12F4805FAF480E931B78039C1E4663
:10E0B0000C93A0FB0330039A238B4FEA5000B2F875
:10E0C00024E0E48C4FF0000200EB40000D930A9432
:10E0D0000BF59674A6EB00003B780D9F08BF7746C2
:10E0E000C0B20B910F9705F1280109907046079473
:10E0F0009E46CDF81880034695F825A0A8469A4C70
:10E100009A4F0698002800F0358338F912605000C5
:10E110001FFA86F9994503D30A9DA94540F2698300
:10E1200057F82260B34580F02D83265EBCF1000FC6
:10E1300040F040830132265206317245E1DB0B98F4
:10E1400073468B4A0F2888F825A088F824000CBF56
:10E1500001210021117000F0CE83864D0120DFF8EF
:10E1600030B2854F2E883A68DBF8081046F0040676
:10E17000CBF80C20521ADBF804102E808A42744E21
:10E18000754D3070287002D900228BF82120002BA9
:10E1900000F0C683059A03991768B1F824C017F4F4
:10E1A0008057B1F818E0754E40F0CC8339466E4880
:10E1B00035460DE06A7802EB820202EB820202F23F
:10E1C000EE2292B20131023520F8022B8B420DD0A3
:10E1D00016F81120002A00F01083022AEAD00288E3
:10E1E0000131023520F8022B8B42F1D10E9A1378BF
:10E1F00001331370FEF7F9BF1D21614803F06DF87C
:10E2000000283FF429AB9BF80330002B7FF424ABAC
:10E21000DFED5C7AC7F5FA634A4938EE678A1BB2CC
:10E22000FDEEC87ACDED037ABDF90C20120381FB17
:10E230000201D217C2EBA11203FB02F343F30F3327
:10E240003B4407EE903A049BF8EEE77AC3ED037A7D
:10E25000FFF702BBDFF83CA14FF00108DFF838916F
:10E260000AF15A063D4D51461AF8010C0CF058FBC4
:10E27000F8B19AF804109AF8023001EB410E9AF8BE
:10E280000300013B08FA01F105EB8E0E03EB43039B
:10E29000DEF8B4204B4493420BD095F8E0208EF882
:10E2A000B00022EA0101CEF8B430CEF8B87085F89B
:10E2B000E0100AF1060A5645D5D1334B00262E4A06
:10E2C00019460893314D234B0968A5F1B00A1B7814
:10E2D000D2F80090099107936B685BB31F784FB336
:10E2E000AA68A9EB0202002A0ADB01219AF8E020C1
:10E2F00009F5FA70B140A86022EA01028AF8E0202C
:10E30000079ABAB12A7859780432D2B2002940F07B
:10E310008B81039934F91220098B01F1C8008242E4
:10E3200040F376839AF8E0109A7841FA06F3DB0717
:10E3300040F1388401360C35042ECDD1FFF7C8B832
:10E340000CAB0120D34D621078A901208CB20120C2
:10E3500070160120C488012071160120902301202D
:10E36000E1B30120ABAAAAAA50700120E4B30120B6
:10E37000C58801206EB101200C94012080B40120D9
:10E380006436012000007A440073012040240120FB
:10E39000A08801201D730120E0720408CD4D95F87E
:10E3A000AA3053B1069B1B78DA0706D5039BB4F954
:10E3B00006205B8B9A4200F3E8831121C64802F0E5
:10E3C0008CFF002800F0148195F8AE302BB995F839
:10E3D000A83013B93223A5F8AC30012385F8AE304C
:10E3E000FFF70AB81146FFF7F5BB037AC3F16403E0
:10E3F00007EE903AFFF763BB0AF1050178790CF05C
:10E400008FFA00283FF487ABB8F1010F40F0478640
:10E4100007F10D01B87A0CF083FA002840F01A8653
:10E42000AE49F87B0CF07CFA00283FF486ABB8F1DB
:10E43000030F40F01286AA49387D0CF071FA0028CB
:10E4400040F02786A749787E0CF06AFA00283FF44E
:10E4500086ABB8F1050F40F01F86A349B87F0CF0DA
:10E460005FFA002840F0FC85A04997F823000CF0E3
:10E4700057FA00283FF486ABB8F1070F40F09783B6
:10E480009B4997F828000CF04BFA002840F0A08335
:10E49000984997F82D000CF043FA00283FF428A97A
:10E4A000B8F1090F3FF424A9FFF780BB894D049A06
:10E4B000D5F88830D31A002BFEF6A4AE8E4A8F4BC7
:10E4C000527C0398089933F8122095F88C30C5F8DF
:10E4D000881092B2817D013392FBF1F203F00F03B9
:10E4E000C17DE81885F88C3080F8902095F891303F
:10E4F00095F8900095F89F20184495F892300344C1
:10E5000095F89300184495F89430184495F8953090
:10E51000034495F89600184495F89730184495F8F8
:10E520009830034495F89900184495F89A301844A7
:10E5300095F89B30034495F89C00184495F89D305D
:10E54000184495F89E3003441A4442F30B12642A8F
:10E55000A8BF642213B209B1C2F1640307EE903A76
:10E560009FED677A674AF8EEE77A67EE877AFCEE06
:10E57000E77A17EE903A1380FEF744BE0221564820
:10E5800002F0ABFE00283FF471AA3580FEF7E0BF31
:10E5900019F00CFE05E425F040039BB2AB4233803A
:10E5A0003FF40DA8584B02201421FF2218700E20B2
:10E5B00059709A7019F0C8FCFFF701B8338823F03E
:10E5C0000405ADB2AB4235803EF4EFAF4E4B0220B6
:10E5D0001421FF2218700E2059709A7019F0B4FCA3
:10E5E0003588FEF7E2BF05238BF82030FFF74DBBDF
:10E5F00095F8A830002B3EF4FFAE069B1B7813F075
:10E6000001037EF4F9AE012285F8A83085F8A9202F
:10E61000FEF7F2BE3D4991F8008032E52D4D012113
:10E6200085F8A010FEF785BE012900F06B84012358
:10E630009AF8E0200C35B34001361343042E8AF8D3
:10E64000E0307FF449AEFEF743BF9FED317A77EEBD
:10E65000677AFFF791B9069B2E4A1B781060DF0797
:10E6600000F1768295F8A61000297EF4BEAEB5F9C9
:10E67000A430322B7EF7B9AE95F8A2200120572A9C
:10E6800085F8A60000F00E85059B1E6806F00403C1
:10E69000760702D55A2A00F0FC855D2A00F06085D5
:10E6A0005B2A00F0BD855E2A00F0D585562A00F071
:10E6B0003386972A00F03F86A72A40F0188516492E
:10E6C000059B0A781B6842F0040203F004030A70F9
:10E6D000FEF78FBE902301206436012015740120BF
:10E6E0001A7401201F740120247401202974012050
:10E6F0002E7401203374012038AC012054AC012069
:10E7000014AE23415830012014750120C488012023
:10E71000DB0F4940749701209C3A0120B3F5FA7F42
:10E72000FEF663AE95F8A620002A7EF45EAE069B48
:10E7300001211B7885F8A610D80700F120851BF071
:10E74000C9FF059B1B6803F00403FEF752BE47F0A8
:10E750000203BB4233803EF4FEAEC54B02201421BF
:10E76000FF2218700E2059709A7019F0EDFB37884F
:10E77000FEF7F1BE002B3AD057F822605000B345A7
:10E78000FFF4D3ACBB4D5FFA82F92E5C0544002E3A
:10E790003ED0022E4DD16E7806EB860606EB86063D
:10E7A00006F2EE26B6B2032A3ADD36B2BCF1000F0D
:10E7B0003FF4C0AC099D21F81560BAF1000F03D1F8
:10E7C0000C9D022D7FF6B6ACB1F802904FF0010A15
:10E7D0000E88A94D4E44B1F804904E4436B285FBE4
:10E7E0000659A64D2E52A9EBE67636B2A2E41E4695
:10E7F0005000079D47F8225098E4CAB2022A05D972
:10E80000032A62463FF4DEAC0288E9E47246D9E4AA
:10E81000B9F1020F40F27483B9F1030F09D10F9ED1
:10E82000012536B205FA02F90B9D25EA09050B957B
:10E830007CE4265AB7E745F04003AB4233807FF4CF
:10E84000B1AEFEF7BCBE45F004039D4233807FF4B9
:10E85000BDAEFEF7AABEDFED8A7AFFF79DB8F4EEF3
:10E86000C77AF1EE10FA40F3C583DFED865A9FEDCB
:10E87000866AF4EEC66A36EEE57AF1EE10FAF0EE4C
:10E88000476AF6DCDFED816AB4EEE67AF1EE10FA63
:10E8900040F1DD83DFED7B5A9FED7D6AB4EEC67AF1
:10E8A00077EE256AF1EE10FAB0EE667AF6D49FEDB7
:10E8B000797AF4EEC76AF1EE10FA40F383809FEDA7
:10E8C000767A77EE666A66EEA65A9FED745A9FEDE9
:10E8D000746A9FED747AA5EE856A26EEA55AA5EEB8
:10E8E000867AE5EE076AFFF702B86F4A01216F48A2
:10E8F0006F4C0E9011701B216E48069302F0EDFCD8
:10E90000069B00287FF429ACDFF8BCB16A4FDBF826
:10E910000C203B68CBF808309B1AC82B00F2898387
:10E92000059B1F6807F4805760E43946614802F090
:10E93000D4FC00283FF48FAE85F8A7701BF0CAFE08
:10E94000FEF74EBD00215A4835460EE06A7802EBCC
:10E95000820202EB820202F2EE2292B2013120F830
:10E96000022B023599423FF441AC16F811201AB13E
:10E97000022AEBD00288F1E75FFA81FC7246BCF113
:10E98000030FEBD90288E9E700230493FFF76AB984
:10E99000B3F5FA7FFEF629AD95F8A620002A7EF49D
:10E9A00024AD069A0121127885F8A61012EA01001A
:10E9B00000F023831BF01AFB059B1B6803F0040384
:10E9C000FEF717BD9FED3D7AF4EEC76AF1EE10FA3F
:10E9D0007FF579AF9FED2D7A77EE666A73E7384B56
:10E9E00047F6FF77374A1968B5F9A430C96982FB41
:10E9F00001E2C9179211A1EB020E7744BB423EF728
:10EA0000E2AC521A13441BB2A5F8A430FEF7DBBCEB
:10EA1000C8398A4280F28F809AF8E0109A7841FAD9
:10EA200006F3D8073FF586AC524201200A9219F04E
:10EA3000A5FB7B1E0A9A162B00F20D81DFE813F06E
:10EA4000ED010E02D401370224024B02BF01AA01DC
:10EA500093017C0165010B01370250014B02BF019C
:10EA6000AA013A0124010E01F900E100CB0000BF28
:10EA70001475012080B401205655555500240120FD
:10EA800000000000DB0FC940E4CB1641DB0F49C09A
:10EA9000E4CB16C1DB0FC93FDB0F494092E741B918
:10EAA0009730083C15A82ABEC5880120E1B3012093
:10EAB00050700120643601200C940120DB0FC9BF87
:10EAC000843F0120D34D6210A08801200126FEF76B
:10EAD000B3BB3A68DBF81C301344CBF81830FFF7AF
:10EAE00063B913F0E3F9032240F6B8338BF8202022
:10EAF000CBF81C30FFF79CB90A200BF039FF3788A0
:10EB00008146002800F03F82FA0640F14083CE4D56
:10EB100095F8F090B9F1000F7EF45EAD0D2019F07C
:10EB200013FA0123378885F8F030B9F1000F7FF42C
:10EB3000F1A9FEF751BD01229AF8E03009F5FA710A
:10EB4000B240A96023EA02038AF8E030FFF7F2BB83
:10EB5000BE4B1B78002B3EF448AC9BF80330002BD7
:10EB60007EF443AC95F8A7300133DBB2032B85F874
:10EB7000A7307EF63AACB64B5B7813B9002E7EF424
:10EB800034AC1BF033FAFEF72BBC0021B14802F085
:10EB9000A4FB00287FF411AC322385F8AA00A5F865
:10EBA000AC300AE4002A0CBF012002203EE7072314
:10EBB0001A4602EB820289F800301744B978787857
:10EBC00016F006FF069B1D7805F00105FEF790BDC7
:10EBD00008231A46EDE7DAF8E400DFF87C8290F8C3
:10EBE000361098F8023011446429A8BF642121EA44
:10EBF000E17180F83610002B40F0048404F040F8F6
:10EC000015E5DAF8E400DFF8508290F8371098F84C
:10EC100002301144FE29A8BFFE2121EAE17180F8EB
:10EC20003710002BEAD016200BF000FFDAF8E400D2
:10EC3000E4E70998DFF8208241781144B1F5967F26
:10EC4000A8BF4FF4967121EAE171417098F8023043
:10EC5000002B40F0D083DAF8E400CFE7DAF8E400E4
:10EC6000DFF8F48181781144C829A8BFC82121EABE
:10EC7000E171817098F80230002BBFD014200BF0A6
:10EC8000D5FEDAF8E400B9E7DAF8E400DFF8C88185
:10EC900041781144C829A8BFC82121EAE171417017
:10ECA00098F80230002BA9D013200BF0BFFEDAF841
:10ECB000E400A3E7DAF8E400DFF89C81017811446E
:10ECC000C829A8BFC82121EAE171017098F8023073
:10ECD000002B93D012200BF0A9FEDAF8E4008DE7A8
:10ECE000DFF87481099898F8023041791144642959
:10ECF000A8BF642121EAE1714171002BABD00E2045
:10ED00000BF094FEDAF8E40078E7DAF8E400DFF8D4
:10ED10004881017A98F802301144C829A8BFC82157
:10ED200021EAE1710172002B3FF468AF0B200BF078
:10ED30007DFEDAF8E40061E7DAF8E400DFF8188134
:10ED4000C17998F802301144C829A8BFC82121EA26
:10ED5000E171C171002B3FF451AF0A200BF066FE48
:10ED6000DAF8E4004AE7DAF8E400DFF8EC808179C9
:10ED700098F802301144C829A8BFC82121EAE171DE
:10ED80008171002B3FF43AAF09200BF04FFEDAF807
:10ED9000E40033E7DAF8E400DFF8BC80417998F862
:10EDA00002301144C829A8BFC82121EAE17141718C
:10EDB000002B40F01283112F7FF454AF1EE7DAF8D6
:10EDC000E400DFF89480017998F802301144C829F2
:10EDD000A8BFC82121EAE1710171002B40F0F18246
:10EDE000102F7FF455AF09E70999DFF86C800F7990
:10EDF0001744642FA8BF642727EAE7770F710BF049
:10EE00002FFE98F80230002B3FF425AF032039463F
:10EE10000BF00CFEDAF8E400F0E60998DFF8388031
:10EE200001781144FA29A8BFFA2121EAE1710170A1
:10EE300098F80230002B3FF40EAF01200BF0F6FDE6
:10EE4000DAF8E400DAE600BF90230120C48801204C
:10EE5000E03601206436012068B601200998DFF809
:10EE6000B484817811446429A8BF642121EAE17146
:10EE7000817098F80230002B3FF4EDAE02200BF0C9
:10EE8000D5FDDAF8E400B9E60998DFF88884C1799D
:10EE900098F80230114481F30801C171002B3FF44E
:10EEA000DAAE05200BF0C2FDDAF8E400A6E6099B15
:10EEB000DFF86084997998F8020011446429A8BFAA
:10EEC000642121EAE1719971002840F08E820D2FB2
:10EED0007FF408AFBFE6DAF8E400DFF83884C178E1
:10EEE00098F802301144C829A8BFC82121EAE1716D
:10EEF000C170002B40F08A820F2F7FF4DFAE7DE6D9
:10EF00000D9E50E498784FF4966134F91230B3F5C1
:10EF1000617F91FBF0F252DB40F633019942A8BFCA
:10EF200019460C2FA1F5617191FBF2F100F09F8160
:10EF3000182F7FF47CABC9B2C8290B46A8BFC823E1
:10EF4000DAF8E420D8B2D77DB8423FF470ABDB1BCF
:10EF5000DFF8C083D07548BF0733DF1098F8023060
:10EF60000137FFB23BB9002F3FF461AB384619F0CF
:10EF700005F9FFF75CBB18200BF058FDF3E7B0EE86
:10EF8000677AFEF7D1BCFB0600F154810B200BF031
:10EF9000EFFC002840F01181BD0600F16081C84DF2
:10EFA00095F8F030002B3FF4B9ADB9F1000F7EF4C5
:10EFB000B1AFFEF711BBF0EE477AFEF7CABC0C2FDB
:10EFC00040F0328100273946BE4B0A915B78BB4244
:10EFD0003FF42DABDFF83C8338461BF06BFE0A99FB
:10EFE00098F802301BB1C9B20C200BF01FFD01379D
:10EFF000FFB2B8E7B0EE667A44E4B34A126812F49E
:10F00000003240F021811046B0490E5C0C300F2ECA
:10F0100029D00132152AF8D1A3F1FA01059B00226B
:10F020001B68A5F8A41085F8A62003F00403FEF7DA
:10F03000E0B9A74A012113888BF82110059923F024
:10F0400004030F68138007F48057FFF7CFB8F0EE82
:10F05000476A2CE402231A46ABE503231A46A8E5C7
:10F0600006231A46A5E59B4F50003E683EB196F830
:10F0700001E0861801EB860676787645CCD21044FE
:10F08000954E002201EB8001944832803960026085
:10F09000C2E704231A468CE505231A4689E50123B5
:10F0A0001A4686E58E4B4FF47A728E491B68B2FB86
:10F0B000F3F2C2EB4210059B02EB80021B68D20008
:10F0C000A1F8B8201A067EF592A9874A1278970708
:10F0D0007EF58DA9854A127D042A7EF688A916F050
:10F0E0002DFB059B1B6803F00403FEF782B900218A
:10F0F000BB2A109100F05181B72A00F04A81BE2A44
:10F1000000F04581BD2A00F02081792A00F0B58108
:10F110007A2A00F0AB819E2A00F0A2819D2A00F09D
:10F120009881AE2A00F0D981AD2A00F0CF81EF2A74
:10F1300000F0C681FD2A00F0BD81FB2A00F0B481F9
:10F14000FE2A00F0AB81F72A00F0A2817B2A7EF430
:10F150004CA94FF4FA6102201BF040FDFEF745B9BF
:10F16000634B002201206349564D0B602A7019F051
:10F1700005F8059B1B6803F00403FEF73AB9059BED
:10F180005D491B680A6003F00403FEF732B91020E2
:10F190004B4D19F023F8202019F008F85749081FA3
:10F1A00016F044FB564B02221A7095F8F030002BF3
:10F1B00000F00F813788FEF7ADBE524B04995B8992
:10F1C00091ED007A07EE903AB0EEC77AF8EEE77A62
:10F1D000B4EEE77AF1EE10FA7FF5DEAE91ED017A4A
:10F1E000B0EEC77AF4EEC77AF1EE10FA7FF7D4AE3C
:10F1F000BB063FF5D4AE324D202018F0EFFFD8F813
:10F2000004202946D8F8003005F1E80041F8EC2F39
:10F21000C5F8E83016F00AFB394B01221A70C4E732
:10F22000394B012202209EE7182F7FF400AA00210B
:10F230000B4685E6102018F0B9FF314B378883F86C
:10F2400000904FF00109A1E6304A1278032A00F03D
:10F25000B3800246D8E62E4B0222032083E720200B
:10F26000174D18F0A3FF264B00221A709DE7CFB26E
:10F27000AAE6002E3EF430A8114D95F8A130002BDF
:10F280003EF45CA818F042FE002385F8A130FEF79A
:10F2900055B895F8A820002A40F0D58095F8AA30F6
:10F2A00083F0010385F8AA30002B40F0C3800C20C6
:10F2B00018F04AFE059B1B6803F00403FEF799B89B
:10F2C00090230120548801201073012034940408F5
:10F2D0006EB1012020230120742301207823012016
:10F2E00068A9012068A101209C3A0120A03A0120D0
:10F2F0004CB501206088012074970120443B012017
:10F30000FE3A01209C3B01209AB50120D82D012016
:10F31000E8B5012068B6012020F056F901F02CFA7A
:10F3200020F03AF9FDF770FD012018F027FF95F85D
:10F33000A220FFF7BEB9059B4FF4C8716A4A1B684B
:10F34000118003F00403FEF754B84FF6FE73674ACA
:10F35000D089968901443344D181938120F034F9D6
:10F3600001F00AFA20F018F9FDF74EFD012018F01F
:10F3700005FFB5F8A420059B0021FA3A1B6885F823
:10F38000A61003F00403A5F8A420FEF732B8022368
:10F39000DDE70B464FF6FE71D9E70B460221D6E7B3
:10F3A0001AF024FE524D002385F8A130FDF7C6BFA8
:10F3B00003230493FEF7C8BD18F0A8FDB5F9A430E7
:10F3C0002AE610200A920BF031FBDAF8E4000A9AE0
:10F3D00006E54FF00109FFF7A1BB11200A920BF0DF
:10F3E00025FBDAF8E4000A9AE5E40D200A920BF016
:10F3F0001DFB0A9A6BE515200BF018FBDAF8E40008
:10F40000FFF7FCBB17200BF011FB24E40F200A923E
:10F410000BF00CFBDAF8E4000A9A6DE5002B3FF4E0
:10F420002BAF34494FF47A70334A096800FB031359
:10F43000136021E70B2018F087FD059B1B6803F084
:10F440000403FDF7D6BF85F8A81085F8A900FDF7DD
:10F45000D0BF0021FF2025F08DF895F8A22060E6AE
:10F46000012025F087F895F8A22057E6234A137A61
:10F4700043F001031372FDF7B8BF204A137A23F05B
:10F4800001031372FDF7B1BF03230493FEF790BC91
:10F49000002104201BF0A2FBFDF7A7BF00210320E1
:10F4A0001BF09CFBFDF7A1BF002102201BF096FB87
:10F4B000FDF79BBF002101201BF090FBFDF795BFDE
:10F4C000002108461BF08AFBFDF78FBFFF210020BB
:10F4D00025F050F895F8A22029E60121002025F01A
:10F4E00049F895F8A2201FE652370120C4360120C2
:10F4F000902301200C940120709701203C3F0120B3
:10F500000B4B30B503F1140493F90020043313F8C6
:10F51000035C072AC8BF143A81180D7313F8025C04
:10F52000855413F8012CA3420A76EDD130BD00BFFB
:10F530002873040803682DE9F041DF691FB13B46D9
:10F54000BDE8F0411847002A164611DD04460D4675
:10F550000E4400E023689B68204698470028F9D0B5
:10F560002368204615F8011B1B689847AE42F1D16D
:10F57000BDE8F081002325212422017042708370B0
:10F58000C3707047094B03F10C0110B593F90020CB
:10F59000043313F8034C8454024413F8024C1471DE
:10F5A00013F8014C8B421472F0D110BD3C73040867
:10F5B000002830B41FDB0928044622DD012303EBB9
:10F5C00083035B00B0FBF3F2092AF8D87BB10F4D3F
:10F5D000A5FB0320B4FBF3F2092A03FB1244CCBFC2
:10F5E00057233023134401F8013BC308F0D1002313
:10F5F00030BC0B7070472D234042013101F8013CB3
:10F60000D9E7303001F8010BF1E700BFCDCCCCCC0D
:10F61000884230B44FF001042ED301FB04F4B0FB58
:10F62000F4F58D42F9D284B1AAB901E0B0FBF4F54A
